
 Start  Stop   Length Name               Class

 00000H 00595H 00596H _TEXT              CODE
 00596H 00596H 00000H MONITOR_TEXT       CODE
 00596H 00596H 00000H MONITORCSIP_TEXT   CODE
 00596H 0068CH 000F7H FORMULA_TEXT       CODE
 0068DH 0068DH 00000H DEBUG_TEXT         CODE
 00690H 02F3FH 028B0H AMXCODE            CODE
 02F40H 03012H 000D3H CONFIGDATA_TEXT    CODE
 03013H 04608H 015F6H DATAMGR_TEXT       CODE
 04609H 049D3H 003CBH INTERRUPTCTRL_TEXT CODE
 049D4H 04A11H 0003EH MAIN_TEXT          CODE
 04A12H 04D57H 00346H MEMORY_TEXT        CODE
 04D58H 050CDH 00376H SYSINIT_TEXT       CODE
 050CEH 05C33H 00B66H UISTATEMGR_TEXT    CODE
 05C34H 0A18FH 0455CH PWSRCCONTROL_TEXT  CODE
 0A190H 0A6AAH 0051BH PWPERIODIC_TEXT    CODE
 0A6ABH 0AC1EH 00574H PWROS_TEXT         CODE
 0AC1FH 0ADADH 0018FH DVRS232_TEXT       CODE
 0ADAEH 0BBA7H 00DFAH DVOUTPUTSCALER_TEXT CODE
 0BBA8H 0BF94H 003EDH DVIMAGEMEMORY_TEXT CODE
 0BF95H 0C319H 00385H DV24CXX_TEXT       CODE
 0C31AH 0DB8AH 01871H DVDPORT_TEXT       CODE
 0DB8BH 12224H 0469AH DVINPUTPORT_TEXT   CODE
 12225H 12857H 00633H DVCLKGENPG18E1_TEXT CODE
 12858H 14CD5H 0247EH DVAD9883_TEXT      CODE
 14CD6H 17522H 0284DH DVVPC3230_TEXT     CODE
 17523H 1781DH 002FBH DVTMDSGENERIC_TEXT CODE
 1781EH 19369H 01B4CH DVPW1230_TEXT      CODE
 1936AH 1A022H 00CB9H DVZ86129_TEXT      CODE
 1A023H 1A6BEH 0069CH DVTDA9851_TEXT     CODE
 1A6BFH 1A8FCH 0023EH DVSWITCHER_SHASTA_II_TEXT CODE
 1A8FDH 1B077H 0077BH DVCOLORSPACE_TEXT  CODE
 1B078H 1C0C9H 01052H DVFI1256_TEXT      CODE
 1C0CAH 1C481H 003B8H DVTDA9885_TEXT     CODE
 1C482H 1D1C6H 00D45H DVNJW1144_TEXT     CODE
 1D1C7H 1D7D3H 0060DH DVDRIVERSERVICE_TEXT CODE
 1D7D4H 1D847H 00074H PWCRC_TEXT         CODE
 1D848H 1FB01H 022BAH PWOEM_TEXT         CODE
 1FB02H 1FCEEH 001EDH HLINT_TEXT         CODE
 1FCEFH 1FCFEH 00010H PWISPCORE_TEXT     CODE
 1FCFFH 209CDH 00CCFH PWMISC_TEXT        CODE
 209CEH 21065H 00698H HLREGISTERS_TEXT   CODE
 21066H 23475H 02410H HLAYER111_TEXT     CODE
 23476H 25660H 021EBH PWHOST_TEXT        CODE
 25661H 25F7CH 0091CH UIBHVVARIABLES_TEXT CODE
 25F7DH 27FB6H 0203AH HLSCALER_TEXT      CODE
 27FB7H 293C0H 0140AH HLDISPP_TEXT       CODE
 293C1H 29812H 00452H HLTIMERS_TEXT      CODE
 29813H 29BB6H 003A4H HLINIT_TEXT        CODE
 29BB7H 29DA5H 001EFH HLWAITSTATE_TEXT   CODE
 29DA6H 2A5DBH 00836H DVGPIO_TEXT        CODE
 2A5DCH 2AA24H 00449H DVOEMINTERFACE_TEXT CODE
 2AA25H 2C637H 01C13H PWDPMS_TEXT        CODE
 2C638H 2E6F8H 020C1H PWOSD_TEXT         CODE
 2E6F9H 2E7DCH 000E4H HLGENCTL_TEXT      CODE
 2E7DDH 2E96FH 00193H PWINPUT_TEXT       CODE
 2E970H 2F479H 00B0AH PWOPERATIONS_TEXT  CODE
 2F47AH 2F729H 002B0H UIEVENTSCAN_TEXT   CODE
 2F72AH 31403H 01CDAH UIBHVMENU_TEXT     CODE
 31404H 318B7H 004B4H UICONTROLS_TEXT    CODE
 318B8H 3316CH 018B5H UICTLMENU_TEXT     CODE
 3316DH 33754H 005E8H UIDRAWOBJECT_TEXT  CODE
 33755H 33CB8H 00564H UIOSDSIZE_TEXT     CODE
 33CB9H 33FA1H 002E9H UITRACKOPS_TEXT    CODE
 33FA2H 348FEH 0095DH UIBHVCONDITIONMGR_TEXT CODE
 348FFH 34F1BH 0061DH UIBHVDYNAMICMGR_TEXT CODE
 34F1CH 35E6EH 00F53H PWSRCINPUT_TEXT    CODE
 35E6FH 3665FH 007F1H PWSRCAUTO_TEXT     CODE
 36660H 376D1H 01072H PWSRCAUTOCALIBRATE_TEXT CODE
 376D2H 3A6E5H 03014H PWSRCSETTINGS_TEXT CODE
 3A6E6H 3BB4FH 0146AH PWSRCDETECTION_TEXT CODE
 3BB50H 3D814H 01CC5H PWSRCDISPLAY_TEXT  CODE
 3D815H 3DCACH 00498H PWSRCTEST_TEXT     CODE
 3DCADH 3E42DH 00781H HLOSDLOC_TEXT      CODE
 3E42EH 3E84EH 00421H PWSRCUTIL_TEXT     CODE
 3E84FH 40799H 01F4BH PWSRCTV_TEXT       CODE
 4079AH 40C3BH 004A2H HLRECT_TEXT        CODE
 40C3CH 411DEH 005A3H HLSERIAL_TEXT      CODE
 411DFH 41BB9H 009DBH DVSCALERMODE_TEXT  CODE
 41BBAH 4207AH 004C1H DVSCALERZOOM_TEXT  CODE
 4207BH 4228CH 00212H DVSCALERFILTER_TEXT CODE
 4228DH 4281CH 00590H DVSCALERNLOPS_TEXT CODE
 4281DH 42DC5H 005A9H HLVIDEO_TEXT       CODE
 42DC6H 432AAH 004E5H DVSCALERPRIV_TEXT  CODE
 432ABH 4389EH 005F4H HLIMGMEM_TEXT      CODE
 4389FH 441A4H 00906H HLGPORT_TEXT       CODE
 441A5H 4436AH 001C6H HLDPORTISP_TEXT    CODE
 4436BH 4476EH 00404H HLAUTO_TEXT        CODE
 4476FH 4488AH 0011CH HLGPORTISP_TEXT    CODE
 4488BH 449A8H 0011EH HLVPORTISP_TEXT    CODE
 449A9H 44CD3H 0032BH MYAPI_TEXT         CODE
 44CD4H 44FA9H 002D6H PWSRCSYNCMONITOR_TEXT CODE
 44FAAH 455CAH 00621H DVKEYPADTASK_TEXT  CODE
 455CBH 45811H 00247H DVOEMPWM16_TEXT    CODE
 45812H 461D6H 009C5H HLOSD_TEXT         CODE
 461D7H 464AAH 002D4H HLINFRED_TEXT      CODE
 464ABH 46552H 000A8H HLDECODE_TEXT      CODE
 46553H 46E07H 008B5H DV2WIRE_TEXT       CODE
 46E08H 47606H 007FFH DVLED_TEXT         CODE
 47607H 47657H 00051H DVOEMLAMP_BACKLIGHT_TEXT CODE
 47658H 47670H 00019H DVOEMUNITPOWER_TEXT CODE
 47671H 483EFH 00D7FH PWBLTMAP_TEXT      CODE
 483F0H 49347H 00F58H PWOPPRINTF_TEXT    CODE
 49348H 49480H 00139H DVIRREMOTETASK_TEXT CODE
 49481H 49759H 002D9H PWOSDOPS_TEXT      CODE
 4975AH 49983H 0022AH UIBHVINSPECT_TEXT  CODE
 49984H 4A008H 00685H UIBHVITERATORS_TEXT CODE
 4A009H 4A4F4H 004ECH UICTLGAUGE_TEXT    CODE
 4A4F5H 4A719H 00225H UICTLNUMBER_TEXT   CODE
 4A71AH 4A86EH 00155H UICTLBUTTON_TEXT   CODE
 4A86FH 4A9E2H 00174H UICTLTEXT_TEXT     CODE
 4A9E3H 4B37EH 0099CH UICTLDYNAMIC_TEXT  CODE
 4B37FH 4B4EEH 00170H UICTLBORDER_TEXT   CODE
 4B4EFH 4B4F0H 00002H UIPANEMGR_TEXT     CODE
 4B4F1H 4B8DCH 003ECH PWSRCAUTOPOSITION_TEXT CODE
 4B8DDH 4C818H 00F3CH PWSRCAUTOFREQPHASE_TEXT CODE
 4C819H 4CD71H 00559H PWSRCAUTOBRIGHTNESS_TEXT CODE
 4CD72H 4D390H 0061FH HLHICOLOR_TEXT     CODE
 4D391H 4D84FH 004BFH HLPRIV_TEXT        CODE
 4D850H 4DD02H 004B3H DVINFRED_TEXT      CODE
 4DD03H 4DD93H 00091H DVKEYPADDIRECT_TEXT CODE
 4DDA0H 4DDABH 0000CH _INIT_             INITDATA
 4DDACH 4DDACH 00000H _INITEND_          INITDATA
 4DDB0H 4DDB0H 00000H _EXIT_             EXITDATA
 4DDB0H 4DDBFH 00010H _EXITEND_          EXITDATA
 4DDC0H 4DDC0H 00000H _RD                ROMDATA
 4DDC0H 4DDCFH 00010H _ERD               ENDROMDATA
 4DDD0H 4DDD0H 00000H _BRFD              ROMFARDATA
 4DDD0H 4DDDFH 00010H _ERFD              ENDROMFARDATA
 4DDE0H 4DDE0H 00000H _BRFUNC            ROMFUNCTION
 4DDE0H 4DDEFH 00010H _ERFUNC            ENDROMFUNCTION
 4DDF0H 4DDF0H 00000H _BFUNC             RAMFUNCTION
 4DDF0H 4DDFFH 00010H _EFUNC             ENDRAMFUNCTION
 4DE00H 4E409H 0060AH _DATA              DATA
 4E40AH 4E40AH 00000H _CVTSEG            DATA
 4E40AH 4E40AH 00000H _SCNSEG            DATA
 4E410H 4E412H 00003H AMXDGRP            DATA
 4E414H 4E43BH 00028H AMXVAR             DATA
 4E440H 4FA57H 01618H _BSS               BSS
 4FA60H 4FA60H 00000H _NVRAM             NVRAM
 4FA60H 4FA6FH 00010H _EDATA             EDATA
 4FA70H 4FB6FH 00100H _STACK             STACK
 4FB70H 4FB7FH 00010H _ESTACK            STACK
 4FB80H 4FB80H 00000H _BFD               FAR_DATA
 4FB80H 4FB8FH 00010H _EFD               ENDFAR_DATA
 4FB90H 4FB90H 00000H _BFC               FAR_CONST
 4FB90H 4FC65H 000D6H CONFIGDATA5_CONST  FAR_CONST
 4FC70H 4FCD5H 00066H CONFIGDATA6_CONST  FAR_CONST
 4FCE0H 4FD5DH 0007EH INTERRUPTCTRL5_CONST FAR_CONST
 4FD60H 4FD73H 00014H DVRS2325_CONST     FAR_CONST
 4FD80H 4FD93H 00014H DVOUTPUTSCALER5_CONST FAR_CONST
 4FDA0H 4FDB3H 00014H DVIMAGEMEMORY5_CONST FAR_CONST
 4FDC0H 4FDD3H 00014H DV24CXX5_CONST     FAR_CONST
 4FDE0H 4FDF3H 00014H DVDPORT5_CONST     FAR_CONST
 4FE00H 4FE13H 00014H DVINPUTPORT5_CONST FAR_CONST
 4FE20H 4FE9FH 00080H DVCLKGENPG18E15_CONST FAR_CONST
 4FEA0H 4FEA3H 00004H DVAD98835_CONST    FAR_CONST
 4FEB0H 4FEC7H 00018H DVAD98836_CONST    FAR_CONST
 4FED0H 4FEE7H 00018H DVAD98837_CONST    FAR_CONST
 4FEF0H 4FEFFH 00010H DVVPC32305_CONST   FAR_CONST
 4FF00H 4FF20H 00021H DVVPC32306_CONST   FAR_CONST
 4FF30H 4FFF7H 000C8H DVVPC32307_CONST   FAR_CONST
 50000H 50003H 00004H DVVPC32308_CONST   FAR_CONST
 50010H 50013H 00004H DVVPC32309_CONST   FAR_CONST
 50020H 50023H 00004H DVVPC323010_CONST  FAR_CONST
 50030H 50033H 00004H DVVPC323011_CONST  FAR_CONST
 50040H 50043H 00004H DVVPC323012_CONST  FAR_CONST
 50050H 50053H 00004H DVVPC323013_CONST  FAR_CONST
 50060H 50063H 00004H DVVPC323014_CONST  FAR_CONST
 50070H 50077H 00008H DVVPC323015_CONST  FAR_CONST
 50080H 5008FH 00010H DVVPC323016_CONST  FAR_CONST
 50090H 50097H 00008H DVVPC323017_CONST  FAR_CONST
 500A0H 500A6H 00007H DVVPC323018_CONST  FAR_CONST
 500B0H 500B6H 00007H DVVPC323019_CONST  FAR_CONST
 500C0H 500C6H 00007H DVVPC323020_CONST  FAR_CONST
 500D0H 500D6H 00007H DVVPC323021_CONST  FAR_CONST
 500E0H 500FAH 0001BH DVVPC323022_CONST  FAR_CONST
 50100H 50113H 00014H DVTMDSGENERIC5_CONST FAR_CONST
 50120H 50177H 00058H DVPW12305_CONST    FAR_CONST
 50180H 501BDH 0003EH DVPW12306_CONST    FAR_CONST
 501C0H 50221H 00062H DVPW12307_CONST    FAR_CONST
 50230H 5028FH 00060H DVPW12308_CONST    FAR_CONST
 50290H 50293H 00004H DVPW12309_CONST    FAR_CONST
 502A0H 502A3H 00004H DVPW123010_CONST   FAR_CONST
 502B0H 502B3H 00004H DVPW123011_CONST   FAR_CONST
 502C0H 502C3H 00004H DVPW123012_CONST   FAR_CONST
 502D0H 502D3H 00004H DVPW123013_CONST   FAR_CONST
 502E0H 502ECH 0000DH DVPW123014_CONST   FAR_CONST
 502F0H 502FCH 0000DH DVPW123015_CONST   FAR_CONST
 50300H 50320H 00021H DVPW123016_CONST   FAR_CONST
 50330H 50343H 00014H DVZ861295_CONST    FAR_CONST
 50350H 50363H 00014H DVTDA98515_CONST   FAR_CONST
 50370H 50383H 00014H DVSWITCHER_SHASTA_II5_CONST FAR_CONST
 50390H 503E3H 00054H DVCOLORSPACE5_CONST FAR_CONST
 503F0H 5043FH 00050H DVCOLORSPACE6_CONST FAR_CONST
 50440H 50465H 00026H DVFI12565_CONST    FAR_CONST
 50470H 50483H 00014H DVTDA98855_CONST   FAR_CONST
 50490H 504F4H 00065H DVNJW11445_CONST   FAR_CONST
 50500H 50564H 00065H DVNJW11446_CONST   FAR_CONST
 50570H 505D4H 00065H DVNJW11447_CONST   FAR_CONST
 505E0H 50644H 00065H DVNJW11448_CONST   FAR_CONST
 50650H 50655H 00006H DVNJW11449_CONST   FAR_CONST
 50660H 506DDH 0007EH DVNJW114410_CONST  FAR_CONST
 506E0H 507DFH 00100H PWCRC5_CONST       FAR_CONST
 507E0H 508DFH 00100H PWCRC6_CONST       FAR_CONST
 508E0H 508E8H 00009H PWOEM5_CONST       FAR_CONST
 508F0H 50953H 00064H PWOEM6_CONST       FAR_CONST
 50960H 50977H 00018H HLINT5_CONST       FAR_CONST
 50980H 50997H 00018H HLINT6_CONST       FAR_CONST
 509A0H 509B7H 00018H HLINT7_CONST       FAR_CONST
 509C0H 509C7H 00008H HLINT8_CONST       FAR_CONST
 509D0H 509DDH 0000EH HLINT9_CONST       FAR_CONST
 509E0H 509F7H 00018H HLINT10_CONST      FAR_CONST
 50A00H 50A11H 00012H HLREGISTERS5_CONST FAR_CONST
 50A20H 50A29H 0000AH PWHOST5_CONST      FAR_CONST
 50A30H 50A63H 00034H PWHOST6_CONST      FAR_CONST
 50A70H 50E8FH 00420H PWOPERATIONS5_CONST FAR_CONST
 50E90H 50EFDH 0006EH PWOPERATIONS6_CONST FAR_CONST
 50F00H 50F23H 00024H PWSRCAUTOCALIBRATE5_CONST FAR_CONST
 50F30H 50FA7H 00078H PWSRCSETTINGS5_CONST FAR_CONST
 50FB0H 51045H 00096H PWSRCDISPLAY5_CONST FAR_CONST
 51050H 510AFH 00060H PWSRCDISPLAY6_CONST FAR_CONST
 510B0H 510EBH 0003CH PWSRCTV5_CONST     FAR_CONST
 510F0H 51103H 00014H PWSRCTV6_CONST     FAR_CONST
 51110H 51110H 00001H PWSRCTV7_CONST     FAR_CONST
 51120H 51121H 00002H PWSRCTV8_CONST     FAR_CONST
 51130H 51157H 00028H MYAPI5_CONST       FAR_CONST
 51160H 5116FH 00010H _EFC               ENDFAR_CONST
 51170H 51170H 00000H _BFB               FAR_BSS
 51170H 5117FH 00010H _EFB               ENDFAR_BSS
 51180H 51180H 00000H _FARHEAP           FAR_HEAP
 51180H 5118FH 00010H _EFH               ENDFAR_HEAP
 51190H 5119FH 00010H INITIALENTRY       INITIALENTRY
 511A0H 5212FH 00F90H AMXDATA            AMXD
 52130H 521F9H 000CAH AMXMES             AMXD
 52200H 5273FH 00540H AMXSTAK            AMXS
 52740H 52BBFH 00480H @T@S1              AMXS
 52BC0H 5307FH 004C0H @T@S2              AMXS
 53080H 53373H 002F4H @T@S3              AMXS
 53374H 53374H 00000H AMXCODL            
 53374H 53374H 00000H AMXCODP            PROG
 53374H 53374H 00000H AMXCODT            TEXT


Detailed map of segments

 0000:0000 0107 C=CODE   S=_TEXT          G=(none)   M=c0         ACBP=68
 0000:0110 0000 C=CODE   S=_TEXT          G=(none)   M=inientry   ACBP=68
 0000:0110 0083 C=CODE   S=_TEXT          G=(none)   M=exit       ACBP=28
 0000:0193 0018 C=CODE   S=_TEXT          G=(none)   M=noxx       ACBP=28
 0000:01AC 0050 C=CODE   S=_TEXT          G=(none)   M=fardata    ACBP=48
 0000:01FC 0044 C=CODE   S=_TEXT          G=(none)   M=farbss     ACBP=48
 0000:0240 00AE C=CODE   S=_TEXT          G=(none)   M=h_ldiv     ACBP=28
 0000:02EE 0017 C=CODE   S=_TEXT          G=(none)   M=f_lxmul    ACBP=28
 0000:0305 0021 C=CODE   S=_TEXT          G=(none)   M=h_lursh    ACBP=28
 0000:0326 0021 C=CODE   S=_TEXT          G=(none)   M=h_llsh     ACBP=28
 0000:0347 002D C=CODE   S=_TEXT          G=(none)   M=atexit     ACBP=28
 0000:0374 0035 C=CODE   S=_TEXT          G=(none)   M=pcpprtl    ACBP=48
 0000:03A9 0032 C=CODE   S=_TEXT          G=(none)   M=h_psbp     ACBP=28
 0000:03DB 001C C=CODE   S=_TEXT          G=(none)   M=f_scopy    ACBP=28
 0000:03F7 0020 C=CODE   S=_TEXT          G=(none)   M=h_lrsh     ACBP=28
 0000:0417 0086 C=CODE   S=_TEXT          G=(none)   M=atol       ACBP=28
 0000:049D 0028 C=CODE   S=_TEXT          G=(none)   M=labs       ACBP=28
 0000:04C5 0038 C=CODE   S=_TEXT          G=(none)   M=strncmp    ACBP=28
 0000:04FE 0005 C=CODE   S=_TEXT          G=(none)   M=term       ACBP=48
 0000:0503 0000 C=CODE   S=_TEXT          G=(none)   M=ctype      ACBP=28
 0000:0503 0093 C=CODE   S=_TEXT          G=(none)   M=h_pada     ACBP=28
 0059:0006 0000 C=CODE   S=MONITOR_TEXT   G=(none)   M=monitor    ACBP=28
 0059:0006 0000 C=CODE   S=MONITORCSIP_TEXT G=(none)   M=monitorcsip ACBP=28
 0059:0006 00F7 C=CODE   S=FORMULA_TEXT   G=(none)   M=formula    ACBP=28
 0068:000D 0000 C=CODE   S=DEBUG_TEXT     G=(none)   M=debug      ACBP=28
 0069:0000 01B0 C=CODE   S=AMXCODE        G=(none)   M=romcfg     ACBP=68
 0069:01B0 0000 C=CODE   S=AMXCODE        G=(none)   M=AJ831PRF   ACBP=68
 0069:01B0 02F5 C=CODE   S=AMXCODE        G=(none)   M=aa831sm    ACBP=28
 0069:04A5 02E7 C=CODE   S=AMXCODE        G=(none)   M=aa831em    ACBP=28
 0069:078C 04AB C=CODE   S=AMXCODE        G=(none)   M=aa831mma   ACBP=28
 0069:0C37 0019 C=CODE   S=AMXCODE        G=(none)   M=aj831kk    ACBP=28
 0069:0C50 003B C=CODE   S=AMXCODE        G=(none)   M=aj831ki    ACBP=28
 0069:0C8B 0065 C=CODE   S=AMXCODE        G=(none)   M=aj831uc    ACBP=28
 0069:0CF0 00B6 C=CODE   S=AMXCODE        G=(none)   M=aj831mma   ACBP=28
 0069:0DA6 00D8 C=CODE   S=AMXCODE        G=(none)   M=aa831kx    ACBP=28
 0069:0E7E 044D C=CODE   S=AMXCODE        G=(none)   M=aa831kc    ACBP=28
 0069:12CB 0441 C=CODE   S=AMXCODE        G=(none)   M=aa831ka    ACBP=28
 0069:170C 064C C=CODE   S=AMXCODE        G=(none)   M=aa831kb    ACBP=28
 0069:1D58 014C C=CODE   S=AMXCODE        G=(none)   M=aa831kk    ACBP=28
 0069:1EA4 008D C=CODE   S=AMXCODE        G=(none)   M=aj831kc    ACBP=28
 0069:1F31 0067 C=CODE   S=AMXCODE        G=(none)   M=aj831em    ACBP=28
 0069:1F98 0056 C=CODE   S=AMXCODE        G=(none)   M=aj831kkr   ACBP=28
 0069:1FEE 0134 C=CODE   S=AMXCODE        G=(none)   M=aj831kb    ACBP=28
 0069:2122 0095 C=CODE   S=AMXCODE        G=(none)   M=aj831sm    ACBP=28
 0069:21B7 0016 C=CODE   S=AMXCODE        G=(none)   M=aj831kd    ACBP=28
 0069:21CD 000D C=CODE   S=AMXCODE        G=(none)   M=aj831kf    ACBP=28
 0069:21DA 0064 C=CODE   S=AMXCODE        G=(none)   M=aa831mmb   ACBP=28
 0069:223E 02E9 C=CODE   S=AMXCODE        G=(none)   M=aa831ki    ACBP=28
 0069:2527 00E6 C=CODE   S=AMXCODE        G=(none)   M=aa831kf    ACBP=28
 0069:260D 0121 C=CODE   S=AMXCODE        G=(none)   M=aa831kkr   ACBP=28
 0069:272E 017B C=CODE   S=AMXCODE        G=(none)   M=aa831kd    ACBP=28
 0069:28A9 0007 C=CODE   S=AMXCODE        G=(none)   M=aa831kkx   ACBP=28
 02F4:0000 00D3 C=CODE   S=CONFIGDATA_TEXT G=(none)   M=configdata ACBP=28
 0301:0003 15F6 C=CODE   S=DATAMGR_TEXT   G=(none)   M=datamgr    ACBP=28
 0460:0009 03CB C=CODE   S=INTERRUPTCTRL_TEXT G=(none)   M=interruptctrl ACBP=28
 049D:0004 003E C=CODE   S=MAIN_TEXT      G=(none)   M=main       ACBP=28
 04A1:0002 0346 C=CODE   S=MEMORY_TEXT    G=(none)   M=memory     ACBP=28
 04D5:0008 0376 C=CODE   S=SYSINIT_TEXT   G=(none)   M=sysinit    ACBP=28
 050C:000E 0B66 C=CODE   S=UISTATEMGR_TEXT G=(none)   M=uistatemgr ACBP=28
 05C3:0004 455C C=CODE   S=PWSRCCONTROL_TEXT G=(none)   M=pwsrccontrol ACBP=28
 0A19:0000 051B C=CODE   S=PWPERIODIC_TEXT G=(none)   M=pwperiodic ACBP=28
 0A6A:000B 0574 C=CODE   S=PWROS_TEXT     G=(none)   M=pwros      ACBP=28
 0AC1:000F 018F C=CODE   S=DVRS232_TEXT   G=(none)   M=dvrs232    ACBP=28
 0ADA:000E 0DFA C=CODE   S=DVOUTPUTSCALER_TEXT G=(none)   M=dvoutputscaler ACBP=28
 0BBA:0008 03ED C=CODE   S=DVIMAGEMEMORY_TEXT G=(none)   M=dvimagememory ACBP=28
 0BF9:0005 0385 C=CODE   S=DV24CXX_TEXT   G=(none)   M=dv24cxx    ACBP=28
 0C31:000A 1871 C=CODE   S=DVDPORT_TEXT   G=(none)   M=dvdport    ACBP=28
 0DB8:000B 469A C=CODE   S=DVINPUTPORT_TEXT G=(none)   M=dvinputport ACBP=28
 1222:0005 0633 C=CODE   S=DVCLKGENPG18E1_TEXT G=(none)   M=dvclkgenpg18e1 ACBP=28
 1285:0008 247E C=CODE   S=DVAD9883_TEXT  G=(none)   M=dvad9883   ACBP=28
 14CD:0006 284D C=CODE   S=DVVPC3230_TEXT G=(none)   M=dvvpc3230  ACBP=28
 1752:0003 02FB C=CODE   S=DVTMDSGENERIC_TEXT G=(none)   M=dvtmdsgeneric ACBP=28
 1781:000E 1B4C C=CODE   S=DVPW1230_TEXT  G=(none)   M=dvpw1230   ACBP=28
 1936:000A 0CB9 C=CODE   S=DVZ86129_TEXT  G=(none)   M=dvz86129   ACBP=28
 1A02:0003 069C C=CODE   S=DVTDA9851_TEXT G=(none)   M=dvtda9851  ACBP=28
 1A6B:000F 023E C=CODE   S=DVSWITCHER_SHASTA_II_TEXT G=(none)   M=dvswitcher_shasta_ii ACBP=28
 1A8F:000D 077B C=CODE   S=DVCOLORSPACE_TEXT G=(none)   M=dvcolorspace ACBP=28
 1B07:0008 1052 C=CODE   S=DVFI1256_TEXT  G=(none)   M=dvfi1256   ACBP=28
 1C0C:000A 03B8 C=CODE   S=DVTDA9885_TEXT G=(none)   M=dvtda9885  ACBP=28
 1C48:0002 0D45 C=CODE   S=DVNJW1144_TEXT G=(none)   M=dvnjw1144  ACBP=28
 1D1C:0007 060D C=CODE   S=DVDRIVERSERVICE_TEXT G=(none)   M=dvdriverservice ACBP=28
 1D7D:0004 0074 C=CODE   S=PWCRC_TEXT     G=(none)   M=pwcrc      ACBP=28
 1D84:0008 22BA C=CODE   S=PWOEM_TEXT     G=(none)   M=pwoem      ACBP=28
 1FB0:0002 01ED C=CODE   S=HLINT_TEXT     G=(none)   M=hlint      ACBP=28
 1FCE:000F 0010 C=CODE   S=PWISPCORE_TEXT G=(none)   M=pwispcore  ACBP=28
 1FCF:000F 0CCF C=CODE   S=PWMISC_TEXT    G=(none)   M=pwmisc     ACBP=28
 209C:000E 0698 C=CODE   S=HLREGISTERS_TEXT G=(none)   M=hlregisters ACBP=28
 2106:0006 2410 C=CODE   S=HLAYER111_TEXT G=(none)   M=hlayer111  ACBP=28
 2347:0006 21EB C=CODE   S=PWHOST_TEXT    G=(none)   M=pwhost     ACBP=28
 2566:0001 091C C=CODE   S=UIBHVVARIABLES_TEXT G=(none)   M=uibhvvariables ACBP=28
 25F7:000D 203A C=CODE   S=HLSCALER_TEXT  G=(none)   M=hlscaler   ACBP=28
 27FB:0007 140A C=CODE   S=HLDISPP_TEXT   G=(none)   M=hldispp    ACBP=28
 293C:0001 0452 C=CODE   S=HLTIMERS_TEXT  G=(none)   M=hltimers   ACBP=28
 2981:0003 03A4 C=CODE   S=HLINIT_TEXT    G=(none)   M=hlinit     ACBP=28
 29BB:0007 01EF C=CODE   S=HLWAITSTATE_TEXT G=(none)   M=hlwaitstate ACBP=28
 29DA:0006 0836 C=CODE   S=DVGPIO_TEXT    G=(none)   M=dvgpio     ACBP=28
 2A5D:000C 0449 C=CODE   S=DVOEMINTERFACE_TEXT G=(none)   M=dvoeminterface ACBP=28
 2AA2:0005 1C13 C=CODE   S=PWDPMS_TEXT    G=(none)   M=pwdpms     ACBP=28
 2C63:0008 20C1 C=CODE   S=PWOSD_TEXT     G=(none)   M=pwosd      ACBP=28
 2E6F:0009 00E4 C=CODE   S=HLGENCTL_TEXT  G=(none)   M=hlgenctl   ACBP=28
 2E7D:000D 0193 C=CODE   S=PWINPUT_TEXT   G=(none)   M=pwinput    ACBP=28
 2E97:0000 0B0A C=CODE   S=PWOPERATIONS_TEXT G=(none)   M=pwoperations ACBP=28
 2F47:000A 02B0 C=CODE   S=UIEVENTSCAN_TEXT G=(none)   M=uieventscan ACBP=28
 2F72:000A 1CDA C=CODE   S=UIBHVMENU_TEXT G=(none)   M=uibhvmenu  ACBP=28
 3140:0004 04B4 C=CODE   S=UICONTROLS_TEXT G=(none)   M=uicontrols ACBP=28
 318B:0008 18B5 C=CODE   S=UICTLMENU_TEXT G=(none)   M=uictlmenu  ACBP=28
 3316:000D 05E8 C=CODE   S=UIDRAWOBJECT_TEXT G=(none)   M=uidrawobject ACBP=28
 3375:0005 0564 C=CODE   S=UIOSDSIZE_TEXT G=(none)   M=uiosdsize  ACBP=28
 33CB:0009 02E9 C=CODE   S=UITRACKOPS_TEXT G=(none)   M=uitrackops ACBP=28
 33FA:0002 095D C=CODE   S=UIBHVCONDITIONMGR_TEXT G=(none)   M=uibhvconditionmgr ACBP=28
 348F:000F 061D C=CODE   S=UIBHVDYNAMICMGR_TEXT G=(none)   M=uibhvdynamicmgr ACBP=28
 34F1:000C 0F53 C=CODE   S=PWSRCINPUT_TEXT G=(none)   M=pwsrcinput ACBP=28
 35E6:000F 07F1 C=CODE   S=PWSRCAUTO_TEXT G=(none)   M=pwsrcauto  ACBP=28
 3666:0000 1072 C=CODE   S=PWSRCAUTOCALIBRATE_TEXT G=(none)   M=pwsrcautocalibrate ACBP=28
 376D:0002 3014 C=CODE   S=PWSRCSETTINGS_TEXT G=(none)   M=pwsrcsettings ACBP=28
 3A6E:0006 146A C=CODE   S=PWSRCDETECTION_TEXT G=(none)   M=pwsrcdetection ACBP=28
 3BB5:0000 1CC5 C=CODE   S=PWSRCDISPLAY_TEXT G=(none)   M=pwsrcdisplay ACBP=28
 3D81:0005 0498 C=CODE   S=PWSRCTEST_TEXT G=(none)   M=pwsrctest  ACBP=28
 3DCA:000D 0781 C=CODE   S=HLOSDLOC_TEXT  G=(none)   M=hlosdloc   ACBP=28
 3E42:000E 0421 C=CODE   S=PWSRCUTIL_TEXT G=(none)   M=pwsrcutil  ACBP=28
 3E84:000F 1F4B C=CODE   S=PWSRCTV_TEXT   G=(none)   M=pwsrctv    ACBP=28
 4079:000A 04A2 C=CODE   S=HLRECT_TEXT    G=(none)   M=hlrect     ACBP=28
 40C3:000C 05A3 C=CODE   S=HLSERIAL_TEXT  G=(none)   M=hlserial   ACBP=28
 411D:000F 09DB C=CODE   S=DVSCALERMODE_TEXT G=(none)   M=dvscalermode ACBP=28
 41BB:000A 04C1 C=CODE   S=DVSCALERZOOM_TEXT G=(none)   M=dvscalerzoom ACBP=28
 4207:000B 0212 C=CODE   S=DVSCALERFILTER_TEXT G=(none)   M=dvscalerfilter ACBP=28
 4228:000D 0590 C=CODE   S=DVSCALERNLOPS_TEXT G=(none)   M=dvscalernlops ACBP=28
 4281:000D 05A9 C=CODE   S=HLVIDEO_TEXT   G=(none)   M=hlvideo    ACBP=28
 42DC:0006 04E5 C=CODE   S=DVSCALERPRIV_TEXT G=(none)   M=dvscalerpriv ACBP=28
 432A:000B 05F4 C=CODE   S=HLIMGMEM_TEXT  G=(none)   M=hlimgmem   ACBP=28
 4389:000F 0906 C=CODE   S=HLGPORT_TEXT   G=(none)   M=hlgport    ACBP=28
 441A:0005 01C6 C=CODE   S=HLDPORTISP_TEXT G=(none)   M=hldportisp ACBP=28
 4436:000B 0404 C=CODE   S=HLAUTO_TEXT    G=(none)   M=hlauto     ACBP=28
 4476:000F 011C C=CODE   S=HLGPORTISP_TEXT G=(none)   M=hlgportisp ACBP=28
 4488:000B 011E C=CODE   S=HLVPORTISP_TEXT G=(none)   M=hlvportisp ACBP=28
 449A:0009 032B C=CODE   S=MYAPI_TEXT     G=(none)   M=myapi      ACBP=28
 44CD:0004 02D6 C=CODE   S=PWSRCSYNCMONITOR_TEXT G=(none)   M=pwsrcsyncmonitor ACBP=28
 44FA:000A 0621 C=CODE   S=DVKEYPADTASK_TEXT G=(none)   M=dvkeypadtask ACBP=28
 455C:000B 0247 C=CODE   S=DVOEMPWM16_TEXT G=(none)   M=dvoempwm16 ACBP=28
 4581:0002 09C5 C=CODE   S=HLOSD_TEXT     G=(none)   M=hlosd      ACBP=28
 461D:0007 02D4 C=CODE   S=HLINFRED_TEXT  G=(none)   M=hlinfred   ACBP=28
 464A:000B 00A8 C=CODE   S=HLDECODE_TEXT  G=(none)   M=hldecode   ACBP=28
 4655:0003 08B5 C=CODE   S=DV2WIRE_TEXT   G=(none)   M=dv2wire    ACBP=28
 46E0:0008 07FF C=CODE   S=DVLED_TEXT     G=(none)   M=dvled      ACBP=28
 4760:0007 0051 C=CODE   S=DVOEMLAMP_BACKLIGHT_TEXT G=(none)   M=dvoemlamp_backlight ACBP=28
 4765:0008 0019 C=CODE   S=DVOEMUNITPOWER_TEXT G=(none)   M=dvoemunitpower ACBP=28
 4767:0001 0D7F C=CODE   S=PWBLTMAP_TEXT  G=(none)   M=pwbltmap   ACBP=28
 483F:0000 0F58 C=CODE   S=PWOPPRINTF_TEXT G=(none)   M=pwopprintf ACBP=28
 4934:0008 0139 C=CODE   S=DVIRREMOTETASK_TEXT G=(none)   M=dvirremotetask ACBP=28
 4948:0001 02D9 C=CODE   S=PWOSDOPS_TEXT  G=(none)   M=pwosdops   ACBP=28
 4975:000A 022A C=CODE   S=UIBHVINSPECT_TEXT G=(none)   M=uibhvinspect ACBP=28
 4998:0004 0685 C=CODE   S=UIBHVITERATORS_TEXT G=(none)   M=uibhviterators ACBP=28
 4A00:0009 04EC C=CODE   S=UICTLGAUGE_TEXT G=(none)   M=uictlgauge ACBP=28
 4A4F:0005 0225 C=CODE   S=UICTLNUMBER_TEXT G=(none)   M=uictlnumber ACBP=28
 4A71:000A 0155 C=CODE   S=UICTLBUTTON_TEXT G=(none)   M=uictlbutton ACBP=28
 4A86:000F 0174 C=CODE   S=UICTLTEXT_TEXT G=(none)   M=uictltext  ACBP=28
 4A9E:0003 099C C=CODE   S=UICTLDYNAMIC_TEXT G=(none)   M=uictldynamic ACBP=28
 4B37:000F 0170 C=CODE   S=UICTLBORDER_TEXT G=(none)   M=uictlborder ACBP=28
 4B4E:000F 0002 C=CODE   S=UIPANEMGR_TEXT G=(none)   M=uipanemgr  ACBP=28
 4B4F:0001 03EC C=CODE   S=PWSRCAUTOPOSITION_TEXT G=(none)   M=pwsrcautoposition ACBP=28
 4B8D:000D 0F3C C=CODE   S=PWSRCAUTOFREQPHASE_TEXT G=(none)   M=pwsrcautofreqphase ACBP=28
 4C81:0009 0559 C=CODE   S=PWSRCAUTOBRIGHTNESS_TEXT G=(none)   M=pwsrcautobrightness ACBP=28
 4CD7:0002 061F C=CODE   S=HLHICOLOR_TEXT G=(none)   M=hlhicolor  ACBP=28
 4D39:0001 04BF C=CODE   S=HLPRIV_TEXT    G=(none)   M=hlpriv     ACBP=28
 4D85:0000 04B3 C=CODE   S=DVINFRED_TEXT  G=(none)   M=dvinfred   ACBP=28
 4DD0:0003 0091 C=CODE   S=DVKEYPADDIRECT_TEXT G=(none)   M=dvkeypaddirect ACBP=28
 4DDA:0000 0000 C=INITDATA S=_INIT_         G=IGROUP   M=c0         ACBP=68
 4DDA:0000 0006 C=INITDATA S=_INIT_         G=IGROUP   M=fardata    ACBP=48
 4DDA:0006 0006 C=INITDATA S=_INIT_         G=IGROUP   M=farbss     ACBP=48
 4DDA:000C 0000 C=INITDATA S=_INITEND_      G=IGROUP   M=c0         ACBP=28
 4DDA:0010 0000 C=EXITDATA S=_EXIT_         G=IGROUP   M=c0         ACBP=68
 4DDA:0010 0010 C=EXITDATA S=_EXITEND_      G=IGROUP   M=c0         ACBP=28
 4DDC:0000 0000 C=ROMDATA S=_RD            G=(none)   M=c0         ACBP=68
 4DDC:0000 0010 C=ENDROMDATA S=_ERD           G=(none)   M=c0         ACBP=68
 4DDD:0000 0000 C=ROMFARDATA S=_BRFD          G=(none)   M=c0         ACBP=68
 4DDD:0000 0010 C=ENDROMFARDATA S=_ERFD          G=(none)   M=c0         ACBP=68
 4DDE:0000 0000 C=ROMFUNCTION S=_BRFUNC        G=(none)   M=c0         ACBP=68
 4DDE:0000 0010 C=ENDROMFUNCTION S=_ERFUNC        G=(none)   M=c0         ACBP=68
 4DDF:0000 0000 C=RAMFUNCTION S=_BFUNC         G=(none)   M=c0         ACBP=68
 4DDF:0000 0010 C=ENDRAMFUNCTION S=_EFUNC         G=(none)   M=c0         ACBP=68
 4DE0:0000 0024 C=DATA   S=_DATA          G=DGROUP   M=c0         ACBP=68
 4DE0:0024 0000 C=DATA   S=_DATA          G=DGROUP   M=monitor    ACBP=48
 4DE0:0024 0000 C=DATA   S=_DATA          G=DGROUP   M=monitorcsip ACBP=48
 4DE0:0024 0000 C=DATA   S=_DATA          G=DGROUP   M=formula    ACBP=48
 4DE0:0024 0000 C=DATA   S=_DATA          G=DGROUP   M=debug      ACBP=48
 4DE0:0030 0040 C=DATA   S=_DATA          G=DGROUP   M=inientry   ACBP=68
 4DE0:0070 0002 C=DATA   S=_DATA          G=DGROUP   M=configdata ACBP=48
 4DE0:0072 0001 C=DATA   S=_DATA          G=DGROUP   M=datamgr    ACBP=48
 4DE0:0074 0000 C=DATA   S=_DATA          G=DGROUP   M=interruptctrl ACBP=48
 4DE0:0074 0000 C=DATA   S=_DATA          G=DGROUP   M=main       ACBP=48
 4DE0:0074 0008 C=DATA   S=_DATA          G=DGROUP   M=memory     ACBP=48
 4DE0:007C 0004 C=DATA   S=_DATA          G=DGROUP   M=sysinit    ACBP=48
 4DE0:0080 000C C=DATA   S=_DATA          G=DGROUP   M=exit       ACBP=48
 4DE0:008C 0000 C=DATA   S=_DATA          G=DGROUP   M=noxx       ACBP=48
 4DE0:008C 0000 C=DATA   S=_DATA          G=DGROUP   M=h_ldiv     ACBP=48
 4DE0:008C 0000 C=DATA   S=_DATA          G=DGROUP   M=f_lxmul    ACBP=48
 4DE0:008C 0000 C=DATA   S=_DATA          G=DGROUP   M=uistatemgr ACBP=48
 4DE0:008C 000C C=DATA   S=_DATA          G=DGROUP   M=pwsrccontrol ACBP=48
 4DE0:0098 0014 C=DATA   S=_DATA          G=DGROUP   M=pwperiodic ACBP=48
 4DE0:00AC 0002 C=DATA   S=_DATA          G=DGROUP   M=pwros      ACBP=48
 4DE0:00AE 0000 C=DATA   S=_DATA          G=DGROUP   M=dvrs232    ACBP=48
 4DE0:00AE 0000 C=DATA   S=_DATA          G=DGROUP   M=dvoutputscaler ACBP=48
 4DE0:00AE 0000 C=DATA   S=_DATA          G=DGROUP   M=dvimagememory ACBP=48
 4DE0:00AE 0000 C=DATA   S=_DATA          G=DGROUP   M=dv24cxx    ACBP=48
 4DE0:00AE 0009 C=DATA   S=_DATA          G=DGROUP   M=dvdport    ACBP=48
 4DE0:00B8 0019 C=DATA   S=_DATA          G=DGROUP   M=dvinputport ACBP=48
 4DE0:00D2 0000 C=DATA   S=_DATA          G=DGROUP   M=dvclkgenpg18e1 ACBP=48
 4DE0:00D2 004C C=DATA   S=_DATA          G=DGROUP   M=dvad9883   ACBP=48
 4DE0:011E 003C C=DATA   S=_DATA          G=DGROUP   M=dvvpc3230  ACBP=48
 4DE0:015A 0000 C=DATA   S=_DATA          G=DGROUP   M=dvtmdsgeneric ACBP=48
 4DE0:015A 002E C=DATA   S=_DATA          G=DGROUP   M=dvpw1230   ACBP=48
 4DE0:0188 0010 C=DATA   S=_DATA          G=DGROUP   M=dvz86129   ACBP=48
 4DE0:0198 0000 C=DATA   S=_DATA          G=DGROUP   M=dvtda9851  ACBP=48
 4DE0:0198 0000 C=DATA   S=_DATA          G=DGROUP   M=dvswitcher_shasta_ii ACBP=48
 4DE0:0198 0000 C=DATA   S=_DATA          G=DGROUP   M=dvcolorspace ACBP=48
 4DE0:0198 0001 C=DATA   S=_DATA          G=DGROUP   M=dvfi1256   ACBP=48
 4DE0:019A 0003 C=DATA   S=_DATA          G=DGROUP   M=dvtda9885  ACBP=48
 4DE0:019E 000C C=DATA   S=_DATA          G=DGROUP   M=dvnjw1144  ACBP=48
 4DE0:01AA 0000 C=DATA   S=_DATA          G=DGROUP   M=dvdriverservice ACBP=48
 4DE0:01AA 0000 C=DATA   S=_DATA          G=DGROUP   M=pwcrc      ACBP=48
 4DE0:01AA 0066 C=DATA   S=_DATA          G=DGROUP   M=pwoem      ACBP=48
 4DE0:0210 0000 C=DATA   S=_DATA          G=DGROUP   M=hlint      ACBP=48
 4DE0:0210 0000 C=DATA   S=_DATA          G=DGROUP   M=pwispcore  ACBP=48
 4DE0:0210 000A C=DATA   S=_DATA          G=DGROUP   M=pwmisc     ACBP=48
 4DE0:021A 0008 C=DATA   S=_DATA          G=DGROUP   M=hlregisters ACBP=48
 4DE0:0222 004D C=DATA   S=_DATA          G=DGROUP   M=hlayer111  ACBP=48
 4DE0:0270 0001 C=DATA   S=_DATA          G=DGROUP   M=pwhost     ACBP=48
 4DE0:0272 0000 C=DATA   S=_DATA          G=DGROUP   M=h_lursh    ACBP=48
 4DE0:0272 0000 C=DATA   S=_DATA          G=DGROUP   M=h_llsh     ACBP=48
 4DE0:0272 0016 C=DATA   S=_DATA          G=DGROUP   M=uibhvvariables ACBP=48
 4DE0:0288 0012 C=DATA   S=_DATA          G=DGROUP   M=hlscaler   ACBP=48
 4DE0:029A 0020 C=DATA   S=_DATA          G=DGROUP   M=hldispp    ACBP=48
 4DE0:02BA 0000 C=DATA   S=_DATA          G=DGROUP   M=hltimers   ACBP=48
 4DE0:02BA 0000 C=DATA   S=_DATA          G=DGROUP   M=hlinit     ACBP=48
 4DE0:02BA 0000 C=DATA   S=_DATA          G=DGROUP   M=hlwaitstate ACBP=48
 4DE0:02BA 0000 C=DATA   S=_DATA          G=DGROUP   M=dvgpio     ACBP=48
 4DE0:02BA 0000 C=DATA   S=_DATA          G=DGROUP   M=dvoeminterface ACBP=48
 4DE0:02BA 0008 C=DATA   S=_DATA          G=DGROUP   M=pwdpms     ACBP=48
 4DE0:02C2 0014 C=DATA   S=_DATA          G=DGROUP   M=pwosd      ACBP=48
 4DE0:02D6 0000 C=DATA   S=_DATA          G=DGROUP   M=hlgenctl   ACBP=48
 4DE0:02D6 0040 C=DATA   S=_DATA          G=DGROUP   M=pwinput    ACBP=48
 4DE0:0316 0000 C=DATA   S=_DATA          G=DGROUP   M=atexit     ACBP=48
 4DE0:0316 0004 C=DATA   S=_DATA          G=DGROUP   M=pcpprtl    ACBP=48
 4DE0:031A 0000 C=DATA   S=_DATA          G=DGROUP   M=h_psbp     ACBP=48
 4DE0:031A 0004 C=DATA   S=_DATA          G=DGROUP   M=pwoperations ACBP=48
 4DE0:031E 0000 C=DATA   S=_DATA          G=DGROUP   M=uieventscan ACBP=48
 4DE0:031E 000E C=DATA   S=_DATA          G=DGROUP   M=uibhvmenu  ACBP=48
 4DE0:032C 0000 C=DATA   S=_DATA          G=DGROUP   M=uicontrols ACBP=48
 4DE0:032C 0002 C=DATA   S=_DATA          G=DGROUP   M=uictlmenu  ACBP=48
 4DE0:032E 0004 C=DATA   S=_DATA          G=DGROUP   M=uidrawobject ACBP=48
 4DE0:0332 0004 C=DATA   S=_DATA          G=DGROUP   M=uiosdsize  ACBP=48
 4DE0:0336 0002 C=DATA   S=_DATA          G=DGROUP   M=uitrackops ACBP=48
 4DE0:0338 0002 C=DATA   S=_DATA          G=DGROUP   M=uibhvconditionmgr ACBP=48
 4DE0:033A 0062 C=DATA   S=_DATA          G=DGROUP   M=uibhvdynamicmgr ACBP=48
 4DE0:039C 0001 C=DATA   S=_DATA          G=DGROUP   M=pwsrcinput ACBP=48
 4DE0:039E 0000 C=DATA   S=_DATA          G=DGROUP   M=pwsrcauto  ACBP=48
 4DE0:039E 0000 C=DATA   S=_DATA          G=DGROUP   M=pwsrcautocalibrate ACBP=48
 4DE0:039E 001E C=DATA   S=_DATA          G=DGROUP   M=pwsrcsettings ACBP=48
 4DE0:03BC 0000 C=DATA   S=_DATA          G=DGROUP   M=pwsrcdetection ACBP=48
 4DE0:03BC 0012 C=DATA   S=_DATA          G=DGROUP   M=pwsrcdisplay ACBP=48
 4DE0:03CE 0018 C=DATA   S=_DATA          G=DGROUP   M=pwsrctest  ACBP=48
 4DE0:03E6 0002 C=DATA   S=_DATA          G=DGROUP   M=hlosdloc   ACBP=48
 4DE0:03E8 0000 C=DATA   S=_DATA          G=DGROUP   M=pwsrcutil  ACBP=48
 4DE0:03E8 002E C=DATA   S=_DATA          G=DGROUP   M=pwsrctv    ACBP=48
 4DE0:0416 0000 C=DATA   S=_DATA          G=DGROUP   M=hlrect     ACBP=48
 4DE0:0416 0000 C=DATA   S=_DATA          G=DGROUP   M=f_scopy    ACBP=48
 4DE0:0416 0004 C=DATA   S=_DATA          G=DGROUP   M=hlserial   ACBP=48
 4DE0:041A 0008 C=DATA   S=_DATA          G=DGROUP   M=dvscalermode ACBP=48
 4DE0:0422 0000 C=DATA   S=_DATA          G=DGROUP   M=dvscalerzoom ACBP=48
 4DE0:0422 0000 C=DATA   S=_DATA          G=DGROUP   M=dvscalerfilter ACBP=48
 4DE0:0422 0000 C=DATA   S=_DATA          G=DGROUP   M=dvscalernlops ACBP=48
 4DE0:0422 0001 C=DATA   S=_DATA          G=DGROUP   M=hlvideo    ACBP=48
 4DE0:0424 0022 C=DATA   S=_DATA          G=DGROUP   M=dvscalerpriv ACBP=48
 4DE0:0446 0002 C=DATA   S=_DATA          G=DGROUP   M=hlimgmem   ACBP=48
 4DE0:0448 0003 C=DATA   S=_DATA          G=DGROUP   M=hlgport    ACBP=48
 4DE0:044C 0001 C=DATA   S=_DATA          G=DGROUP   M=hldportisp ACBP=48
 4DE0:044E 0008 C=DATA   S=_DATA          G=DGROUP   M=hlauto     ACBP=48
 4DE0:0456 0000 C=DATA   S=_DATA          G=DGROUP   M=hlgportisp ACBP=48
 4DE0:0456 0000 C=DATA   S=_DATA          G=DGROUP   M=hlvportisp ACBP=48
 4DE0:0456 0000 C=DATA   S=_DATA          G=DGROUP   M=myapi      ACBP=48
 4DE0:0456 0000 C=DATA   S=_DATA          G=DGROUP   M=pwsrcsyncmonitor ACBP=48
 4DE0:0456 0000 C=DATA   S=_DATA          G=DGROUP   M=h_lrsh     ACBP=48
 4DE0:0456 000C C=DATA   S=_DATA          G=DGROUP   M=dvkeypadtask ACBP=48
 4DE0:0462 0000 C=DATA   S=_DATA          G=DGROUP   M=dvoempwm16 ACBP=48
 4DE0:0462 0000 C=DATA   S=_DATA          G=DGROUP   M=hlosd      ACBP=48
 4DE0:0462 0000 C=DATA   S=_DATA          G=DGROUP   M=hlinfred   ACBP=48
 4DE0:0462 0000 C=DATA   S=_DATA          G=DGROUP   M=hldecode   ACBP=48
 4DE0:0462 0000 C=DATA   S=_DATA          G=DGROUP   M=dv2wire    ACBP=48
 4DE0:0462 0000 C=DATA   S=_DATA          G=DGROUP   M=atol       ACBP=48
 4DE0:0462 0000 C=DATA   S=_DATA          G=DGROUP   M=labs       ACBP=48
 4DE0:0462 0000 C=DATA   S=_DATA          G=DGROUP   M=strncmp    ACBP=48
 4DE0:0462 0004 C=DATA   S=_DATA          G=DGROUP   M=dvled      ACBP=48
 4DE0:0466 0000 C=DATA   S=_DATA          G=DGROUP   M=dvoemlamp_backlight ACBP=48
 4DE0:0466 0002 C=DATA   S=_DATA          G=DGROUP   M=dvoemunitpower ACBP=48
 4DE0:0468 0006 C=DATA   S=_DATA          G=DGROUP   M=pwbltmap   ACBP=48
 4DE0:046E 0009 C=DATA   S=_DATA          G=DGROUP   M=pwopprintf ACBP=48
 4DE0:0478 0000 C=DATA   S=_DATA          G=DGROUP   M=dvirremotetask ACBP=48
 4DE0:0478 0000 C=DATA   S=_DATA          G=DGROUP   M=pwosdops   ACBP=48
 4DE0:0478 0000 C=DATA   S=_DATA          G=DGROUP   M=uibhvinspect ACBP=48
 4DE0:0478 0006 C=DATA   S=_DATA          G=DGROUP   M=uibhviterators ACBP=48
 4DE0:047E 0000 C=DATA   S=_DATA          G=DGROUP   M=uictlgauge ACBP=48
 4DE0:047E 0000 C=DATA   S=_DATA          G=DGROUP   M=uictlnumber ACBP=48
 4DE0:047E 0000 C=DATA   S=_DATA          G=DGROUP   M=uictlbutton ACBP=48
 4DE0:047E 0000 C=DATA   S=_DATA          G=DGROUP   M=uictltext  ACBP=48
 4DE0:047E 0000 C=DATA   S=_DATA          G=DGROUP   M=uictldynamic ACBP=48
 4DE0:047E 0000 C=DATA   S=_DATA          G=DGROUP   M=uictlborder ACBP=48
 4DE0:047E 0000 C=DATA   S=_DATA          G=DGROUP   M=uipanemgr  ACBP=48
 4DE0:047E 0000 C=DATA   S=_DATA          G=DGROUP   M=pwsrcautoposition ACBP=48
 4DE0:047E 0080 C=DATA   S=_DATA          G=DGROUP   M=pwsrcautofreqphase ACBP=48
 4DE0:04FE 0000 C=DATA   S=_DATA          G=DGROUP   M=pwsrcautobrightness ACBP=48
 4DE0:04FE 0000 C=DATA   S=_DATA          G=DGROUP   M=hlhicolor  ACBP=48
 4DE0:04FE 0000 C=DATA   S=_DATA          G=DGROUP   M=hlpriv     ACBP=48
 4DE0:04FE 0009 C=DATA   S=_DATA          G=DGROUP   M=dvinfred   ACBP=48
 4DE0:0508 0000 C=DATA   S=_DATA          G=DGROUP   M=dvkeypaddirect ACBP=48
 4DE0:0508 0101 C=DATA   S=_DATA          G=DGROUP   M=ctype      ACBP=48
 4DE0:060A 0000 C=DATA   S=_DATA          G=DGROUP   M=h_pada     ACBP=48
 4DE0:060A 0000 C=DATA   S=_CVTSEG        G=DGROUP   M=c0         ACBP=48
 4DE0:060A 0000 C=DATA   S=_SCNSEG        G=DGROUP   M=c0         ACBP=48
 4DE0:0610 0002 C=DATA   S=AMXDGRP        G=DGROUP   M=romcfg     ACBP=68
 4DE0:0612 0001 C=DATA   S=AMXDGRP        G=DGROUP   M=aj831uc    ACBP=48
 4DE0:0614 0028 C=DATA   S=AMXVAR         G=DGROUP   M=romcfg     ACBP=48
 4DE0:0640 0002 C=BSS    S=_BSS           G=DGROUP   M=c0         ACBP=68
 4DE0:0642 0000 C=BSS    S=_BSS           G=DGROUP   M=monitor    ACBP=48
 4DE0:0642 0000 C=BSS    S=_BSS           G=DGROUP   M=monitorcsip ACBP=48
 4DE0:0642 0000 C=BSS    S=_BSS           G=DGROUP   M=formula    ACBP=48
 4DE0:0642 0000 C=BSS    S=_BSS           G=DGROUP   M=debug      ACBP=48
 4DE0:0642 0004 C=BSS    S=_BSS           G=DGROUP   M=configdata ACBP=48
 4DE0:0646 08BA C=BSS    S=_BSS           G=DGROUP   M=datamgr    ACBP=48
 4DE0:0F00 0032 C=BSS    S=_BSS           G=DGROUP   M=interruptctrl ACBP=48
 4DE0:0F32 0004 C=BSS    S=_BSS           G=DGROUP   M=main       ACBP=48
 4DE0:0F36 0012 C=BSS    S=_BSS           G=DGROUP   M=memory     ACBP=48
 4DE0:0F48 0000 C=BSS    S=_BSS           G=DGROUP   M=sysinit    ACBP=48
 4DE0:0F48 0000 C=BSS    S=_BSS           G=DGROUP   M=exit       ACBP=48
 4DE0:0F48 0008 C=BSS    S=_BSS           G=DGROUP   M=noxx       ACBP=48
 4DE0:0F50 002D C=BSS    S=_BSS           G=DGROUP   M=uistatemgr ACBP=48
 4DE0:0F7E 006E C=BSS    S=_BSS           G=DGROUP   M=pwsrccontrol ACBP=48
 4DE0:0FEC 0000 C=BSS    S=_BSS           G=DGROUP   M=pwperiodic ACBP=48
 4DE0:0FEC 0001 C=BSS    S=_BSS           G=DGROUP   M=pwros      ACBP=48
 4DE0:0FEE 0004 C=BSS    S=_BSS           G=DGROUP   M=dvrs232    ACBP=48
 4DE0:0FF2 0006 C=BSS    S=_BSS           G=DGROUP   M=dvoutputscaler ACBP=48
 4DE0:0FF8 0000 C=BSS    S=_BSS           G=DGROUP   M=dvimagememory ACBP=48
 4DE0:0FF8 0006 C=BSS    S=_BSS           G=DGROUP   M=dv24cxx    ACBP=48
 4DE0:0FFE 0021 C=BSS    S=_BSS           G=DGROUP   M=dvdport    ACBP=48
 4DE0:1020 0096 C=BSS    S=_BSS           G=DGROUP   M=dvinputport ACBP=48
 4DE0:10B6 0000 C=BSS    S=_BSS           G=DGROUP   M=dvclkgenpg18e1 ACBP=48
 4DE0:10B6 0046 C=BSS    S=_BSS           G=DGROUP   M=dvad9883   ACBP=48
 4DE0:10FC 0034 C=BSS    S=_BSS           G=DGROUP   M=dvvpc3230  ACBP=48
 4DE0:1130 0002 C=BSS    S=_BSS           G=DGROUP   M=dvtmdsgeneric ACBP=48
 4DE0:1132 011A C=BSS    S=_BSS           G=DGROUP   M=dvpw1230   ACBP=48
 4DE0:124C 0013 C=BSS    S=_BSS           G=DGROUP   M=dvz86129   ACBP=48
 4DE0:1260 0004 C=BSS    S=_BSS           G=DGROUP   M=dvtda9851  ACBP=48
 4DE0:1264 0000 C=BSS    S=_BSS           G=DGROUP   M=dvswitcher_shasta_ii ACBP=48
 4DE0:1264 0008 C=BSS    S=_BSS           G=DGROUP   M=dvcolorspace ACBP=48
 4DE0:126C 0009 C=BSS    S=_BSS           G=DGROUP   M=dvfi1256   ACBP=48
 4DE0:1276 0002 C=BSS    S=_BSS           G=DGROUP   M=dvtda9885  ACBP=48
 4DE0:1278 000E C=BSS    S=_BSS           G=DGROUP   M=dvnjw1144  ACBP=48
 4DE0:1286 0004 C=BSS    S=_BSS           G=DGROUP   M=dvdriverservice ACBP=48
 4DE0:128A 0000 C=BSS    S=_BSS           G=DGROUP   M=pwcrc      ACBP=48
 4DE0:128A 0072 C=BSS    S=_BSS           G=DGROUP   M=pwoem      ACBP=48
 4DE0:12FC 0000 C=BSS    S=_BSS           G=DGROUP   M=hlint      ACBP=48
 4DE0:12FC 0000 C=BSS    S=_BSS           G=DGROUP   M=pwispcore  ACBP=48
 4DE0:12FC 0000 C=BSS    S=_BSS           G=DGROUP   M=pwmisc     ACBP=48
 4DE0:12FC 00AE C=BSS    S=_BSS           G=DGROUP   M=hlregisters ACBP=48
 4DE0:13AA 001A C=BSS    S=_BSS           G=DGROUP   M=hlayer111  ACBP=48
 4DE0:13C4 0088 C=BSS    S=_BSS           G=DGROUP   M=pwhost     ACBP=48
 4DE0:144C 001A C=BSS    S=_BSS           G=DGROUP   M=uibhvvariables ACBP=48
 4DE0:1466 004C C=BSS    S=_BSS           G=DGROUP   M=hlscaler   ACBP=48
 4DE0:14B2 0003 C=BSS    S=_BSS           G=DGROUP   M=hldispp    ACBP=48
 4DE0:14B6 001A C=BSS    S=_BSS           G=DGROUP   M=hltimers   ACBP=48
 4DE0:14D0 002C C=BSS    S=_BSS           G=DGROUP   M=hlinit     ACBP=48
 4DE0:14FC 0000 C=BSS    S=_BSS           G=DGROUP   M=hlwaitstate ACBP=48
 4DE0:14FC 001B C=BSS    S=_BSS           G=DGROUP   M=dvgpio     ACBP=48
 4DE0:1518 0008 C=BSS    S=_BSS           G=DGROUP   M=dvoeminterface ACBP=48
 4DE0:1520 004E C=BSS    S=_BSS           G=DGROUP   M=pwdpms     ACBP=48
 4DE0:156E 0074 C=BSS    S=_BSS           G=DGROUP   M=pwosd      ACBP=48
 4DE0:15E2 0003 C=BSS    S=_BSS           G=DGROUP   M=hlgenctl   ACBP=48
 4DE0:15E6 0002 C=BSS    S=_BSS           G=DGROUP   M=pwinput    ACBP=48
 4DE0:15E8 0022 C=BSS    S=_BSS           G=DGROUP   M=atexit     ACBP=48
 4DE0:160A 0002 C=BSS    S=_BSS           G=DGROUP   M=pcpprtl    ACBP=48
 4DE0:160C 0009 C=BSS    S=_BSS           G=DGROUP   M=pwoperations ACBP=48
 4DE0:1616 0000 C=BSS    S=_BSS           G=DGROUP   M=uieventscan ACBP=48
 4DE0:1616 0200 C=BSS    S=_BSS           G=DGROUP   M=uibhvmenu  ACBP=48
 4DE0:1816 000E C=BSS    S=_BSS           G=DGROUP   M=uicontrols ACBP=48
 4DE0:1824 0000 C=BSS    S=_BSS           G=DGROUP   M=uictlmenu  ACBP=48
 4DE0:1824 0000 C=BSS    S=_BSS           G=DGROUP   M=uidrawobject ACBP=48
 4DE0:1824 000E C=BSS    S=_BSS           G=DGROUP   M=uiosdsize  ACBP=48
 4DE0:1832 002A C=BSS    S=_BSS           G=DGROUP   M=uitrackops ACBP=48
 4DE0:185C 001E C=BSS    S=_BSS           G=DGROUP   M=uibhvconditionmgr ACBP=48
 4DE0:187A 00C8 C=BSS    S=_BSS           G=DGROUP   M=uibhvdynamicmgr ACBP=48
 4DE0:1942 0012 C=BSS    S=_BSS           G=DGROUP   M=pwsrcinput ACBP=48
 4DE0:1954 0002 C=BSS    S=_BSS           G=DGROUP   M=pwsrcauto  ACBP=48
 4DE0:1956 0000 C=BSS    S=_BSS           G=DGROUP   M=pwsrcautocalibrate ACBP=48
 4DE0:1956 001D C=BSS    S=_BSS           G=DGROUP   M=pwsrcsettings ACBP=48
 4DE0:1974 0006 C=BSS    S=_BSS           G=DGROUP   M=pwsrcdetection ACBP=48
 4DE0:197A 002E C=BSS    S=_BSS           G=DGROUP   M=pwsrcdisplay ACBP=48
 4DE0:19A8 0000 C=BSS    S=_BSS           G=DGROUP   M=pwsrctest  ACBP=48
 4DE0:19A8 004E C=BSS    S=_BSS           G=DGROUP   M=hlosdloc   ACBP=48
 4DE0:19F6 0001 C=BSS    S=_BSS           G=DGROUP   M=pwsrcutil  ACBP=48
 4DE0:19F8 0022 C=BSS    S=_BSS           G=DGROUP   M=pwsrctv    ACBP=48
 4DE0:1A1A 0000 C=BSS    S=_BSS           G=DGROUP   M=hlrect     ACBP=48
 4DE0:1A1A 0021 C=BSS    S=_BSS           G=DGROUP   M=hlserial   ACBP=48
 4DE0:1A3C 0000 C=BSS    S=_BSS           G=DGROUP   M=dvscalermode ACBP=48
 4DE0:1A3C 000C C=BSS    S=_BSS           G=DGROUP   M=dvscalerzoom ACBP=48
 4DE0:1A48 0000 C=BSS    S=_BSS           G=DGROUP   M=dvscalerfilter ACBP=48
 4DE0:1A48 0000 C=BSS    S=_BSS           G=DGROUP   M=dvscalernlops ACBP=48
 4DE0:1A48 0016 C=BSS    S=_BSS           G=DGROUP   M=hlvideo    ACBP=48
 4DE0:1A5E 0004 C=BSS    S=_BSS           G=DGROUP   M=dvscalerpriv ACBP=48
 4DE0:1A62 0002 C=BSS    S=_BSS           G=DGROUP   M=hlimgmem   ACBP=48
 4DE0:1A64 0022 C=BSS    S=_BSS           G=DGROUP   M=hlgport    ACBP=48
 4DE0:1A86 0012 C=BSS    S=_BSS           G=DGROUP   M=hldportisp ACBP=48
 4DE0:1A98 0002 C=BSS    S=_BSS           G=DGROUP   M=hlauto     ACBP=48
 4DE0:1A9A 0012 C=BSS    S=_BSS           G=DGROUP   M=hlgportisp ACBP=48
 4DE0:1AAC 0012 C=BSS    S=_BSS           G=DGROUP   M=hlvportisp ACBP=48
 4DE0:1ABE 0000 C=BSS    S=_BSS           G=DGROUP   M=myapi      ACBP=48
 4DE0:1ABE 0020 C=BSS    S=_BSS           G=DGROUP   M=pwsrcsyncmonitor ACBP=48
 4DE0:1ADE 0036 C=BSS    S=_BSS           G=DGROUP   M=dvkeypadtask ACBP=48
 4DE0:1B14 000C C=BSS    S=_BSS           G=DGROUP   M=dvoempwm16 ACBP=48
 4DE0:1B20 0030 C=BSS    S=_BSS           G=DGROUP   M=hlosd      ACBP=48
 4DE0:1B50 0004 C=BSS    S=_BSS           G=DGROUP   M=hlinfred   ACBP=48
 4DE0:1B54 0000 C=BSS    S=_BSS           G=DGROUP   M=hldecode   ACBP=48
 4DE0:1B54 0014 C=BSS    S=_BSS           G=DGROUP   M=dv2wire    ACBP=48
 4DE0:1B68 0000 C=BSS    S=_BSS           G=DGROUP   M=atol       ACBP=48
 4DE0:1B68 0000 C=BSS    S=_BSS           G=DGROUP   M=labs       ACBP=48
 4DE0:1B68 0000 C=BSS    S=_BSS           G=DGROUP   M=strncmp    ACBP=48
 4DE0:1B68 0030 C=BSS    S=_BSS           G=DGROUP   M=dvled      ACBP=48
 4DE0:1B98 0000 C=BSS    S=_BSS           G=DGROUP   M=dvoemlamp_backlight ACBP=48
 4DE0:1B98 0000 C=BSS    S=_BSS           G=DGROUP   M=dvoemunitpower ACBP=48
 4DE0:1B98 0038 C=BSS    S=_BSS           G=DGROUP   M=pwbltmap   ACBP=48
 4DE0:1BD0 0050 C=BSS    S=_BSS           G=DGROUP   M=pwopprintf ACBP=48
 4DE0:1C20 0008 C=BSS    S=_BSS           G=DGROUP   M=dvirremotetask ACBP=48
 4DE0:1C28 0000 C=BSS    S=_BSS           G=DGROUP   M=pwosdops   ACBP=48
 4DE0:1C28 0000 C=BSS    S=_BSS           G=DGROUP   M=uibhvinspect ACBP=48
 4DE0:1C28 0000 C=BSS    S=_BSS           G=DGROUP   M=uibhviterators ACBP=48
 4DE0:1C28 0000 C=BSS    S=_BSS           G=DGROUP   M=uictlgauge ACBP=48
 4DE0:1C28 0000 C=BSS    S=_BSS           G=DGROUP   M=uictlnumber ACBP=48
 4DE0:1C28 0000 C=BSS    S=_BSS           G=DGROUP   M=uictlbutton ACBP=48
 4DE0:1C28 0000 C=BSS    S=_BSS           G=DGROUP   M=uictltext  ACBP=48
 4DE0:1C28 0000 C=BSS    S=_BSS           G=DGROUP   M=uictldynamic ACBP=48
 4DE0:1C28 0000 C=BSS    S=_BSS           G=DGROUP   M=uictlborder ACBP=48
 4DE0:1C28 0000 C=BSS    S=_BSS           G=DGROUP   M=uipanemgr  ACBP=48
 4DE0:1C28 0002 C=BSS    S=_BSS           G=DGROUP   M=pwsrcautoposition ACBP=48
 4DE0:1C2A 0012 C=BSS    S=_BSS           G=DGROUP   M=pwsrcautofreqphase ACBP=48
 4DE0:1C3C 0002 C=BSS    S=_BSS           G=DGROUP   M=pwsrcautobrightness ACBP=48
 4DE0:1C3E 0000 C=BSS    S=_BSS           G=DGROUP   M=hlhicolor  ACBP=48
 4DE0:1C3E 0000 C=BSS    S=_BSS           G=DGROUP   M=hlpriv     ACBP=48
 4DE0:1C3E 0018 C=BSS    S=_BSS           G=DGROUP   M=dvinfred   ACBP=48
 4DE0:1C56 0002 C=BSS    S=_BSS           G=DGROUP   M=dvkeypaddirect ACBP=48
 4DE0:1C58 0000 C=BSS    S=_BSS           G=DGROUP   M=ctype      ACBP=48
 4DE0:1C60 0000 C=NVRAM  S=_NVRAM         G=DGROUP   M=c0         ACBP=68
 4DE0:1C60 0000 C=NVRAM  S=_NVRAM         G=DGROUP   M=monitor    ACBP=48
 4DE0:1C60 0000 C=NVRAM  S=_NVRAM         G=DGROUP   M=monitorcsip ACBP=48
 4DE0:1C60 0000 C=NVRAM  S=_NVRAM         G=DGROUP   M=formula    ACBP=48
 4DE0:1C60 0000 C=NVRAM  S=_NVRAM         G=DGROUP   M=debug      ACBP=48
 4DE0:1C60 0000 C=NVRAM  S=_NVRAM         G=DGROUP   M=configdata ACBP=48
 4DE0:1C60 0000 C=NVRAM  S=_NVRAM         G=DGROUP   M=datamgr    ACBP=48
 4DE0:1C60 0000 C=NVRAM  S=_NVRAM         G=DGROUP   M=interruptctrl ACBP=48
 4DE0:1C60 0000 C=NVRAM  S=_NVRAM         G=DGROUP   M=main       ACBP=48
 4DE0:1C60 0000 C=NVRAM  S=_NVRAM         G=DGROUP   M=memory     ACBP=48
 4DE0:1C60 0000 C=NVRAM  S=_NVRAM         G=DGROUP   M=sysinit    ACBP=48
 4DE0:1C60 0000 C=NVRAM  S=_NVRAM         G=DGROUP   M=exit       ACBP=48
 4DE0:1C60 0000 C=NVRAM  S=_NVRAM         G=DGROUP   M=noxx       ACBP=48
 4DE0:1C60 0000 C=NVRAM  S=_NVRAM         G=DGROUP   M=uistatemgr ACBP=48
 4DE0:1C60 0000 C=NVRAM  S=_NVRAM         G=DGROUP   M=pwsrccontrol ACBP=48
 4DE0:1C60 0000 C=NVRAM  S=_NVRAM         G=DGROUP   M=pwperiodic ACBP=48
 4DE0:1C60 0000 C=NVRAM  S=_NVRAM         G=DGROUP   M=pwros      ACBP=48
 4DE0:1C60 0000 C=NVRAM  S=_NVRAM         G=DGROUP   M=dvrs232    ACBP=48
 4DE0:1C60 0000 C=NVRAM  S=_NVRAM         G=DGROUP   M=dvoutputscaler ACBP=48
 4DE0:1C60 0000 C=NVRAM  S=_NVRAM         G=DGROUP   M=dvimagememory ACBP=48
 4DE0:1C60 0000 C=NVRAM  S=_NVRAM         G=DGROUP   M=dv24cxx    ACBP=48
 4DE0:1C60 0000 C=NVRAM  S=_NVRAM         G=DGROUP   M=dvdport    ACBP=48
 4DE0:1C60 0000 C=NVRAM  S=_NVRAM         G=DGROUP   M=dvinputport ACBP=48
 4DE0:1C60 0000 C=NVRAM  S=_NVRAM         G=DGROUP   M=dvclkgenpg18e1 ACBP=48
 4DE0:1C60 0000 C=NVRAM  S=_NVRAM         G=DGROUP   M=dvad9883   ACBP=48
 4DE0:1C60 0000 C=NVRAM  S=_NVRAM         G=DGROUP   M=dvvpc3230  ACBP=48
 4DE0:1C60 0000 C=NVRAM  S=_NVRAM         G=DGROUP   M=dvtmdsgeneric ACBP=48
 4DE0:1C60 0000 C=NVRAM  S=_NVRAM         G=DGROUP   M=dvpw1230   ACBP=48
 4DE0:1C60 0000 C=NVRAM  S=_NVRAM         G=DGROUP   M=dvz86129   ACBP=48
 4DE0:1C60 0000 C=NVRAM  S=_NVRAM         G=DGROUP   M=dvtda9851  ACBP=48
 4DE0:1C60 0000 C=NVRAM  S=_NVRAM         G=DGROUP   M=dvswitcher_shasta_ii ACBP=48
 4DE0:1C60 0000 C=NVRAM  S=_NVRAM         G=DGROUP   M=dvcolorspace ACBP=48
 4DE0:1C60 0000 C=NVRAM  S=_NVRAM         G=DGROUP   M=dvfi1256   ACBP=48
 4DE0:1C60 0000 C=NVRAM  S=_NVRAM         G=DGROUP   M=dvtda9885  ACBP=48
 4DE0:1C60 0000 C=NVRAM  S=_NVRAM         G=DGROUP   M=dvnjw1144  ACBP=48
 4DE0:1C60 0000 C=NVRAM  S=_NVRAM         G=DGROUP   M=dvdriverservice ACBP=48
 4DE0:1C60 0000 C=NVRAM  S=_NVRAM         G=DGROUP   M=pwcrc      ACBP=48
 4DE0:1C60 0000 C=NVRAM  S=_NVRAM         G=DGROUP   M=pwoem      ACBP=48
 4DE0:1C60 0000 C=NVRAM  S=_NVRAM         G=DGROUP   M=hlint      ACBP=48
 4DE0:1C60 0000 C=NVRAM  S=_NVRAM         G=DGROUP   M=pwispcore  ACBP=48
 4DE0:1C60 0000 C=NVRAM  S=_NVRAM         G=DGROUP   M=pwmisc     ACBP=48
 4DE0:1C60 0000 C=NVRAM  S=_NVRAM         G=DGROUP   M=hlregisters ACBP=48
 4DE0:1C60 0000 C=NVRAM  S=_NVRAM         G=DGROUP   M=hlayer111  ACBP=48
 4DE0:1C60 0000 C=NVRAM  S=_NVRAM         G=DGROUP   M=pwhost     ACBP=48
 4DE0:1C60 0000 C=NVRAM  S=_NVRAM         G=DGROUP   M=uibhvvariables ACBP=48
 4DE0:1C60 0000 C=NVRAM  S=_NVRAM         G=DGROUP   M=hlscaler   ACBP=48
 4DE0:1C60 0000 C=NVRAM  S=_NVRAM         G=DGROUP   M=hldispp    ACBP=48
 4DE0:1C60 0000 C=NVRAM  S=_NVRAM         G=DGROUP   M=hltimers   ACBP=48
 4DE0:1C60 0000 C=NVRAM  S=_NVRAM         G=DGROUP   M=hlinit     ACBP=48
 4DE0:1C60 0000 C=NVRAM  S=_NVRAM         G=DGROUP   M=hlwaitstate ACBP=48
 4DE0:1C60 0000 C=NVRAM  S=_NVRAM         G=DGROUP   M=dvgpio     ACBP=48
 4DE0:1C60 0000 C=NVRAM  S=_NVRAM         G=DGROUP   M=dvoeminterface ACBP=48
 4DE0:1C60 0000 C=NVRAM  S=_NVRAM         G=DGROUP   M=pwdpms     ACBP=48
 4DE0:1C60 0000 C=NVRAM  S=_NVRAM         G=DGROUP   M=pwosd      ACBP=48
 4DE0:1C60 0000 C=NVRAM  S=_NVRAM         G=DGROUP   M=hlgenctl   ACBP=48
 4DE0:1C60 0000 C=NVRAM  S=_NVRAM         G=DGROUP   M=pwinput    ACBP=48
 4DE0:1C60 0000 C=NVRAM  S=_NVRAM         G=DGROUP   M=atexit     ACBP=48
 4DE0:1C60 0000 C=NVRAM  S=_NVRAM         G=DGROUP   M=pwoperations ACBP=48
 4DE0:1C60 0000 C=NVRAM  S=_NVRAM         G=DGROUP   M=uieventscan ACBP=48
 4DE0:1C60 0000 C=NVRAM  S=_NVRAM         G=DGROUP   M=uibhvmenu  ACBP=48
 4DE0:1C60 0000 C=NVRAM  S=_NVRAM         G=DGROUP   M=uicontrols ACBP=48
 4DE0:1C60 0000 C=NVRAM  S=_NVRAM         G=DGROUP   M=uictlmenu  ACBP=48
 4DE0:1C60 0000 C=NVRAM  S=_NVRAM         G=DGROUP   M=uidrawobject ACBP=48
 4DE0:1C60 0000 C=NVRAM  S=_NVRAM         G=DGROUP   M=uiosdsize  ACBP=48
 4DE0:1C60 0000 C=NVRAM  S=_NVRAM         G=DGROUP   M=uitrackops ACBP=48
 4DE0:1C60 0000 C=NVRAM  S=_NVRAM         G=DGROUP   M=uibhvconditionmgr ACBP=48
 4DE0:1C60 0000 C=NVRAM  S=_NVRAM         G=DGROUP   M=uibhvdynamicmgr ACBP=48
 4DE0:1C60 0000 C=NVRAM  S=_NVRAM         G=DGROUP   M=pwsrcinput ACBP=48
 4DE0:1C60 0000 C=NVRAM  S=_NVRAM         G=DGROUP   M=pwsrcauto  ACBP=48
 4DE0:1C60 0000 C=NVRAM  S=_NVRAM         G=DGROUP   M=pwsrcautocalibrate ACBP=48
 4DE0:1C60 0000 C=NVRAM  S=_NVRAM         G=DGROUP   M=pwsrcsettings ACBP=48
 4DE0:1C60 0000 C=NVRAM  S=_NVRAM         G=DGROUP   M=pwsrcdetection ACBP=48
 4DE0:1C60 0000 C=NVRAM  S=_NVRAM         G=DGROUP   M=pwsrcdisplay ACBP=48
 4DE0:1C60 0000 C=NVRAM  S=_NVRAM         G=DGROUP   M=pwsrctest  ACBP=48
 4DE0:1C60 0000 C=NVRAM  S=_NVRAM         G=DGROUP   M=hlosdloc   ACBP=48
 4DE0:1C60 0000 C=NVRAM  S=_NVRAM         G=DGROUP   M=pwsrcutil  ACBP=48
 4DE0:1C60 0000 C=NVRAM  S=_NVRAM         G=DGROUP   M=pwsrctv    ACBP=48
 4DE0:1C60 0000 C=NVRAM  S=_NVRAM         G=DGROUP   M=hlrect     ACBP=48
 4DE0:1C60 0000 C=NVRAM  S=_NVRAM         G=DGROUP   M=hlserial   ACBP=48
 4DE0:1C60 0000 C=NVRAM  S=_NVRAM         G=DGROUP   M=dvscalermode ACBP=48
 4DE0:1C60 0000 C=NVRAM  S=_NVRAM         G=DGROUP   M=dvscalerzoom ACBP=48
 4DE0:1C60 0000 C=NVRAM  S=_NVRAM         G=DGROUP   M=dvscalerfilter ACBP=48
 4DE0:1C60 0000 C=NVRAM  S=_NVRAM         G=DGROUP   M=dvscalernlops ACBP=48
 4DE0:1C60 0000 C=NVRAM  S=_NVRAM         G=DGROUP   M=hlvideo    ACBP=48
 4DE0:1C60 0000 C=NVRAM  S=_NVRAM         G=DGROUP   M=dvscalerpriv ACBP=48
 4DE0:1C60 0000 C=NVRAM  S=_NVRAM         G=DGROUP   M=hlimgmem   ACBP=48
 4DE0:1C60 0000 C=NVRAM  S=_NVRAM         G=DGROUP   M=hlgport    ACBP=48
 4DE0:1C60 0000 C=NVRAM  S=_NVRAM         G=DGROUP   M=hldportisp ACBP=48
 4DE0:1C60 0000 C=NVRAM  S=_NVRAM         G=DGROUP   M=hlauto     ACBP=48
 4DE0:1C60 0000 C=NVRAM  S=_NVRAM         G=DGROUP   M=hlgportisp ACBP=48
 4DE0:1C60 0000 C=NVRAM  S=_NVRAM         G=DGROUP   M=hlvportisp ACBP=48
 4DE0:1C60 0000 C=NVRAM  S=_NVRAM         G=DGROUP   M=myapi      ACBP=48
 4DE0:1C60 0000 C=NVRAM  S=_NVRAM         G=DGROUP   M=pwsrcsyncmonitor ACBP=48
 4DE0:1C60 0000 C=NVRAM  S=_NVRAM         G=DGROUP   M=dvkeypadtask ACBP=48
 4DE0:1C60 0000 C=NVRAM  S=_NVRAM         G=DGROUP   M=dvoempwm16 ACBP=48
 4DE0:1C60 0000 C=NVRAM  S=_NVRAM         G=DGROUP   M=hlosd      ACBP=48
 4DE0:1C60 0000 C=NVRAM  S=_NVRAM         G=DGROUP   M=hlinfred   ACBP=48
 4DE0:1C60 0000 C=NVRAM  S=_NVRAM         G=DGROUP   M=hldecode   ACBP=48
 4DE0:1C60 0000 C=NVRAM  S=_NVRAM         G=DGROUP   M=dv2wire    ACBP=48
 4DE0:1C60 0000 C=NVRAM  S=_NVRAM         G=DGROUP   M=atol       ACBP=48
 4DE0:1C60 0000 C=NVRAM  S=_NVRAM         G=DGROUP   M=labs       ACBP=48
 4DE0:1C60 0000 C=NVRAM  S=_NVRAM         G=DGROUP   M=strncmp    ACBP=48
 4DE0:1C60 0000 C=NVRAM  S=_NVRAM         G=DGROUP   M=dvled      ACBP=48
 4DE0:1C60 0000 C=NVRAM  S=_NVRAM         G=DGROUP   M=dvoemlamp_backlight ACBP=48
 4DE0:1C60 0000 C=NVRAM  S=_NVRAM         G=DGROUP   M=dvoemunitpower ACBP=48
 4DE0:1C60 0000 C=NVRAM  S=_NVRAM         G=DGROUP   M=pwbltmap   ACBP=48
 4DE0:1C60 0000 C=NVRAM  S=_NVRAM         G=DGROUP   M=pwopprintf ACBP=48
 4DE0:1C60 0000 C=NVRAM  S=_NVRAM         G=DGROUP   M=dvirremotetask ACBP=48
 4DE0:1C60 0000 C=NVRAM  S=_NVRAM         G=DGROUP   M=pwosdops   ACBP=48
 4DE0:1C60 0000 C=NVRAM  S=_NVRAM         G=DGROUP   M=uibhvinspect ACBP=48
 4DE0:1C60 0000 C=NVRAM  S=_NVRAM         G=DGROUP   M=uibhviterators ACBP=48
 4DE0:1C60 0000 C=NVRAM  S=_NVRAM         G=DGROUP   M=uictlgauge ACBP=48
 4DE0:1C60 0000 C=NVRAM  S=_NVRAM         G=DGROUP   M=uictlnumber ACBP=48
 4DE0:1C60 0000 C=NVRAM  S=_NVRAM         G=DGROUP   M=uictlbutton ACBP=48
 4DE0:1C60 0000 C=NVRAM  S=_NVRAM         G=DGROUP   M=uictltext  ACBP=48
 4DE0:1C60 0000 C=NVRAM  S=_NVRAM         G=DGROUP   M=uictldynamic ACBP=48
 4DE0:1C60 0000 C=NVRAM  S=_NVRAM         G=DGROUP   M=uictlborder ACBP=48
 4DE0:1C60 0000 C=NVRAM  S=_NVRAM         G=DGROUP   M=uipanemgr  ACBP=48
 4DE0:1C60 0000 C=NVRAM  S=_NVRAM         G=DGROUP   M=pwsrcautoposition ACBP=48
 4DE0:1C60 0000 C=NVRAM  S=_NVRAM         G=DGROUP   M=pwsrcautofreqphase ACBP=48
 4DE0:1C60 0000 C=NVRAM  S=_NVRAM         G=DGROUP   M=pwsrcautobrightness ACBP=48
 4DE0:1C60 0000 C=NVRAM  S=_NVRAM         G=DGROUP   M=hlhicolor  ACBP=48
 4DE0:1C60 0000 C=NVRAM  S=_NVRAM         G=DGROUP   M=hlpriv     ACBP=48
 4DE0:1C60 0000 C=NVRAM  S=_NVRAM         G=DGROUP   M=dvinfred   ACBP=48
 4DE0:1C60 0000 C=NVRAM  S=_NVRAM         G=DGROUP   M=dvkeypaddirect ACBP=48
 4DE0:1C60 0000 C=NVRAM  S=_NVRAM         G=DGROUP   M=ctype      ACBP=48
 4DE0:1C60 0010 C=EDATA  S=_EDATA         G=DGROUP   M=c0         ACBP=68
 4FA7:0000 0000 C=STACK  S=_STACK         G=SGROUP   M=c0         ACBP=74
 4FA7:0000 0000 C=STACK  S=_STACK         G=SGROUP   M=inientry   ACBP=74
 4FA7:0000 0100 C=STACK  S=_STACK         G=SGROUP   M=LinkStack  ACBP=74
 4FA7:0100 0010 C=STACK  S=_ESTACK        G=SGROUP   M=c0         ACBP=74
 4FB8:0000 0000 C=FAR_DATA S=_BFD           G=(none)   M=c0         ACBP=68
 4FB8:0000 0010 C=ENDFAR_DATA S=_EFD           G=(none)   M=c0         ACBP=68
 4FB9:0000 0000 C=FAR_CONST S=_BFC           G=(none)   M=c0         ACBP=68
 4FB9:0000 00D6 C=FAR_CONST S=CONFIGDATA5_CONST G=(none)   M=configdata ACBP=68
 4FC7:0000 0066 C=FAR_CONST S=CONFIGDATA6_CONST G=(none)   M=configdata ACBP=68
 4FCE:0000 007E C=FAR_CONST S=INTERRUPTCTRL5_CONST G=(none)   M=interruptctrl ACBP=68
 4FD6:0000 0014 C=FAR_CONST S=DVRS2325_CONST G=(none)   M=dvrs232    ACBP=68
 4FD8:0000 0014 C=FAR_CONST S=DVOUTPUTSCALER5_CONST G=(none)   M=dvoutputscaler ACBP=68
 4FDA:0000 0014 C=FAR_CONST S=DVIMAGEMEMORY5_CONST G=(none)   M=dvimagememory ACBP=68
 4FDC:0000 0014 C=FAR_CONST S=DV24CXX5_CONST G=(none)   M=dv24cxx    ACBP=68
 4FDE:0000 0014 C=FAR_CONST S=DVDPORT5_CONST G=(none)   M=dvdport    ACBP=68
 4FE0:0000 0014 C=FAR_CONST S=DVINPUTPORT5_CONST G=(none)   M=dvinputport ACBP=68
 4FE2:0000 0080 C=FAR_CONST S=DVCLKGENPG18E15_CONST G=(none)   M=dvclkgenpg18e1 ACBP=68
 4FEA:0000 0004 C=FAR_CONST S=DVAD98835_CONST G=(none)   M=dvad9883   ACBP=68
 4FEB:0000 0018 C=FAR_CONST S=DVAD98836_CONST G=(none)   M=dvad9883   ACBP=68
 4FED:0000 0018 C=FAR_CONST S=DVAD98837_CONST G=(none)   M=dvad9883   ACBP=68
 4FEF:0000 0010 C=FAR_CONST S=DVVPC32305_CONST G=(none)   M=dvvpc3230  ACBP=68
 4FF0:0000 0021 C=FAR_CONST S=DVVPC32306_CONST G=(none)   M=dvvpc3230  ACBP=68
 4FF3:0000 00C8 C=FAR_CONST S=DVVPC32307_CONST G=(none)   M=dvvpc3230  ACBP=68
 5000:0000 0004 C=FAR_CONST S=DVVPC32308_CONST G=(none)   M=dvvpc3230  ACBP=68
 5001:0000 0004 C=FAR_CONST S=DVVPC32309_CONST G=(none)   M=dvvpc3230  ACBP=68
 5002:0000 0004 C=FAR_CONST S=DVVPC323010_CONST G=(none)   M=dvvpc3230  ACBP=68
 5003:0000 0004 C=FAR_CONST S=DVVPC323011_CONST G=(none)   M=dvvpc3230  ACBP=68
 5004:0000 0004 C=FAR_CONST S=DVVPC323012_CONST G=(none)   M=dvvpc3230  ACBP=68
 5005:0000 0004 C=FAR_CONST S=DVVPC323013_CONST G=(none)   M=dvvpc3230  ACBP=68
 5006:0000 0004 C=FAR_CONST S=DVVPC323014_CONST G=(none)   M=dvvpc3230  ACBP=68
 5007:0000 0008 C=FAR_CONST S=DVVPC323015_CONST G=(none)   M=dvvpc3230  ACBP=68
 5008:0000 0010 C=FAR_CONST S=DVVPC323016_CONST G=(none)   M=dvvpc3230  ACBP=68
 5009:0000 0008 C=FAR_CONST S=DVVPC323017_CONST G=(none)   M=dvvpc3230  ACBP=68
 500A:0000 0007 C=FAR_CONST S=DVVPC323018_CONST G=(none)   M=dvvpc3230  ACBP=68
 500B:0000 0007 C=FAR_CONST S=DVVPC323019_CONST G=(none)   M=dvvpc3230  ACBP=68
 500C:0000 0007 C=FAR_CONST S=DVVPC323020_CONST G=(none)   M=dvvpc3230  ACBP=68
 500D:0000 0007 C=FAR_CONST S=DVVPC323021_CONST G=(none)   M=dvvpc3230  ACBP=68
 500E:0000 001B C=FAR_CONST S=DVVPC323022_CONST G=(none)   M=dvvpc3230  ACBP=68
 5010:0000 0014 C=FAR_CONST S=DVTMDSGENERIC5_CONST G=(none)   M=dvtmdsgeneric ACBP=68
 5012:0000 0058 C=FAR_CONST S=DVPW12305_CONST G=(none)   M=dvpw1230   ACBP=68
 5018:0000 003E C=FAR_CONST S=DVPW12306_CONST G=(none)   M=dvpw1230   ACBP=68
 501C:0000 0062 C=FAR_CONST S=DVPW12307_CONST G=(none)   M=dvpw1230   ACBP=68
 5023:0000 0060 C=FAR_CONST S=DVPW12308_CONST G=(none)   M=dvpw1230   ACBP=68
 5029:0000 0004 C=FAR_CONST S=DVPW12309_CONST G=(none)   M=dvpw1230   ACBP=68
 502A:0000 0004 C=FAR_CONST S=DVPW123010_CONST G=(none)   M=dvpw1230   ACBP=68
 502B:0000 0004 C=FAR_CONST S=DVPW123011_CONST G=(none)   M=dvpw1230   ACBP=68
 502C:0000 0004 C=FAR_CONST S=DVPW123012_CONST G=(none)   M=dvpw1230   ACBP=68
 502D:0000 0004 C=FAR_CONST S=DVPW123013_CONST G=(none)   M=dvpw1230   ACBP=68
 502E:0000 000D C=FAR_CONST S=DVPW123014_CONST G=(none)   M=dvpw1230   ACBP=68
 502F:0000 000D C=FAR_CONST S=DVPW123015_CONST G=(none)   M=dvpw1230   ACBP=68
 5030:0000 0021 C=FAR_CONST S=DVPW123016_CONST G=(none)   M=dvpw1230   ACBP=68
 5033:0000 0014 C=FAR_CONST S=DVZ861295_CONST G=(none)   M=dvz86129   ACBP=68
 5035:0000 0014 C=FAR_CONST S=DVTDA98515_CONST G=(none)   M=dvtda9851  ACBP=68
 5037:0000 0014 C=FAR_CONST S=DVSWITCHER_SHASTA_II5_CONST G=(none)   M=dvswitcher_shasta_ii ACBP=68
 5039:0000 0054 C=FAR_CONST S=DVCOLORSPACE5_CONST G=(none)   M=dvcolorspace ACBP=68
 503F:0000 0050 C=FAR_CONST S=DVCOLORSPACE6_CONST G=(none)   M=dvcolorspace ACBP=68
 5044:0000 0026 C=FAR_CONST S=DVFI12565_CONST G=(none)   M=dvfi1256   ACBP=68
 5047:0000 0014 C=FAR_CONST S=DVTDA98855_CONST G=(none)   M=dvtda9885  ACBP=68
 5049:0000 0065 C=FAR_CONST S=DVNJW11445_CONST G=(none)   M=dvnjw1144  ACBP=68
 5050:0000 0065 C=FAR_CONST S=DVNJW11446_CONST G=(none)   M=dvnjw1144  ACBP=68
 5057:0000 0065 C=FAR_CONST S=DVNJW11447_CONST G=(none)   M=dvnjw1144  ACBP=68
 505E:0000 0065 C=FAR_CONST S=DVNJW11448_CONST G=(none)   M=dvnjw1144  ACBP=68
 5065:0000 0006 C=FAR_CONST S=DVNJW11449_CONST G=(none)   M=dvnjw1144  ACBP=68
 5066:0000 007E C=FAR_CONST S=DVNJW114410_CONST G=(none)   M=dvnjw1144  ACBP=68
 506E:0000 0100 C=FAR_CONST S=PWCRC5_CONST   G=(none)   M=pwcrc      ACBP=68
 507E:0000 0100 C=FAR_CONST S=PWCRC6_CONST   G=(none)   M=pwcrc      ACBP=68
 508E:0000 0009 C=FAR_CONST S=PWOEM5_CONST   G=(none)   M=pwoem      ACBP=68
 508F:0000 0064 C=FAR_CONST S=PWOEM6_CONST   G=(none)   M=pwoem      ACBP=68
 5096:0000 0018 C=FAR_CONST S=HLINT5_CONST   G=(none)   M=hlint      ACBP=68
 5098:0000 0018 C=FAR_CONST S=HLINT6_CONST   G=(none)   M=hlint      ACBP=68
 509A:0000 0018 C=FAR_CONST S=HLINT7_CONST   G=(none)   M=hlint      ACBP=68
 509C:0000 0008 C=FAR_CONST S=HLINT8_CONST   G=(none)   M=hlint      ACBP=68
 509D:0000 000E C=FAR_CONST S=HLINT9_CONST   G=(none)   M=hlint      ACBP=68
 509E:0000 0018 C=FAR_CONST S=HLINT10_CONST  G=(none)   M=hlint      ACBP=68
 50A0:0000 0012 C=FAR_CONST S=HLREGISTERS5_CONST G=(none)   M=hlregisters ACBP=68
 50A2:0000 000A C=FAR_CONST S=PWHOST5_CONST  G=(none)   M=pwhost     ACBP=68
 50A3:0000 0034 C=FAR_CONST S=PWHOST6_CONST  G=(none)   M=pwhost     ACBP=68
 50A7:0000 0420 C=FAR_CONST S=PWOPERATIONS5_CONST G=(none)   M=pwoperations ACBP=68
 50E9:0000 006E C=FAR_CONST S=PWOPERATIONS6_CONST G=(none)   M=pwoperations ACBP=68
 50F0:0000 0024 C=FAR_CONST S=PWSRCAUTOCALIBRATE5_CONST G=(none)   M=pwsrcautocalibrate ACBP=68
 50F3:0000 0078 C=FAR_CONST S=PWSRCSETTINGS5_CONST G=(none)   M=pwsrcsettings ACBP=68
 50FB:0000 0096 C=FAR_CONST S=PWSRCDISPLAY5_CONST G=(none)   M=pwsrcdisplay ACBP=68
 5105:0000 0060 C=FAR_CONST S=PWSRCDISPLAY6_CONST G=(none)   M=pwsrcdisplay ACBP=68
 510B:0000 003C C=FAR_CONST S=PWSRCTV5_CONST G=(none)   M=pwsrctv    ACBP=68
 510F:0000 0014 C=FAR_CONST S=PWSRCTV6_CONST G=(none)   M=pwsrctv    ACBP=68
 5111:0000 0001 C=FAR_CONST S=PWSRCTV7_CONST G=(none)   M=pwsrctv    ACBP=68
 5112:0000 0002 C=FAR_CONST S=PWSRCTV8_CONST G=(none)   M=pwsrctv    ACBP=68
 5113:0000 0028 C=FAR_CONST S=MYAPI5_CONST   G=(none)   M=myapi      ACBP=68
 5116:0000 0010 C=ENDFAR_CONST S=_EFC           G=(none)   M=c0         ACBP=68
 5117:0000 0000 C=FAR_BSS S=_BFB           G=(none)   M=c0         ACBP=68
 5117:0000 0010 C=ENDFAR_BSS S=_EFB           G=(none)   M=c0         ACBP=68
 5118:0000 0000 C=FAR_HEAP S=_FARHEAP       G=(none)   M=c0         ACBP=68
 5118:0000 0010 C=ENDFAR_HEAP S=_EFH           G=(none)   M=c0         ACBP=68
 5119:0000 0010 C=INITIALENTRY S=INITIALENTRY   G=(none)   M=inientry   ACBP=68
 511A:0000 0F90 C=AMXD   S=AMXDATA        G=(none)   M=romcfg     ACBP=68
 511A:0F90 0000 C=AMXD   S=AMXDATA        G=(none)   M=AJ831PRF   ACBP=68
 5213:0000 00CA C=AMXD   S=AMXMES         G=(none)   M=romcfg     ACBP=60
 5220:0000 0540 C=AMXS   S=AMXSTAK        G=(none)   M=romcfg     ACBP=68
 5220:0540 0000 C=AMXS   S=AMXSTAK        G=(none)   M=AJ831PRF   ACBP=68
 5274:0000 0480 C=AMXS   S=@T@S1          G=(none)   M=romcfg     ACBP=60
 52BC:0000 04C0 C=AMXS   S=@T@S2          G=(none)   M=romcfg     ACBP=60
 5308:0000 02F4 C=AMXS   S=@T@S3          G=(none)   M=romcfg     ACBP=60
 5337:0004 0000 C=       S=AMXCODL        G=(none)   M=AJ831PRF   ACBP=40
 5337:0004 0000 C=PROG   S=AMXCODP        G=(none)   M=AJ831PRF   ACBP=40
 5337:0004 0000 C=TEXT   S=AMXCODT        G=(none)   M=AJ831PRF   ACBP=40


  Address         Publics by Name

 0069:1DE9       AABERH
 0069:0E7E       AACLK
 0069:1DFB       AADERH
 0069:1522 idle  AAEND
 0069:2244       AAENTR
 0069:04E8       AAEVCRE
 0069:052C       AAEVDEL
 0069:076E       AAEVNT
 0069:0753       AAEVRD
 0069:04A5       AAEVRR
 0069:0656       AAEVSIG
 0069:077E       AAEVTAG
 0069:056F       AAEVWAT
 0069:15DB       AAFATL
 0069:164B idle  AAHOOK
 0069:28A9 idle  AAIDTM
 0069:28A9 idle  AAIDTR
 0069:28A9 idle  AAIDTS
 0069:28A9 idle  AAIDTW
 0069:28A9 idle  AAIDTX
 0069:1D58       AAINT
 0069:1DAA       AAINX
 0069:26A7       AAISPM
 0069:28A9 idle  AAISPW
 0069:1E64       AAITRP
 0069:264C       AAIVTR
 0069:267D       AAIVTW
 0069:260D       AAIVTX
 0069:09C1       AAMAU
 0069:0855       AAMFRE
 0069:0825       AAMGEH
 0069:0806       AAMGET
 0069:0972       AAMGSZ
 0069:07FA       AAMHAN
 0069:078C       AAMMRR
 0069:1DF2       AAOVFH
 0069:1623       AAPRVL
 0069:1604       AAPRVR
 0069:1734       AARESUM
 0069:17BF       AASEND
 0069:1AFA       AASGNL
 0069:1B89       AASGRD
 0069:1B9C       AASGRES
 0069:1A60       AASGWAT
 0069:01F1       AASMCRE
 0069:0255       AASMDEL
 0069:0393       AASMFRE
 0069:0466       AASMGET
 0069:0362       AASMRLS
 0069:01B0       AASMRR
 0069:0297       AASMRSV
 0069:03B3       AASMSIG
 0069:0497       AASMTAG
 0069:0297       AASMWAT
 0069:174A       AASUSP
 0069:1239       AATICK
 0069:272E       AATKCRE
 0069:1CEF       AATKID
 0069:2536       AATKPRY
 0069:1BBC       AATKSTS
 0069:1CA5       AATKTAG
 0069:1D40       AATKTCB
 0069:124F       AATMCNV
 0069:106D       AATMCRE
 0069:10F2       AATMDEL
 0069:11E9       AATMRD
 0069:12B9       AATMTAG
 0069:1146       AATMWR
 0069:170C       AATRIG
 0069:1343 idle  AAVER
 0069:1989       AAWAIT
 0069:190E       AAWAKC
 0069:1917       AAWAKCS
 0069:19FA       AAWAKE
 0069:1A4E       AAWAPR
 0069:1992       AAWATM
 0069:1327 idle  AMBITN
 0069:1323 idle  AMBITP
 0069:16FC       AMCFH
 0069:158D       AMERR
 0069:1337       AMGDP
 0069:133D       AMGVP
 0069:1600 idle  AMHALT
 0069:1361       AMHANG
 0069:135C idle  AMHANGC
 0069:13BA idle  AMIDLE
 0069:136D       AMIHNG
 0069:28B0       AMINPM
 0069:26D4       AMINRM
 0069:1E54 idle  AMIRET
 0069:28B0 idle  AMIRPM
 0069:2708 idle  AMIRRM
 0069:0DA6       AMKRNL
 0069:0E0F       AMKRNX
 0069:21DA       AMMAL
 0069:1E54       AMPOPF
 0069:169A       AMSGEV
 0069:138B idle  AMSHED
 0069:1438       AMTASK
 0069:0F93       AMTIMR
 0069:2527 idle  AMTKPRY
 0069:2595       AMTKSLC
 0069:11D7       AMTTRD
 0069:113D       AMTTWR
 0069:1577       AMUPEM
 0069:134B       AMUSRP
 0069:1CFC       AMUTAG
 0000:03A7 idle  DGROUP@
 0000:0243       F_LDIV@
 0000:0252       F_LMOD@
 0000:024A       F_LUDIV@
 0000:025A       F_LUMOD@
 0000:0329       F_LXLSH@
 0000:02EE       F_LXMUL@
 0000:03FA       F_LXRSH@
 0000:0308       F_LXURSH@
 0000:039A idle  F_OVERFLOW@
 0000:0506       F_PADA@
 0000:0550 idle  F_PSBA@
 0000:03AC       F_PSBP@
 0000:03DB       F_SCOPY@
 0000:0243 idle  LDIV@
 0000:0252 idle  LMOD@
 0000:024A idle  LUDIV@
 0000:025A idle  LUMOD@
 0000:0329 idle  LXLSH@
 0000:02EE idle  LXMUL@
 0000:03FA idle  LXRSH@
 0000:0308 idle  LXURSH@
 0000:0240 idle  N_LDIV@
 0000:024F idle  N_LMOD@
 0000:0247 idle  N_LUDIV@
 0000:0257 idle  N_LUMOD@
 0000:0326 idle  N_LXLSH@
 0000:03F7 idle  N_LXRSH@
 0000:0305 idle  N_LXURSH@
 0000:039A idle  N_OVERFLOW@
 0000:0503 idle  N_PADA@
 0000:054D idle  N_PSBA@
 0000:03A9 idle  N_PSBP@
 0000:039A idle  OVERFLOW@
 0000:0506 idle  PADA@
 0000:0550 idle  PSBA@
 0000:03AC idle  PSBP@
 0000:03DB idle  SCOPY@
 4DE0:126C idle  _afcCOUNT
 0069:1F0F       _ajclk
 0069:0CBA idle  _AJDATP_
 0069:0C50       _ajentr
 0069:1F31       _ajevcre
 0069:1F56 idle  _ajevdel
 0069:1F79 idle  _ajevnt
 0069:1F64 idle  _ajevrd
 0069:1F53       _ajevsig
 0069:1F7C idle  _ajevtag
 0069:1F50       _ajevwat
 0069:0C37       _ajint
 0069:0C3A       _ajinx
 0069:1FD8 idle  _ajispm
 0069:0C3D idle  _ajitrp
 0069:1FB2 idle  _ajivtr
 0069:1FC5       _ajivtw
 0069:1F98 idle  _ajivtx
 0069:0D93 idle  _ajmau
 0069:0D69       _ajmfre
 0069:0D3D idle  _ajmgeh
 0069:0D14       _ajmget
 0069:0D79       _ajmgsz
 0069:0CF0 idle  _ajmhan
 0069:0CEA idle  _ajmodl
 0069:2004       _ajresum
 0069:2023       _ajsend
 0069:200E idle  _ajsendp
 0069:2027       _ajsenw
 0069:2012 idle  _ajsenwp
 0069:2099       _ajsgnl
 0069:20BE idle  _ajsgrd
 0069:20C1 idle  _ajsgres
 0069:206A       _ajsgwat
 0069:2122       _ajsmcre
 0069:218E       _ajsmdel
 0069:2181 idle  _ajsmfre
 0069:2167 idle  _ajsmget
 0069:2174       _ajsmrls
 0069:2141       _ajsmrsv
 0069:215A       _ajsmsig
 0069:219B idle  _ajsmtag
 0069:2141       _ajsmwat
 0069:1FFA       _ajsusp
 0069:1F12       _ajtick
 0069:21B7       _ajtkcre
 0069:20E8       _ajtkid
 0069:21CD       _ajtkpry
 0069:20EB       _ajtksts
 0069:20CE       _ajtktag
 0069:20FE       _ajtktcb
 0069:1EFC       _ajtmcnv
 0069:1EA4       _ajtmcres
 0069:1ECE       _ajtmdel
 0069:1EEC       _ajtmrd
 0069:1F17 idle  _ajtmtag
 0069:1ED8       _ajtmwr
 0069:1FEE       _ajtrig
 0069:0C8B       _ajupt
 0069:0CD3 idle  _AJVERP_
 0069:204D idle  _ajwait
 0069:2040 idle  _ajwakc
 0069:2043 idle  _ajwakcs
 0069:2050       _ajwake
 0069:205A idle  _ajwapr
 0069:205D       _ajwatm
 04A1:0138       _AllocMemory
 04A1:0309       _AllocMemoryWithError
 0069:0000       _AMDATP_
 0069:12CB idle  _AMVER_
 0069:0004       _AMXUPT_
 0000:0347 idle  _atexit
 0000:048C idle  _atoi
 0000:0417       _atol
 0A19:042B       _BackgroundMgr
 4DE0:0618       _bgndid
 4DE0:061E       _bksemid
 4767:0127       _BlitMapSetTranslucent
 1D84:1F62 idle  _BlueScreen
 3E84:1DE0 idle  _Bri_Con_Col_Back
 3E84:1D9A idle  _Bri_Con_Col_Zero
 449A:0040       _BroadcastOperationID
 2347:1F09 idle  _BufferBytes
 0BF9:017E idle  _CalcData
 1C48:0C01 idle  _ChangeChannelMute
 1781:19A6       _ChangePipAlpha
 1781:190C       _ChangePipLeftPos
 1781:16C2       _ChangePipSize
 1781:1959       _ChangePipTopPos
 1B07:0CBE       _ChangeTunerStandard
 14CD:0F88 idle  _CheckFormat
 1D84:205D       _Check_Video_Caption_Pos
 14CD:270A idle  _ColseCaptureSetup
 04A1:029B       _CompareStrings
 0059:001B       _ComputeHorzFrequency
 0059:0006       _ComputeVertFrequency
 0059:0033       _ComputeVertFreqX100
 02F4:0047       _ConfigDataGetPointer
 02F4:000E       _ConfigDataInitialize
 04A1:0024       _CopyMemory
 0301:0475       _DataMgrForceRead
 0301:03CE       _DataMgrForceUpdate
 0301:062C       _DataMgrGetNodeDefaults
 0301:0003       _DataMgrInitialize
 0301:0664 idle  _DataMgrIsNodeCal
 0301:064D idle  _DataMgrIsNodeConst
 0301:026C       _DataMgrLockNodeForRead
 0301:0294       _DataMgrLockNodeForWrite
 0301:0351       _DataMgrNodeUpdated
 0301:0543       _DataMgrReset
 0301:0610       _DataMgrResetNode
 0301:067B       _DataMgrRestartUpdate
 0301:02F0       _DataMgrSetCallback
 0301:02CE       _DataMgrUnlockNode
 0301:02BC       _DataMgrUnlockNodeDirty
 0301:0306       _DataMgrUpdateImmediate
 0301:05F9 idle  _DataMgrUpdateMode
 0301:03AF       _DataMgrValidateNodeSize
 4DE0:0000 idle  _DATASEG@
 4DE0:0630       _dmsemid
 2AA2:19F0 idle  _DPMSTimer
 4DE0:0632       _dpsemid
 4655:0281       _dv2wireBlockRead
 4655:0195       _dv2wireBlockReadAddress
 4655:0115       _dv2wireBlockWrite
 4655:007D       _dv2wireBlockWriteAddress
 4655:0003       _dv2wireInitialize
 4655:0009       _dv2wireReserve
 1D1C:02E3       _dvDriverClassService
 1D1C:03E9       _dvDriverClassServiceDeviceIDs
 1D1C:03B5       _dvDriverClassServiceDevices
 1D1C:02A3       _dvDriverCreateRequestData
 1D1C:04EC       _dvDriverGetOpDescriptor
 1D1C:00B7       _dvDriverGetParameter
 1D1C:0161       _dvDriverGetParameterDescriptor
 1D1C:04A4       _dvDriverGetParameterDword
 1D1C:01B6       _dvDriverIsRequestAvailable
 1D1C:0063       _dvDriverService
 1D1C:0555 idle  _dvDriverServiceGetFirstClassDev
 1D1C:0007       _dvDriverServiceInitialize
 1D1C:0047       _dvDriverServiceInitializeDrivers
 1D1C:0520       _dvDriverServiceSend
 1D1C:010C       _dvDriverSetParameter
 1D1C:043B       _dvDriverSetParameterDword
 1D1C:046F idle  _dvDriverSetParameterPointer
 1D1C:020B       _dvDriverValidateData
 29DA:0412 idle  _dvGPIOgetBool
 29DA:02A7       _dvGPIOgetField
 29DA:04A2 idle  _dvGPIOgetFlags
 29DA:0443       _dvGPIOgetMask
 29DA:0205       _dvGPIOInitGPO
 29DA:0032       _dvGPIOInitialize
 29DA:0253       _dvGPIOsetField
 4D85:01AB       _dvInfraredGetRepeatCount
 4D85:01B9 idle  _dvInfraredSetRepeatCount
 4934:00A5 idle  _dvIRAnyKey
 4D85:0000       _dvIRDriverInitialize
 4D85:020E       _dvIRGetJoystickData
 4D85:01CF       _dvIRGetKeycode
 4934:005A       _dvIRProcessJoystickCommand
 4934:0081       _dvIRProcessKeycodeCommand
 4934:0008       _dvIRremoteInitialize
 4D85:01C4       _dvIRSetKeycode
 44FA:0425 idle  _dvKeypadAnyKey
 4DD0:0003       _dvKeypadDriverInit
 44FA:00F8       _dvKeypadInitialize
 4DD0:0027       _dvKeypadPoll
 44FA:0204       _dvKeypadProcessCommand
 44FA:000A       _dvKeypadService
 46E0:0514       _dvLEDBlinkPause
 46E0:0526       _dvLEDBlinkResume
 46E0:017B idle  _dvLEDGet
 46E0:0038       _dvLEDInitialize
 46E0:013B idle  _dvLEDSet
 46E0:01C4 idle  _dvLEDSetStateMultiple
 46E0:0189       _dvLEDSetStateSingle
 46E0:0513       _dvLEDUpdateLEDs
 2A5D:0318 idle  _dvOemInterfaceBlockAccess
 2A5D:01BE idle  _dvOemInterfaceBlockAccessDevice
 2A5D:0347       _dvOemInterfaceBlockRead
 2A5D:0365       _dvOemInterfaceBlockReadAddress
 2A5D:0385       _dvOemInterfaceBlockWrite
 2A5D:03A3       _dvOemInterfaceBlockWriteAddress
 2A5D:03FA       _dvOemInterfaceGetId
 2A5D:000C idle  _dvOemInterfaceGetIndex
 2A5D:0040       _dvOemInterfaceInitialize
 2A5D:018A       _dvOemInterfaceReadRegisters
 2A5D:0062 idle  _dvOemInterfaceRegistersAccess
 2A5D:03C7 idle  _dvOemInterfaceReserve
 2A5D:01A4       _dvOemInterfaceWriteRegisters
 4760:0007       _dvOemLampBacklightInit
 4760:0028       _dvOemLampEnable
 4760:003A       _dvOemLampGetEnable
 4760:000B       _dvOEMLampGetLampRange
 4760:000A       _dvOemLampSetLevel
 4765:0013       _dvOemUnitPowerIsOn
 4765:0008       _dvOemUnitPowerSet
 455C:000B idle  _dvPwmEnable
 455C:021A       _dvPwmGetLevel
 455C:022E       _dvPwmGetRange
 455C:009B idle  _dvPwmInitialize
 455C:016C       _dvPwmSetLevel
 4DE0:160A idle  _errno
 0000:0172       _exit
 0A6A:04FC       _FatalExit
 04A1:0002       _FillMemory
 2347:1B92 idle  _FindHostTask
 04A1:021A       _FreeMemory
 1D84:1ED7 idle  _Get3230SignalLoss
 1D84:1F45 idle  _Get3230VideoStandard
 1C0C:0398       _GetAFCStatus
 04A1:0130 idle  _GetAllocatedMemorySize
 1D84:2036 idle  _GetBlueScreen1230
 2347:2114 idle  _GetBytes
 1D84:18DD       _GetCurrentSourceID
 1D84:1D13 idle  _GetFP13State
 1D84:1C39 idle  _GetFP13State1111
 1C48:0CFA idle  _GetMuteState
 3E84:1F3F       _GetnotsaveFlag
 1B07:0E80 idle  _GetTunerAFCStandard
 1B07:0DCA       _GetTunerAudioStandard
 1B07:0EDE idle  _GetTunerHz50_60
 1B07:0C09       _GetTunerStatus
 1B07:0D00       _GetTunerVideoStandard
 1B07:1021       _GetVideoAudioStandard
 4DE0:0638       _gisemid
 0DB8:3AC0 idle  _GPGetGPortPhase
 4DE0:00C8 idle  _GPMonitorVSyncData
 4DE0:062C       _gpsemid
 4FDC:0000       _g_drv24CxxDriverVTable
 4FED:0004       _g_drvadAD9883DriverVTable
 4FE2:006C       _g_drvckPG18E1DriverVTable
 503F:003C       _g_drvColorSpaceDriverVTable
 5030:000D       _g_drvdePW1230DriverVTable
 5047:0000       _g_drvdeTDA9885DriverVTable
 4FDE:0000       _g_drvDPortDriverVTable
 5044:0012       _g_drvFI1256DriverVTable
 4FDA:0000       _g_drvImageMemoryDriverVTable
 4FE0:0000       _g_drvInputPortDriverVTable
 5066:006A       _g_drvNJW1144DriverVTable
 4FD8:0000       _g_drvOutputScalerDriverVTable
 4FD6:0000       _g_drvRS232DriverVTable
 5037:0000       _g_drvSwitcherSHASTA2DriverVTable
 5035:0000       _g_drvTDA9851DriverVTable
 5010:0000       _g_drvTMDSGenericDriverVTable
 500E:0007       _g_drvvdVPC3230DriverVTable
 5033:0000       _g_drvZ86129DriverVTable
 4DE0:0F32       _g_pGlobals
 2106:01AB       _hlAdjustClockRates
 4436:03B3       _hlAutoEndVideoInit
 4436:0279       _hlAutoForceInterlacedMode
 4436:000B       _hlAutoInitialize
 4436:0284       _hlAutoInitVideoPort
 4436:01EE idle  _hlAutoIsInterlaced
 4436:0247 idle  _hlAutoIsInterlacedDetected
 4436:001E       _hlAutoPhaseModeEnable
 29BB:010C       _hlCfgWaitStates
 2106:0132 idle  _hlChangeMemConstraint
 2106:0245 idle  _hlChangeMemoryConfiguration
 27FB:0E3F       _hlDispCheckFramelock
 27FB:0EFE       _hlDispGetCurrentPanelParams
 27FB:08F9 idle  _hlDisplayGetBrightness
 27FB:0D77       _hlDisplayHasBorder
 27FB:0007       _hlDisplayInitialize
 27FB:0049       _hlDisplayInitTCON
 27FB:0865       _hlDisplaySetBlankColor
 27FB:08B5 idle  _hlDisplaySetBrightness
 27FB:0D04       _hlDisplaySetColorMatrix
 27FB:094D       _hlDisplaySetContrast
 27FB:0AA9       _hlDisplaySetPower
 27FB:0D7A       _hlDisplaySetVLockMode
 27FB:0C52       _hlDisplaySetWindowPos
 27FB:0856 idle  _hlDisplayUpdateShadowedRegisterImages
 27FB:0E96       _hlDispSetPanel
 441A:0051 idle  _hlDPortISPGetVBlankCount
 441A:0005       _hlDPortISPInitialize
 209C:0320       _hldpRegisterGet
 209C:0338       _hldpRegisterSet
 209C:02F3 idle  _hledpRegisterGet
 209C:030B       _hledpRegisterSet
 209C:02C6       _hlegpRegisterGet
 209C:02DE       _hlegpRegisterSet
 209C:037A       _hlGammaRegisterSet
 209C:01BE       _hlgcRegisterGet
 209C:01D5       _hlgcRegisterSet
 2E6F:0082       _hlGenCtlBlockOperationLock
 2E6F:00CB       _hlGenCtlBlockOperationUnlock
 2E6F:00E9       _hlGenCtlHasFailsafe
 2E6F:0009       _hlGenCtlInitialize
 2E6F:005C idle  _hlGenCtlIsLockEnabled
 2E6F:004A       _hlGenCtlLockRegistersEnable
 2E6F:003C idle  _hlGenCtlLockRegistersFromUpdate
 2E6F:005F idle  _hlGenCtlLockSyncStateClear
 2E6F:0067 idle  _hlGenCtlLockSyncStateRestore
 2E6F:006F idle  _hlGenCtlShadowRegistersEnable
 2E6F:0081 idle  _hlGenCtlShadowRegistersUpdate
 2106:0160       _hlGetClockRates
 2106:0180       _hlGetClockRatesPtr
 2106:034E       _hlGetInputResolutionRect
 2106:0339       _hlGetInputResolutionSize
 464A:0070       _hlGetInternalCpuRamSize
 2106:0313 idle  _hlGetMemoryConfiguration
 2981:03A1       _hlGetSettings
 2106:0102       _hlGetSignalValidFlag
 4389:0339 idle  _hlGPortGetActualHLines
 4389:032B       _hlGPortGetInputSourceHLines
 4389:02FD       _hlGPortInputResolutionChange
 4476:005F       _hlGPortISPEnable
 4476:007F       _hlGPortISPGetVBlankCount
 4476:000F       _hlGPortISPInitialize
 4476:007B idle  _hlGPortISPIsSafetyModeEnabled
 4389:0347       _hlGPortSetActualHLines
 209C:01E9       _hlgpRegisterGet
 209C:0200       _hlgpRegisterSet
 4389:000F idle  _hlGraphicGetCaptureWindowExpansion
 4389:00A9 idle  _hlGraphicGetCaptureWindowOffsets
 4389:0202       _hlGraphicGetCaptureWindowPos
 4389:0025       _hlGraphicSetCaptureWindowExpansion
 4389:00C0       _hlGraphicSetCaptureWindowPos
 27FB:0D00       _hlHasColorMatrix
 27FB:0D74       _hlHasColorWarping
 4CD7:0002       _hlHiColorDrawBitmap
 4CD7:019C       _hlHiColorDrawTiledBitmap
 4CD7:015D       _hlHiColorPackedToRef
 4CD7:013E       _hlHiColorRefToPacked
 4CD7:0116       _hlHiColorRgbToPacked
 2106:0006       _hlHlayerInit
 209C:0299 idle  _hlhsRegisterGet
 209C:02B1       _hlhsRegisterSet
 432A:01D2       _hlImageMemCalcPoint
 432A:0051       _hlImageMemFill
 432A:000B       _hlImageMemFillRect
 432A:027D idle  _hlImageMemPixelCount
 432A:00C7 idle  _hlImageMemReadRect
 432A:030F       _hlImagePixelGranularity
 432A:034D       _hlImageRead24BitPixel
 432A:02D6       _hlImageWordGranularity
 461D:0083       _hlInfraredGetData
 461D:012A idle  _hlInfraredGetPulseWidth
 461D:0007       _hlInfraredInitialize
 461D:0115 idle  _hlInfraredInitializeEdgeDetectMode
 461D:016B idle  _hlInfraredSetIRPOL
 461D:001C       _hlInfraredSetTimeBase
 2981:0003       _hlInitialize
 2106:001F       _hlInitializeAfterDataMgr
 293C:0001       _hlInitTimers
 1FB0:0149       _hlIntClearActiveFlag
 1FB0:0115       _hlIntClearPendingFlag
 1FB0:012F       _hlIntClearPendingFlagFromTheInterrupt
 1FB0:007F idle  _hlIntDisableAll
 1FB0:00F7       _hlIntEnable
 1FB0:0002       _hlIntInitialize
 1FB0:0038       _hlIntMasterEnable
 209C:0475       _hlintRegisterGet
 209C:048D       _hlintRegisterSet
 1FB0:0163 idle  _hlIntSetExternalIntMode
 1FB0:0181       _hlIntSetPolarity
 1FB0:019F       _hlIntSetPriority
 1FB0:0010       _hlIntSetVectorBase
 209C:041B       _hlioRegisterGet
 209C:0433       _hlioRegisterSet
 209C:051C       _hlirRegisterGet
 209C:0534       _hlirRegisterSet
 2106:0225       _hlIsModeSupported
 2106:0109       _hlIsSourceGport
 2106:00A6       _hlIsWrapModeOn
 2106:01D6       _hlMemChangeNeeded
 464A:0043 idle  _hlMiscChipSelectEnable
 29BB:00B5       _hlMiscCSWaitStatesSet
 4581:0411       _hlOsdBlankModeEnable
 4581:0708       _hlOsdCaptureOverlap
 4581:06D3       _hlOsdComputeOsdSize
 3DCA:00ED       _hlOsdGetGrayMode
 3DCA:00E7       _hlOsdGetGrayTable
 4581:0068 idle  _hlOsdGetMode
 4581:0397       _hlOsdGetWindowPos
 4581:0002       _hlOsdInitialize
 4581:0455 idle  _hlOsdIsBlankModeEnabled
 4581:0687       _hlOsdIsPixelDoublingEnabled
 4581:010F idle  _hlOsdIsWindowEnabled
 3DCA:01E0       _hlOsdLoColorDrawBitmap
 3DCA:02CC       _hlOsdLoColorDrawBitmapRect
 3DCA:0106       _hlOsdLoColorDrawRectangle
 3DCA:03A4       _hlOsdLoColorGetPixel
 4581:046D       _hlOsdOverlayFunctionEnable
 209C:03F9       _hlosdPaletteRegisterGet
 209C:03D7       _hlosdPaletteRegisterSet
 4581:0633       _hlOsdPixelDoublingEnable
 209C:023F       _hlosdRegisterGet
 209C:0257       _hlosdRegisterSet
 3DCA:00F1       _hlOsdSetGrayMode
 4581:0067       _hlOsdSetMode
 4581:061D idle  _hlOsdSetOverlayColorGain
 4581:048C       _hlOsdSetOverlayColors
 3DCA:0024       _hlOsdSetPalette
 3DCA:0043       _hlOsdSetPaletteColor
 3DCA:000D idle  _hlOsdSetPaletteGain
 4581:0116       _hlOsdSetWindowPos
 4581:073D       _hlOsdUpdateDuringBlankingPeriod
 4581:0075       _hlOsdWindowEnable
 2106:036F       _hlPositionUpdateDuringBlankingPeriod
 29BB:005E       _hlRamWaitStatesSet
 4079:0462       _hlRect1EnclosesRect2
 4079:00EE       _hlRectCenterOnPoint
 4079:008B       _hlRectCenterRect
 4079:000A       _hlRectCopy
 4079:0215       _hlRectExpandToFit
 4079:0199       _hlRectFromSize
 4079:0205       _hlRectHeight
 4079:0153       _hlRectInflate
 4079:034A       _hlRectLimitToRect
 4079:0300       _hlRectLocate
 4079:0045       _hlRectOffset
 4079:01F6       _hlRectWidth
 209C:01BD       _hlRegisterShadowFill
 209C:0166       _hlRegisterWaitForField
 293C:0445       _hlResetWatchDogTimer
 29BB:0007       _hlRomWaitStatesSet
 25F7:03AB       _hlRotateRectIfNeeded
 209C:0592       _hlrsDelayedRegisterWrite
 209C:0576       _hlrsDelayedWriteBegin
 209C:05E3       _hlrsDelayedWriteEnd
 209C:05F3       _hlrsDelayedWriteUpdateDuringBlankingPeriod
 209C:04EF       _hlrsRegisterGet
 209C:0507       _hlrsRegisterSet
 25F7:0431       _hlScalerConfigure
 25F7:038E idle  _hlScalerFlipping
 25F7:02C3 idle  _hlScalerGetDesiredOutputRes
 25F7:02D8       _hlScalerGetInputRect
 25F7:0250 idle  _hlScalerGetInputRes
 25F7:023E       _hlScalerGetMode
 25F7:02EF       _hlScalerGetOutputAspect
 25F7:02FD       _hlScalerGetOutputRect
 25F7:02AE idle  _hlScalerGetOutputRes
 25F7:052B       _hlScalerGetZoom
 25F7:03F9 idle  _hlScalerHasEnhancedVideo
 25F7:03F6 idle  _hlScalerHasKeystone
 25F7:03EE       _hlScalerHasNonlinear
 25F7:03EB idle  _hlScalerHasRotation
 25F7:03F2       _hlScalerHasZoom
 25F7:000D       _hlScalerInit
 25F7:021E idle  _hlScalerInputRes
 25F7:03A4       _hlScalerIsRotateEnabled
 25F7:03FC       _hlScalerKeystoneMode
 25F7:0407 idle  _hlScalerKeystoneModeGet
 25F7:0377       _hlScalerNonlinearity
 25F7:033F       _hlScalerOffset
 25F7:0265       _hlScalerOutputRes
 25F7:0314 idle  _hlScalerPosition
 25F7:0399       _hlScalerRotate
 25F7:048B       _hlScalerSetFrameBufferMode
 25F7:013D idle  _hlScalerSetInputClipRect
 25F7:0515       _hlScalerSetKeystoneVertScaleMax
 25F7:0420       _hlScalerSetLinearRegion
 25F7:0233       _hlScalerSetMode
 25F7:01A5 idle  _hlScalerSetOutputDispRect
 25F7:0110       _hlScalerSetupWindows
 25F7:0520       _hlScalerSetZoom
 25F7:0354       _hlScalerSharpness
 25F7:04A2 idle  _hlScalerUpdateCoefficients
 25F7:04F4       _hlScalerUpdateDuringBlankingPeriod
 25F7:040B       _hlScalerUpdateEnable
 25F7:00DD idle  _hlScalerVSSetWindow
 4DE0:0628       _hlsemid
 40C3:052D idle  _hlSerialClearReceiveBuffer
 40C3:0517 idle  _hlSerialClearTransmitBuffer
 40C3:053D       _hlSerialEnable
 40C3:00AF       _hlSerialGetBaudRate
 40C3:0290 idle  _hlSerialGetByte
 40C3:02B1       _hlSerialGetData
 40C3:0565 idle  _hlSerialGetEnable
 40C3:000C       _hlSerialInitialize
 40C3:0569       _hlSerialRestart
 40C3:00C7       _hlSerialSetBaudRate
 40C3:04F8 idle  _hlSerialTransmitByte
 40C3:03D5       _hlSerialTransmitData
 2106:018B       _hlSetClockRates
 27FB:0CE9       _hlSetGammaEntry
 2106:029F       _hlSetMemoryConfiguration
 464A:000B idle  _hlSetMiscChipSelectBaseAddress
 2106:00AF       _hlSetSignalValidFlag
 4079:01C8       _hlSizeFromRect
 293C:0276 idle  _hlTimerGetTimeTicks
 293C:017F idle  _hlTimerGetTimeuSecs
 293C:02E8       _hlTimerRestore
 293C:0295       _hlTimerSave
 293C:0063       _hlTimerSetup
 293C:00A0 idle  _hlTimerSetupTicks
 293C:0361       _hlTimersSetPrescaler
 293C:03D3       _hlTimerStart
 293C:0407       _hlTimerStop
 209C:0448       _hltmRegisterGet
 209C:0460       _hltmRegisterSet
 209C:0549 idle  _hltwRegisterGet
 209C:0561 idle  _hltwRegisterSet
 4281:006B       _hlVideoCaptureEnable
 4281:0079 idle  _hlVideoGetCaptureWindowExpansion
 4281:0113 idle  _hlVideoGetCaptureWindowOffsets
 4281:027F       _hlVideoGetCaptureWindowPos
 4281:000D       _hlVideoInitialize
 4281:008F       _hlVideoSetCaptureWindowExpansion
 4281:012A       _hlVideoSetCaptureWindowPos
 4281:0457       _hlVideoSetFrameBufferMode
 4281:038A       _hlVideoSetInputMode
 4281:036F       _hlVideoSetRotateMode
 4281:04A1       _hlVPortInputResolutionChange
 4488:005C       _hlVPortISPEnable
 4488:007C       _hlVPortISPGetVBlankCount
 4488:000B       _hlVPortISPInitialize
 4488:0078 idle  _hlVPortISPIsSafetyModeEnabled
 209C:0214       _hlvpRegisterGet
 209C:022B       _hlvpRegisterSet
 209C:026C       _hlvsRegisterGet
 209C:0284       _hlvsRegisterSet
 209C:034D       _hlwdRegisterGet
 209C:0365       _hlwdRegisterSet
 4DE0:0626       _hssemid
 1D84:2189       _INSearchMenu
 0460:0139       _IntCtrlGetHandlerProc
 0460:0009       _IntCtrlInitialize
 0460:011D       _IntCtrlSetHandlerProc
 4DE0:062A       _iosemid
 1D1C:059E       _i_dvDriverUnusedFunctionCP
 1D1C:059B       _i_dvDriverUnusedFunctionCPC
 29DA:0599       _i_dvGPIOgetAddress
 29DA:05E8       _i_dvGPIOgetMask
 29DA:04E3 idle  _i_dvGPIOgetPortType
 29DA:0549 idle  _i_dvGPIOgetShadowPointer
 29DA:052D       _i_dvGPIOlock
 29DA:053E       _i_dvGPIOunlock
 4228:00FA       _i_dvScalerGetClipping
 4228:038F       _i_dvScalerGetClippingOffset
 4207:000B       _i_dvScalerGetFilter
 4228:0539       _i_dvScalerGetLinearRegion
 4228:000D       _i_dvScalerGetStretch
 4228:0572       _i_dvScalerLinearRegionGetRange
 411D:000F       _i_dvScalerModeGet
 411D:007A       _i_dvScalerModeSet
 4207:009D idle  _i_dvScalerResetFilter
 4228:01EE       _i_dvScalerSetClipping
 4228:03F0       _i_dvScalerSetClippingOffset
 4207:0022       _i_dvScalerSetFilter
 4228:0550       _i_dvScalerSetLinearRegion
 4228:0024       _i_dvScalerSetStretch
 4207:008A       _i_dvScalerSetupFilter
 4228:00CF       _i_dvScalerStretchGetRange
 411D:0178       _i_dvScalerUpdate
 41BB:0170       _i_dvScalerZoomGetCenter
 41BB:004C       _i_dvScalerZoomGetMagnification
 41BB:040D       _i_dvScalerZoomGetMaximum
 41BB:046D       _i_dvScalerZoomGetMinimum
 41BB:02FA       _i_dvScalerZoomGetPan
 41BB:005F       _i_dvScalerZoomGetRange
 41BB:000A       _i_dvScalerZoomInitialize
 41BB:002B       _i_dvScalerZoomReset
 41BB:0185       _i_dvScalerZoomSetCenter
 41BB:019A       _i_dvScalerZoomSetMagnification
 41BB:0336       _i_dvScalerZoomSetPan
 41BB:04B4 idle  _i_dvZoomSetRect
 2106:073C idle  _i_hlCalculateDpldly
 2106:0650 idle  _i_hlCalculateFramelockValues
 2106:13D0       _i_hlCheckFailsafeMode
 27FB:0F2F       _i_hlDisplayVsyncProcessing
 441A:00E7       _i_hlDPortEnableDvpcntUpdates
 441A:0092       _i_hlDPortISPGetDvpcnt
 441A:0055       _i_hlDPortISPGetOsdColor
 441A:0082       _i_hlDPortISPSetOsdColor
 2106:1444       _i_hlGetActualRequestedDCLK
 2106:1317       _i_hlGetDvpcnt
 2106:0631       _i_hlGetIOResolutionRects
 2106:0564       _i_hlGetOutputResolutionRect
 2106:0538       _i_hlGetOutputResolutionSize
 2106:062D idle  _i_hlGetVLDelay
 4389:061F       _i_hlGPortChangeVPosition
 4389:06E4 idle  _i_hlGPortGetFieldSize
 4389:06CB       _i_hlGPortGetVDataStart
 4389:06D3       _i_hlGPortSetDataEnableOffset
 4389:065A       _i_hlGportUpdateOnDportVSync
 4389:04A0       _i_hlGraphicCaptureEnable
 4389:0643       _i_hlGraphicChangedScaleMode
 4389:04F9 idle  _i_hlGraphicDualRevSetting
 4389:0466       _i_hlGraphicGetHalfSampleMode
 4389:0357       _i_hlGraphicInitialize
 4389:0425       _i_hlGraphicMemoryWasReconfigured
 4389:0439       _i_hlGraphicSetBlackDetectLevel
 4389:0596       _i_hlGraphicSetChannelMode
 4389:0473       _i_hlGraphicSetFrameBufferMode
 4389:0536       _i_hlGraphicUpdateLineAB
 2106:059F       _i_hlHlayerDataGet
 2106:05A5       _i_hlHlayerTempDataGet
 27FB:0FC9       _i_hlInitOutputDisplay
 2106:1309 idle  _i_hlIsHperInvalid
 2106:1385       _i_hlIsModeSupported
 4581:07CB       _i_hlOsdGetOsdConfig
 2106:12A5       _i_hlRecalculateFramelockValues
 25F7:05F3 idle  _i_hlScalerGetDataHeight
 25F7:00D5 idle  _i_hlScalerGetNLFlags
 25F7:00D9 idle  _i_hlScalerGetNLVStretch
 25F7:024C idle  _i_hlScalerGetScaleSource
 25F7:0539       _i_hlScalerGetZoomMinInputSize
 25F7:0587       _i_hlScalerResetCallback
 25F7:0592       _i_hlScalerSetOverlap
 40C3:059D idle  _i_hlSerialGetOutBuffCharCount
 2106:13E4 idle  _i_hlSetDefaultDCLK
 2106:1432       _i_hlSetLastDCLK
 2106:13AB       _i_hlSetModeData
 2106:05AB       _i_hlSetupOutputDisplay
 4281:0570       _i_hlVideoChangedScaleMode
 4281:055C       _i_hlVideoMemoryWasReconfigured
 4281:04C3       _i_hlVPortChangeVPosition
 4281:05A0 idle  _i_hlVPortGetFieldSize
 4281:0587       _i_hlVPortGetVDataStart
 4281:058F       _i_hlVPortSetDataEnableOffset
 4281:04E7       _i_hlVportUpdateOnDportVSync
 0460:017D idle  _i_IntCtrlEnableInterruptNesting
 0ADA:000E       _i_OutputScalerGetDataMgrNode
 1D7D:0004       _i_pwCalculateCRC16
 1D7D:001C       _i_pwCalculateCRC16Continuation
 2AA2:0258 idle  _i_pwDpmsTask
 2347:1B5D idle  _i_pwHostIsSuspended
 2347:1ACC idle  _i_pwHostSuspend
 2C63:1B0C idle  _i_pwOsdClearColor
 2C63:1B1E       _i_pwOsdResumeDrawing
 2C63:1B3B       _i_pwOsdRotatedOsdPosition
 2C63:1B78       _i_pwOsdRotateOsdRectangle
 3666:0000       _i_pwSrcAutoADCCalibrate
 4C81:0010       _i_pwSrcAutoBrightContCancelAuto
 4C81:0009       _i_pwSrcAutoBrightContClearData
 35E6:001B       _i_pwSrcAutoCancelAuto
 35E6:0031       _i_pwSrcAutoComputeAutoFlags
 4B8D:000D       _i_pwSrcAutoFreqPhaseCancelAuto
 4B8D:0278       _i_pwSrcAutoFreqPhaseClearData
 4B8D:0014       _i_pwSrcAutoFreqPhaseInitialize
 35E6:000F       _i_pwSrcAutoInitialize
 4C81:0017       _i_pwSrcAutoOptimizeBrightnessAndContrast
 4B8D:02FF       _i_pwSrcAutoOptimizeFrequency
 4B8D:02D5       _i_pwSrcAutoOptimizePhaseGPort
 4B4F:000F       _i_pwSrcAutoOptimizePosition
 4B4F:0001       _i_pwSrcAutoPositionCancelAuto
 4B4F:0008       _i_pwSrcAutoPositionClearData
 05C3:17F1       _i_pwSrcChannelSearch
 3A6E:09EF idle  _i_pwSrcDetCancelDetection
 3A6E:08A7       _i_pwSrcDetCheckOutOfRange
 3A6E:09FA       _i_pwSrcDetectionGetAlternate
 3A6E:0AF5       _i_pwSrcDetGetModeData
 3A6E:0006       _i_pwSrcDetInitialize
 3A6E:0978       _i_pwSrcDetMonitor
 3A6E:0015       _i_pwSrcDetPort
 3A6E:0BBE       _i_pwSrcDetSetPixelMode
 3A6E:0954       _i_pwSrcDetSpecificMode
 3BB5:1370       _i_pwSrcDisplayChange
 3BB5:0F5A       _i_pwSrcDisplayClearBitmap
 3BB5:1141       _i_pwSrcDisplayClearSource
 3BB5:0540       _i_pwSrcDisplayGetOp
 3BB5:05F1       _i_pwSrcDisplayGetOpWindow
 3BB5:1349       _i_pwSrcDisplayInhibit
 3BB5:0000       _i_pwSrcDisplayInitialize
 3BB5:0815       _i_pwSrcDisplayIsOpAvailWindow
 3BB5:0A4B       _i_pwSrcDisplayOpDescriptor
 3BB5:08AC       _i_pwSrcDisplayOpDescriptorWindow
 3BB5:0AC9       _i_pwSrcDisplayScaleWindow
 3BB5:00C8       _i_pwSrcDisplaySetOp
 3BB5:01DF       _i_pwSrcDisplaySetOpWindow
 3BB5:1224       _i_pwSrcDisplaySetupForAutoX
 3BB5:0DF9       _i_pwSrcDisplayShowBitmap
 3BB5:0F83       _i_pwSrcDisplayShowSource
 3BB5:1305       _i_pwSrcDisplayWindowDisplayable
 3BB5:13F5       _i_pwSrcDisplayWindowMgrRefresh
 05C3:178D       _i_pwSrcForceResync
 05C3:181B       _i_pwSrcGetSrc
 05C3:1864       _i_pwSrcGetWindow
 34F1:0423 idle  _i_pwSrcInputCancelRoute
 34F1:069D       _i_pwSrcInputDriverService
 34F1:065D       _i_pwSrcInputDriverServiceAllDevices
 34F1:045B idle  _i_pwSrcInputGetDevice
 34F1:043E idle  _i_pwSrcInputGetLastDeviceIndex
 34F1:009C       _i_pwSrcInputGetNextSrc
 34F1:03E2 idle  _i_pwSrcInputGetPortRoute
 34F1:00B4       _i_pwSrcInputGetPreviousSrc
 34F1:0401       _i_pwSrcInputGetSource
 34F1:0096       _i_pwSrcInputGetSourceCount
 34F1:03AB       _i_pwSrcInputGetSourceRoute
 34F1:000C       _i_pwSrcInputInitialize
 34F1:0480 idle  _i_pwSrcInputIsDeviceInActiveRoute
 34F1:054D       _i_pwSrcInputIsDriverServiceAvail
 34F1:08B7       _i_pwSrcInputPortIndex
 34F1:00D1       _i_pwSrcInputRouteSrc
 34F1:01C3       _i_pwSrcInputRouteSrcMonitor
 34F1:08CF       _i_pwSrcInputSearchDeviceList
 34F1:036C       _i_pwSrcInputUnRouteSrc
 35E6:0099       _i_pwSrcSettingAutoSetup
 376D:0F2B       _i_pwSrcSettingBroadcastSettings
 376D:0EE7       _i_pwSrcSettingClearSetting
 376D:1233       _i_pwSrcSettingGetDefaultBrightness
 376D:127C       _i_pwSrcSettingGetDefaultContrast
 376D:0561       _i_pwSrcSettingGetOp
 376D:0002       _i_pwSrcSettingInitialize
 376D:09E3       _i_pwSrcSettingIsOpAvail
 376D:0F45       _i_pwSrcSettingOpDescriptor
 376D:1152       _i_pwSrcSettingRestoreOriginalSettings
 376D:0098       _i_pwSrcSettingSetOp
 376D:0B02       _i_pwSrcSettingSetup
 376D:10F3       _i_pwSrcSettingUpdateFactoryDefaults
 376D:11D7       _i_pwSrcSettingUpdateOriginalSettings
 44CD:0116       _i_pwSrcSyncMonitorDisable
 44CD:01C5 idle  _i_pwSrcSyncMonitorDisableAll
 44CD:001A       _i_pwSrcSyncMonitorEnable
 44CD:0004       _i_pwSrcSyncMonitorInitialize
 05C3:4426       _i_pwSrcTask
 3D81:001E       _i_pwSrcTestDisplayBitmap
 3D81:0005       _i_pwSrcTestDisplayPattern
 3D81:00E2       _i_pwSrcTestDraw
 3D81:0047       _i_pwSrcTestGetParameters
 3E84:0E2D       _i_pwSrcTVChannelSearchAdvance
 3E84:083F       _i_pwSrcTVGetOp
 3E84:0993       _i_pwSrcTVGetOpWindow
 3E84:000F       _i_pwSrcTVInitialize
 3E84:0B95       _i_pwSrcTVIsOpAvail
 3E84:0C35       _i_pwSrcTVOpDescriptor
 3E84:0CE4       _i_pwSrcTVOpDescriptorWindow
 3E84:00AB       _i_pwSrcTVSetOp
 3E84:03F3       _i_pwSrcTVSetOpWindow
 3E84:1D79 idle  _i_pwSrcTvUpdateRating
 3E42:03B8       _i_pwSrcUtilAutoDisable
 3E42:0291       _i_pwSrcUtilDisplayBlank
 3E42:0257       _i_pwSrcUtilEnableCapture
 3E42:040F       _i_pwSrcUtilGetAutoDisable
 3E42:042B       _i_pwSrcUtilGetAutoDisables
 3E42:02BF       _i_pwSrcUtilGetNextSrc
 3E42:0323       _i_pwSrcUtilGetPrevSrc
 3E42:0387       _i_pwSrcUtilGetStatus
 3E42:000E       _i_pwSrcUtilIntialize
 3E42:02A8       _i_pwSrcUtilOsdBlank
 3E42:002E       _i_pwSrcUtilSendSourceBasedEvent
 3E42:0120       _i_pwSrcUtilSendWindowBasedEvent
 3E42:020B       _i_pwSrcUtilSrcCtlReadLock
 3E42:0226       _i_pwSrcUtilSrcCtlReadUnlock
 3E42:0233       _i_pwSrcUtilSrcCtlWriteLock
 3E42:024E       _i_pwSrcUtilSrcCtlWriteUnlock
 318B:0AE9       _i_uiCtlMenuSuspendDrawing
 0000:049D       _labs
 42DC:0006 idle  _LimitXTo
 04A1:02E9       _lintoseg
 049D:0004       _main
 04A1:004D       _MemoryAssign
 449A:0308       _MyDelay
 3E84:177E idle  _MySetupDefaultDisplayMode
 4DE0:113C       _m_b60Hz
 4DE0:0416 idle  _m_bSignalCallingTask
 4DE0:1290       _m_bSystemPowerOff
 4DE0:12FA       _m_bTimerOnFlag
 4DE0:12F8       _m_cPannelType
 4DE0:12F9 idle  _m_cUserScaleMode
 5044:0000 idle  _m_cVideoFormatSTD
 4DE0:03F0 idle  _m_dwCurrentChannel
 4DE0:10F6       _m_HSINPOL_ACTIVE
 4DE0:0424       _m_InputClipWindow
 4DE0:0442       _m_nHorzLinearRegion
 4DE0:043C       _m_nHorzStretch
 4DE0:0444       _m_nVertLinearRegion
 4DE0:043E       _m_nVertStretch
 4DE0:1A5E idle  _m_nXOffset
 4DE0:1A60 idle  _m_nYOffset
 4DE0:0434       _m_OriginalScaleModeInputWindow
 4DE0:042C       _m_OutputDispWindow
 4DE0:1274 idle  _m_TunerVideoAudioStandard
 5066:0000 idle  _m_VolumeControlTable2
 4DE0:1A26 idle  _m_wBytesToWrite
 5044:0006 idle  _m_wCableChDivideRF
 4DE0:0440       _m_wNLFlags
 4DE0:1A24 idle  _m_wOutThreshold
 4DE0:01DF       _m_wPipLeftPos
 4DE0:061C       _o2semid
 4DE0:063A       _o3semid
 4D39:0089 idle  _OutputByteBlock
 4D39:00BF       _OutputByteBlocksSkip
 4D39:020B       _OutputRleByteBlockRLE
 4D39:0427       _OutputRleWordBlockRLE
 4D39:01CD       _OutputWordBlock
 3E84:1E84 idle  _Picture_UnBlack
 1B07:04DA idle  _PoweronHardware
 2347:0D99 idle  _ProcessDiagReadMessage
 2347:14F4 idle  _ProcessDiagWriteMessage
 2347:1A48 idle  _ProcessDMReadMessage
 2347:1A9C idle  _ProcessDMWriteMessage
 2347:08E0 idle  _ProcessEventMessage
 2347:0C26 idle  _ProcessForceModeMessage
 2347:1BD3 idle  _ProcessOemMessage
 2347:08FE idle  _ProcessOperationMessage
 1D84:218D idle  _ProcessPerfectPicture
 2347:1C02 idle  _ProcessPWCmdMessage
 2347:07D4 idle  _ProcessSystemMessage
 2347:0BC9 idle  _ProcessUIStateMessage
 2347:0AB1 idle  _ProcessVariableMessage
 1781:16BA       _PW1230_50_60_Init
 2347:1D51 idle  _pwCmdExecute
 2AA2:0612 idle  _pwDPMSEnable
 2AA2:06A0 idle  _pwDPMSEnableGet
 2AA2:05C3       _pwDPMSExecuteAction
 2AA2:06BF idle  _pwDPMSForcePowerState
 2AA2:06B1       _pwDPMSGetCurrentState
 2AA2:0A3C idle  _pwDPMSGetLampParms
 2AA2:0B0A idle  _pwDPMSGetLampRange
 2AA2:0791 idle  _pwDPMSGetOnTime
 2AA2:06E9 idle  _pwDPMSGetOnTimeRange
 2AA2:0463       _pwDPMSGetOp
 2AA2:038C       _pwDPMSGetOpDescriptor
 2AA2:000A       _pwDPMSInitialize
 2AA2:030B       _pwDPMSIsOpAvail
 2AA2:05E9 idle  _pwDPMSPause
 2AA2:05FF idle  _pwDPMSPauseGet
 2AA2:09B6 idle  _pwDPMSResetOnTime
 2AA2:0A8A idle  _pwDPMSSetLampParms
 2AA2:0846 idle  _pwDPMSSetOnTime
 2AA2:0524       _pwDPMSSetOp
 2AA2:024D       _pwDpmsStartTask
 2AA2:0B50       _pwDPMSUserInput
 2347:0695       _pwHostLogError
 2347:05E0       _pwHostLogTrace
 2347:0750 idle  _pwHostSendOemMessage
 2347:04D8       _pwHostStart
 2347:0006 idle  _pwHostTask
 2E7D:0012       _pwInputInitialize
 2E7D:00BA       _pwInputRegisterCallback
 2E7D:00A6       _pwInputSendSignal
 2E7D:00F5       _pwInputTaskStart
 1FCE:0019       _pwIspCoreArrayBounds
 1FCE:0015       _pwIspCoreBreakpoint
 1FCE:000F       _pwIspCoreDivideError
 1FCE:001D       _pwIspCoreEscOpcode
 1FCE:0017       _pwIspCoreIntoOverflow
 1FCE:0013       _pwIspCoreNMI
 1FCE:0011       _pwIspCoreSingleStep
 1FCE:001B       _pwIspCoreUnusedOpcode
 1FCF:046B       _pwMiscAwakeDisplayVSync
 1FCF:083B       _pwMiscExecuteAction
 1FCF:04A8       _pwMiscGetOp
 1FCF:048C       _pwMiscGetOpDescriptor
 1FCF:038A idle  _pwMiscGetParm
 1FCF:00F9 idle  _pwMiscGetRange
 1FCF:0018       _pwMiscInitialize
 1FCF:0292       _pwMiscIsOpAvail
 1FCF:0045       _pwMiscSaveAndRestoreInit
 1FCF:066B       _pwMiscSetOp
 1FCF:03DB idle  _pwMiscSetParm
 1FCF:0448       _pwMiscWaitForDisplayVSync
 1D84:18C6       _pwOemDataMgrInitialize
 1D84:18CB       _pwOemDisplaySetPower
 1D84:0171       _pwOemDPMSStateChange
 1D84:1130       _pwOEMExecuteAction
 1D84:189D       _pwOemGetCustomString
 1D84:17A4 idle  _pwOEMGetGuiData
 1D84:03B2       _pwOEMGetOp
 1D84:0008       _pwOemInitialize
 1D84:18CF idle  _pwOemIsNV320
 1D84:0172       _pwOEMIsOpAvail
 1D84:1897       _pwOEMMatchEvent
 1D84:1896       _pwOEMNewSourceFound
 1D84:14C8       _pwOEMOpDescriptor
 1D84:18C5       _pwOemOsdWindowEnable
 1D84:0159       _pwOemReceiveHostMessage
 1D84:1817 idle  _pwOEMSetGuiData
 1D84:0932       _pwOEMSetOp
 1D84:18CA       _pwOemSpecialProcessing
 2E97:095F idle  _pwOpCroppingMode
 2E97:0000       _pwOperationsInitialize
 2E97:08DB       _pwOpExecuteAction
 2E97:069F       _pwOpExecuteGetCropRange
 2E97:0855 idle  _pwOpExecuteGetLongRange
 2E97:081F       _pwOpExecuteGetRange
 2E97:02A2       _pwOpExecuteGetValue
 2E97:0463       _pwOpExecuteIncrement
 2E97:03BF       _pwOpExecuteIncrementCrop
 2E97:0066       _pwOpExecuteIsOpAvail
 2E97:00DE       _pwOpExecuteSetValue
 2E97:0980       _pwOpGetDescriptor
 2E97:0037 idle  _pwOpGetUIIncrement
 483F:002A       _pwOpPrintf
 483F:0000       _pwOpPrintfIsStringFormatted
 2C63:1A38       _pwOsdBackgroundIsSolid
 2C63:028B       _pwOsdBlankCapture
 2C63:0789 idle  _pwOsdBlockOperationLock
 2C63:079A idle  _pwOsdBlockOperationUnlock
 2C63:1AEE       _pwOsdClearColorOverride
 2C63:08F8       _pwOsdClearRectangle
 2C63:18C4 idle  _pwOsdClearWindow
 2C63:0BC0       _pwOsdDrawBitmap
 2C63:0D57       _pwOsdDrawBlitItem
 2C63:0CD5       _pwOsdDrawBlitmap
 2C63:0E23 idle  _pwOsdDrawChar
 2C63:0936       _pwOsdDrawHollowRect
 2C63:1608       _pwOsdDrawNumber
 2C63:07DC       _pwOsdDrawRectangle
 2C63:0E66 idle  _pwOsdDrawString
 2C63:12E2       _pwOsdDrawText
 2C63:1342       _pwOsdDrawText2
 2C63:19C6       _pwOsdEnableSolidBackground
 4948:0289       _pwOSDExecuteAction
 2C63:1869       _pwOsdFillWindow
 2C63:07C5 idle  _pwOsdGetGraphicOffset
 2C63:0701       _pwOsdGetGridWindow
 4948:0136       _pwOSDGetOp
 4948:0001       _pwOSDGetOpDescriptor
 2C63:1A93       _pwOsdGetOrientation
 2C63:0514       _pwOsdGetPosDiscrete
 2C63:04EC       _pwOsdGetPosHorz
 2C63:0500       _pwOsdGetPosVert
 2C63:11EE       _pwOsdGetStringSize
 2C63:00E7       _pwOsdGetTransparentColor
 2C63:062F       _pwOsdGetUserPosition
 2C63:04BE       _pwOsdGetWindowPos
 2C63:1AF5       _pwOsdHollowForceModeEnable
 2C63:0008       _pwOsdInitialize
 2C63:0247       _pwOsdIsCaptureBlanked
 4948:00D7       _pwOSDIsOpAvail
 2C63:18D0       _pwOsdIsPointValid
 2C63:18F9 idle  _pwOsdIsRectangleValid
 2C63:00DD idle  _pwOsdIsTransparentModeEnabled
 2C63:039F       _pwOsdIsWindowEnabled
 2C63:198B       _pwOsdLowColorOverlayFunctionEnable
 2C63:020B       _pwOsdRestoreWindow
 2C63:1A41 idle  _pwOsdRotateWindowPos
 2C63:0256       _pwOsdSetBlankingColor
 2C63:0DFB idle  _pwOsdSetCharFont
 2C63:1AD1       _pwOsdSetColorOverride
 2C63:07A5       _pwOsdSetGraphicOffset
 2C63:0169       _pwOsdSetMode
 4948:0197       _pwOSDSetOp
 2C63:1A9D       _pwOsdSetOrientation
 2C63:1969       _pwOsdSetOverlayColors
 2C63:0566       _pwOsdSetPosDiscrete
 2C63:0528       _pwOsdSetPosHorz
 2C63:0547       _pwOsdSetPosVert
 2C63:03A9       _pwOsdSetWindowPos
 2C63:01EB       _pwOsdSuspendDrawing
 2C63:00C6 idle  _pwOsdTransparentModeEnable
 2C63:02EB       _pwOsdUnblankCapture
 2C63:0355       _pwOsdWindowEnable
 0A19:00DB       _pwPeriodicCreate
 0A19:0197 idle  _pwPeriodicDelete
 0A19:0000       _pwPeriodicInitialize
 0A19:02BE       _pwPeriodicRestart
 0A19:01CC idle  _pwPeriodicStart
 0A19:00B2       _pwPeriodicStartTask
 0A19:03D6 idle  _pwPeriodicStop
 0A6A:0339       _pwRosAreInterruptsEnabled
 0A6A:04E3       _pwRosCalledFromInterrupt
 0A6A:01BC       _pwRosConvertMsToSystemTicks
 0A6A:00E2       _pwRosCreateSemaphore
 0A6A:0061       _pwRosCreateTimer
 0A6A:0105 idle  _pwRosDeleteSemaphore
 0A6A:009C idle  _pwRosDeleteTimer
 0A6A:02EB       _pwRosEventFlagCreate
 0A6A:034C       _pwRosEventFlagSignal
 0A6A:0306       _pwRosEventFlagWait
 0A6A:025E       _pwRosGetCurrentTaskId
 0A6A:0287       _pwRosGetCurrentTaskPriority
 0A6A:0203       _pwRosGetSystemClock
 0A6A:026E       _pwRosGetTaskId
 0A6A:02A3       _pwRosGetTaskPriority
 0A6A:0336 idle  _pwRosGetTaskStack
 0A6A:000B       _pwRosInitialize
 0A6A:000C       _pwRosInSysInit
 0A6A:0017 idle  _pwRosIsInSysInit
 0A6A:02CF       _pwRosIsTaskSuspended
 0A6A:04DD       _pwRosReadSystemTicks
 0A6A:00D4       _pwRosReadTimer
 0A6A:0160       _pwRosReleaseSemaphore
 0A6A:011A       _pwRosReserveSemaphore
 0A6A:001D       _pwRosSendMessage
 0A6A:0041       _pwRosSendMessageWait
 0A6A:01E7       _pwRosSetInterruptVector
 0A6A:02BC       _pwRosSetTaskPriority
 0A6A:01A7       _pwRosSignalSemaphore
 0A6A:00AA       _pwRosStartTimer
 0A6A:00C0       _pwRosStopTimer
 0A6A:01FD       _pwRosSystemTick
 0A6A:03DC idle  _pwRosTaskCreate
 0A6A:0419       _pwRosTaskCreateComplete
 0A6A:0227       _pwRosTaskDelay
 0A6A:0370       _pwRosTaskResume
 0A6A:038C       _pwRosTaskSignal
 0A6A:03AC       _pwRosTaskSignalWait
 0A6A:0362       _pwRosTaskSuspend
 0A6A:04CF       _pwRosTaskTrigger
 0A6A:037E       _pwRosTaskWake
 0A6A:0175       _pwRosWaitSemaphore
 05C3:15F2       _pwSrcChangeState
 3A6E:0D82       _pwSrcDetectionCheckAlternateResolution
 05C3:1762 idle  _pwSrcEnableAll
 05C3:16CA idle  _pwSrcEnableSource
 05C3:06F2       _pwSrcExecuteAction
 05C3:1310       _pwSrcForceMode
 05C3:1338 idle  _pwSrcForceModeCancel
 05C3:14CE idle  _pwSrcGetModeInfo
 05C3:1462       _pwSrcGetModeSource
 05C3:1402 idle  _pwSrcGetModeWindow
 05C3:0708       _pwSrcGetOp
 05C3:0D5C       _pwSrcGetOpDescriptor
 05C3:153C       _pwSrcGetSourceStatus
 05C3:15FD idle  _pwSrcGetSourceStatusSpecific
 05C3:10AC       _pwSrcInitialize
 05C3:0BAF       _pwSrcIsOpAvail
 05C3:135A idle  _pwSrcSelectMode
 05C3:0004       _pwSrcSetOp
 05C3:1305       _pwSrcStart
 05C3:1679       _pwSrcSuspend
 05C3:16B4       _pwSrcSuspended
 3D81:01C7       _pwSrcTestGetNumberOfTestPatterns
 1FCF:000F idle  _pwVersion
 1781:11D4 idle  _Read1230Reg
 4767:0001       _RenderBlitMap
 4767:0087       _RenderBlitMapMenuItems
 4D85:024F idle  _RepeatValid
 2347:1EDB idle  _ResetBuffer
 42DC:0029       _ResolutionsAreValid
 4DE0:0622       _rxsemid
 1D84:1999       _SavePictureUserMode
 5066:0067 idle  _SCART_INPUT_PRESCALE_AV
 5066:0065 idle  _SCART_INPUT_PRESCALE_DEFAULT
 5066:0069 idle  _SCART_INPUT_PRESCALE_PC
 5066:0066 idle  _SCART_INPUT_PRESCALE_TV
 5066:0068 idle  _SCART_INPUT_PRESCALE_YPbPr
 4DE0:0624       _scsemid
 4DE0:0616       _sctlid
 04A1:02CF       _segtolin
 2347:1EE1 idle  _SendBuffer
 2347:21A9 idle  _SendBytes
 2347:1FB7 idle  _SendMessage
 449A:0095       _SendMessageToDevice
 2347:20B3 idle  _SendResponse
 1D84:1FC4 idle  _SetBlueScreen1230
 1B07:0B0A       _SetChannel
 3E84:17AB       _SetCurrentChannel
 3E84:17BD       _SetCurrentDivisor
 4D39:0001       _SetDataTransferInfo
 3E84:1F53 idle  _SetFirstTimeChangeBand
 1C48:0CFE idle  _SetMuteState
 1D84:18E1       _SetPictureUserMode
 1D84:207B idle  _SetPW1230ToCinameScalerMode
 1D84:212B idle  _SetPW1230ToNormalScalerMode
 1D84:20D3 idle  _SetPW1230ToSubtitleScalerMode
 42DC:00D8       _SetScaleParamsPct
 42DC:03FE       _SetScaleParamsRect
 1B07:0EE8       _SetStandardAndChannel
 1B07:0E21 idle  _SetTunerAFCStandard
 1B07:0D4F       _SetTunerAudioStandard
 3E84:1836 idle  _SetTunerDivisorMaxMin
 1B07:0E8A idle  _SetTunerHz50_60
 14CD:26F7       _SetTunerVideoFormat
 1B07:0C23       _SetTunerVideoStandard
 1C48:0CAA idle  _SetVolume
 0DB8:467B       _Set_Capture_Enable
 449A:013C       _SoftReset
 1A02:063A idle  _SrvSetupDisplayMode
 4FA7:0000 idle  _STACKSEG@
 4DE0:1292 idle  _Start_Always_Power_Off_Timer_Flag
 0000:04C5       _strncmp
 04D5:0008       _sysSystemInitialize
 29DA:0006 idle  _TempDelay
 46E0:0008 idle  _TestLEDops
 1D84:1AFE       _TimerOneMin
 1D84:1ABB idle  _TimerOneSec
 4DE0:01C7 idle  _Timer_No_Signal
 4DE0:0620       _txsemid
 33CB:0010       _uiAddToModifiedOpsList
 4975:002D       _uiBhvBoundOp
 4975:0045       _uiBhvBoundOpType
 4975:0039       _uiBhvBoundTarget
 4975:00A9       _uiBhvBoundValue
 2566:00E6       _uiBhvClearSystemVariable
 2566:005B       _uiBhvClearUserVariable
 33FA:01D4       _uiBhvConditionMgrGetCondition
 33FA:0002       _uiBhvConditionMgrSetupState
 33FA:00B5       _uiBhvConditionMgrUpdateConditions
 33FA:0114       _uiBhvConditionMgrUpdateState
 4975:01F7       _uiBhvControlItemID
 4975:0022 idle  _uiBhvControlType
 348F:0462       _uiBhvDynamicMgrGetBehaviorEntry
 348F:000F       _uiBhvDynamicMgrSetupState
 348F:009D       _uiBhvDynamicMgrUpdateState
 2566:0527       _uiBhvEnableConditionCache
 2566:0267       _uiBhvEvaluateCondition
 2F72:01B8       _uiBhvGetActiveMenu
 2566:0436       _uiBhvGetAlternateRendering
 2566:010E       _uiBhvGetBehaveInfo
 2F72:02F0       _uiBhvGetFirstVisibleMenu
 2566:036A       _uiBhvGetGrayCondition
 2566:039D       _uiBhvGetHideCondition
 2F72:0672       _uiBhvGetItemGrayFlag
 2F72:0647       _uiBhvGetItemInvertFlag
 2566:0403       _uiBhvGetManualChildMenu
 2F72:0309       _uiBhvGetNextVisibleMenu
 4975:0106       _uiBhvGetRectangle
 2566:03D0       _uiBhvGetSelectCondition
 2566:0279       _uiBhvGetSubMenu
 2566:02A1       _uiBhvGetSubMenuParent
 2566:00CE       _uiBhvGetSystemVariable
 2566:003F       _uiBhvGetUserVariable
 4975:0203       _uiBhvIsContainerMenu
 2F72:0686       _uiBhvIsMenuItemGray
 2F72:06B8       _uiBhvIsMenuItemVisible
 2F72:01AF       _uiBhvIsMenuState
 2F72:06F4       _uiBhvMenuAreSubItemsPresent
 2F72:082D       _uiBhvMenuGetChanged
 2F72:029C       _uiBhvMenuGetChild
 2F72:0837       _uiBhvMenuGetInfo
 2F72:0393       _uiBhvMenuGetInfoByID
 2F72:0251       _uiBhvMenuGetParent
 2F72:0728       _uiBhvMenuGetWrapEnable
 2F72:05C5       _uiBhvMenuGridRowItems
 4975:000A       _uiBhvMenuID
 2F72:04DC       _uiBhvMenuIsVisible
 4975:0016       _uiBhvMenuItem
 2F72:0746       _uiBhvMenuNextItem
 2F72:07B2       _uiBhvMenuPrevItem
 2F72:03FA       _uiBhvMenuSetActiveItem
 2F72:0827       _uiBhvMenuSetChanged
 2F72:000A       _uiBhvMenuSetupState
 2F72:04BF       _uiBhvMenuSetVisibility
 2F72:04FB       _uiBhvMenuShowChild
 2F72:08E0       _uiBhvMenuUpdateChildPositions
 33FA:043D       _uiBhvResetOffsetPaint
 2F72:01EB       _uiBhvSetActiveMenu
 2F72:065B       _uiBhvSetItemGrayFlag
 2F72:0630       _uiBhvSetItemInvertFlag
 2566:008B       _uiBhvSetSystemVariable
 33FA:0213       _uiBhvSetupOffsetPaint
 2566:0001       _uiBhvSetUserVariable
 2566:00FA       _uiBhvToggleSystemVariable
 2566:0073       _uiBhvToggleUserVariable
 3140:01F4       _uiCheckClipping
 33CB:0009       _uiClearModifiedOpsList
 3375:027C       _uiClearOSD
 3140:015C       _uiClipControlRectangle
 3140:0344 idle  _uiCtlApplyCropping
 4B37:000F       _uiCtlBorder
 4A71:000A       _uiCtlButton
 4A9E:0003       _uiCtlDynamic
 4A00:0009       _uiCtlGauge
 318B:0008       _uiCtlMenu
 318B:09CB       _uiCtlMenuRenderContent
 318B:0A5D idle  _uiCtlMenuSelectItem
 4A4F:0005       _uiCtlNumber
 4A86:000F       _uiCtlText
 3140:0234       _uiCtlUpdateDisplay
 3316:000D       _uiDrawDrawList
 3316:02C8       _uiDrawItem
 2F47:0072       _uiEventMatchEnterExitFirst
 2F47:00B1       _uiEventMatchEnterExitNext
 2F47:000A       _uiEventMatchFirst
 2F47:003A       _uiEventMatchNext
 3140:0004       _uiExecuteAllControls
 33CB:0095       _uiExecuteEnterExitOperations
 318B:01BF       _uiExecuteMenuActiveItem
 318B:052C       _uiExecuteMenuNavigate
 318B:08CA       _uiExecuteMenuSelectList
 3316:02AE       _uiGetBackgroundColor
 4998:0509       _uiGetControlByID
 050C:0446       _uiGetCurrentState
 4998:03E3       _uiGetFirstBoundControl
 4998:0004 idle  _uiGetFirstControl
 4998:0030       _uiGetFirstMenu
 4998:00CF       _uiGetFirstMenuItem
 4998:031B       _uiGetFirstMenuItemBound
 4998:047B       _uiGetFirstTopLevelControl
 4998:0404       _uiGetNextBoundControl
 4998:001D idle  _uiGetNextControl
 4998:0051       _uiGetNextMenu
 4998:0292       _uiGetNextMenuItem
 4998:0372       _uiGetNextMenuItemBound
 4998:049C       _uiGetNextTopLevelControl
 050C:04E0       _uiGetNumLanguages
 050C:042B       _uiGetStatePtr
 050C:050D       _uiGetUpdatedState
 4B4E:0010       _uiHidePaneByIndex
 050C:0147       _UIManagerInit
 33CB:005B       _uiModifiedOpListIsEmpty
 33CB:006A       _uiOpIsInModifedOpsList
 3375:0094       _uiOsdChangePosAndSize
 3375:003C       _uiOsdGetHorzStepSize
 3375:0068       _uiOsdGetVertStepSize
 3375:01D8       _uiOsdUpdatePosition
 3375:0005       _uiOsdZeroPosition
 050C:044A       _uiRedrawCurrentState
 050C:00E9       _uiSendOperationUpdate
 050C:00C3       _uiSendStateChangeMessage
 050C:0122       _uiSendUpdateAll
 050C:000E       _uiSendUserMessage
 050C:0034       _uiSendUserMessageWait
 050C:005A       _uiSendUserMessageWithData
 050C:008C       _uiSendUserMessageWithDataWait
 050C:010F       _uiSendVariableUpdate
 3316:02B6       _uiSetBackgroundColor
 3316:0259       _uiSetDefaultOsdPalette
 3316:026E       _uiSetDefaultOverlayFunctions
 3140:014A       _uiSetNewStateForClipping
 050C:03DB       _uiSetNextState
 050C:03F3       _uiSetUserVariable
 4B4E:000F       _uiShowPaneByIndex
 33CB:011D       _uiStartStopTimer
 050C:01CF       _UIStateManager
 4DE0:0614       _uistid
 050C:0511       _UITimerProc
 050C:0541       _uiTimerProcess
 4DE0:061A       _uitmid
 3316:03C4       _uiUndrawItem
 3140:00A5       _uiUpdateControls
 050C:0502       _uiUpdateStateChange
 4DE0:0634 idle  _ursemid
 4DE0:0636 idle  _ussemid
 04A1:0090       _uumemget
 2347:1E5C idle  _ValidHeader
 14CD:10CE idle  _VideoFormatChanged
 1D84:1C76       _VPC3230FPAccess
 4DE0:062E       _vpsemid
 1781:1213 idle  _Write1230Reg
 1B07:0AB8       _WriteTunerDiv
 4DE0:0022 idle  __8086
 0000:0380 idle  __abort
 0000:000C idle  __AHSHIFT
 4DE0:15E8       __atexitcnt
 4DE0:15EA       __atexittbl
 4767:013F idle  __BlastBits
 4DE0:0640 idle  __bss_start
 0000:037F       __checknull
 0000:00AE       __cleanup
 0000:01AC       __CopyFarData
 4DE0:0508       __ctype
 4DE0:0000 idle  __data_start
 0000:0374       __DefaultRtlError
 0000:01A4       __ExceptInit
 4DE0:0020 idle  __Exception_list
 0000:0181 idle  __exit
 4DE0:0080 idle  __exitbuf
 4DE0:0084 idle  __exitfopen
 4DE0:0088 idle  __exitopen
 5117:0000       __farbss_end
 5117:0000       __farbss_start
 5116:0000 idle  __farconst_end
 4FB9:0000 idle  __farconst_start
 4FB8:0000       __fardata_end
 4FB8:0000       __fardata_start
 5118:0000 idle  __farheap_end
 5118:0000       __farheap_start
 0000:038D idle  __fpure_error_
 0000:01A5 idle  __GetPolymorphicDTC(void*,unsigned int)
 0000:01A8 idle  __GetPolymorphicDTCfar(void*,unsigned int)
 0000:01FC       __InitFarBss
 0000:038D idle  __npure_error_
 4DE0:1C60 idle  __nvram_start
 0000:04FE       __ParadigmTerminate
 0000:000C idle  __PCFAST
 0000:1000       __PCINCR
 0000:000F       __PCMASK
 0000:0000 idle  __PCMODE
 0000:0004       __PCSHIFT
 4DDF:0000 idle  __ramfunction_end
 4DDF:0000 idle  __ramfunction_start
 4DE0:060A idle  __RealCvtVector
 0000:0193 idle  __RefDestructorCount()
 0000:0199 idle  __RefExceptionList()
 4DDC:0000 idle  __romdata_end
 4DDC:0000 idle  __romdata_start
 4DDD:0000       __romfardata_end
 4DDD:0000       __romfardata_start
 4DDE:0000 idle  __romfunction_end
 4DDE:0000 idle  __romfunction_start
 4DE0:060A idle  __ScanTodVector
 4FA7:0000 idle  __stack_bottom
 4FA7:0000 idle  __stack_segment
 4FA7:0100 idle  __stack_top
 0000:0000       __startup
 4DE0:1C60       __staticdata_end
 4DE0:0640       __stklen
 0000:0375       __terminate
 4DE0:0316 idle  ___brklvl
 0000:01A0 idle  ___ExitExceptBlocks
 4DE0:0318 idle  ___heapbase
 0000:01A3 idle  ___InitExceptBlock
 0000:019F idle  ___InitExceptBlocks


  Address         Publics by Value

 0000:0000       __startup
 0000:0000 idle  __PCMODE
 0000:0004       __PCSHIFT
 0000:000C idle  __AHSHIFT
 0000:000C idle  __PCFAST
 0000:000F       __PCMASK
 0000:00AE       __cleanup
 0000:0172       _exit
 0000:0181 idle  __exit
 0000:0193 idle  __RefDestructorCount()
 0000:0199 idle  __RefExceptionList()
 0000:019F idle  ___InitExceptBlocks
 0000:01A0 idle  ___ExitExceptBlocks
 0000:01A3 idle  ___InitExceptBlock
 0000:01A4       __ExceptInit
 0000:01A5 idle  __GetPolymorphicDTC(void*,unsigned int)
 0000:01A8 idle  __GetPolymorphicDTCfar(void*,unsigned int)
 0000:01AC       __CopyFarData
 0000:01FC       __InitFarBss
 0000:0240 idle  N_LDIV@
 0000:0243       F_LDIV@
 0000:0243 idle  LDIV@
 0000:0247 idle  N_LUDIV@
 0000:024A       F_LUDIV@
 0000:024A idle  LUDIV@
 0000:024F idle  N_LMOD@
 0000:0252       F_LMOD@
 0000:0252 idle  LMOD@
 0000:0257 idle  N_LUMOD@
 0000:025A idle  LUMOD@
 0000:025A       F_LUMOD@
 0000:02EE       F_LXMUL@
 0000:02EE idle  LXMUL@
 0000:0305 idle  N_LXURSH@
 0000:0308       F_LXURSH@
 0000:0308 idle  LXURSH@
 0000:0326 idle  N_LXLSH@
 0000:0329       F_LXLSH@
 0000:0329 idle  LXLSH@
 0000:0347 idle  _atexit
 0000:0374       __DefaultRtlError
 0000:0375       __terminate
 0000:037F       __checknull
 0000:0380 idle  __abort
 0000:038D idle  __fpure_error_
 0000:038D idle  __npure_error_
 0000:039A idle  F_OVERFLOW@
 0000:039A idle  N_OVERFLOW@
 0000:039A idle  OVERFLOW@
 0000:03A7 idle  DGROUP@
 0000:03A9 idle  N_PSBP@
 0000:03AC idle  PSBP@
 0000:03AC       F_PSBP@
 0000:03DB idle  SCOPY@
 0000:03DB       F_SCOPY@
 0000:03F7 idle  N_LXRSH@
 0000:03FA idle  LXRSH@
 0000:03FA       F_LXRSH@
 0000:0417       _atol
 0000:048C idle  _atoi
 0000:049D       _labs
 0000:04C5       _strncmp
 0000:04FE       __ParadigmTerminate
 0000:0503 idle  N_PADA@
 0000:0506       F_PADA@
 0000:0506 idle  PADA@
 0000:054D idle  N_PSBA@
 0000:0550 idle  PSBA@
 0000:0550 idle  F_PSBA@
 0000:1000       __PCINCR
 0059:0006       _ComputeVertFrequency
 0059:001B       _ComputeHorzFrequency
 0059:0033       _ComputeVertFreqX100
 0069:0000       _AMDATP_
 0069:0004       _AMXUPT_
 0069:01B0       AASMRR
 0069:01F1       AASMCRE
 0069:0255       AASMDEL
 0069:0297       AASMRSV
 0069:0297       AASMWAT
 0069:0362       AASMRLS
 0069:0393       AASMFRE
 0069:03B3       AASMSIG
 0069:0466       AASMGET
 0069:0497       AASMTAG
 0069:04A5       AAEVRR
 0069:04E8       AAEVCRE
 0069:052C       AAEVDEL
 0069:056F       AAEVWAT
 0069:0656       AAEVSIG
 0069:0753       AAEVRD
 0069:076E       AAEVNT
 0069:077E       AAEVTAG
 0069:078C       AAMMRR
 0069:07FA       AAMHAN
 0069:0806       AAMGET
 0069:0825       AAMGEH
 0069:0855       AAMFRE
 0069:0972       AAMGSZ
 0069:09C1       AAMAU
 0069:0C37       _ajint
 0069:0C3A       _ajinx
 0069:0C3D idle  _ajitrp
 0069:0C50       _ajentr
 0069:0C8B       _ajupt
 0069:0CBA idle  _AJDATP_
 0069:0CD3 idle  _AJVERP_
 0069:0CEA idle  _ajmodl
 0069:0CF0 idle  _ajmhan
 0069:0D14       _ajmget
 0069:0D3D idle  _ajmgeh
 0069:0D69       _ajmfre
 0069:0D79       _ajmgsz
 0069:0D93 idle  _ajmau
 0069:0DA6       AMKRNL
 0069:0E0F       AMKRNX
 0069:0E7E       AACLK
 0069:0F93       AMTIMR
 0069:106D       AATMCRE
 0069:10F2       AATMDEL
 0069:113D       AMTTWR
 0069:1146       AATMWR
 0069:11D7       AMTTRD
 0069:11E9       AATMRD
 0069:1239       AATICK
 0069:124F       AATMCNV
 0069:12B9       AATMTAG
 0069:12CB idle  _AMVER_
 0069:1323 idle  AMBITP
 0069:1327 idle  AMBITN
 0069:1337       AMGDP
 0069:133D       AMGVP
 0069:1343 idle  AAVER
 0069:134B       AMUSRP
 0069:135C idle  AMHANGC
 0069:1361       AMHANG
 0069:136D       AMIHNG
 0069:138B idle  AMSHED
 0069:13BA idle  AMIDLE
 0069:1438       AMTASK
 0069:1522 idle  AAEND
 0069:1577       AMUPEM
 0069:158D       AMERR
 0069:15DB       AAFATL
 0069:1600 idle  AMHALT
 0069:1604       AAPRVR
 0069:1623       AAPRVL
 0069:164B idle  AAHOOK
 0069:169A       AMSGEV
 0069:16FC       AMCFH
 0069:170C       AATRIG
 0069:1734       AARESUM
 0069:174A       AASUSP
 0069:17BF       AASEND
 0069:190E       AAWAKC
 0069:1917       AAWAKCS
 0069:1989       AAWAIT
 0069:1992       AAWATM
 0069:19FA       AAWAKE
 0069:1A4E       AAWAPR
 0069:1A60       AASGWAT
 0069:1AFA       AASGNL
 0069:1B89       AASGRD
 0069:1B9C       AASGRES
 0069:1BBC       AATKSTS
 0069:1CA5       AATKTAG
 0069:1CEF       AATKID
 0069:1CFC       AMUTAG
 0069:1D40       AATKTCB
 0069:1D58       AAINT
 0069:1DAA       AAINX
 0069:1DE9       AABERH
 0069:1DF2       AAOVFH
 0069:1DFB       AADERH
 0069:1E54 idle  AMIRET
 0069:1E54       AMPOPF
 0069:1E64       AAITRP
 0069:1EA4       _ajtmcres
 0069:1ECE       _ajtmdel
 0069:1ED8       _ajtmwr
 0069:1EEC       _ajtmrd
 0069:1EFC       _ajtmcnv
 0069:1F0F       _ajclk
 0069:1F12       _ajtick
 0069:1F17 idle  _ajtmtag
 0069:1F31       _ajevcre
 0069:1F50       _ajevwat
 0069:1F53       _ajevsig
 0069:1F56 idle  _ajevdel
 0069:1F64 idle  _ajevrd
 0069:1F79 idle  _ajevnt
 0069:1F7C idle  _ajevtag
 0069:1F98 idle  _ajivtx
 0069:1FB2 idle  _ajivtr
 0069:1FC5       _ajivtw
 0069:1FD8 idle  _ajispm
 0069:1FEE       _ajtrig
 0069:1FFA       _ajsusp
 0069:2004       _ajresum
 0069:200E idle  _ajsendp
 0069:2012 idle  _ajsenwp
 0069:2023       _ajsend
 0069:2027       _ajsenw
 0069:2040 idle  _ajwakc
 0069:2043 idle  _ajwakcs
 0069:204D idle  _ajwait
 0069:2050       _ajwake
 0069:205A idle  _ajwapr
 0069:205D       _ajwatm
 0069:206A       _ajsgwat
 0069:2099       _ajsgnl
 0069:20BE idle  _ajsgrd
 0069:20C1 idle  _ajsgres
 0069:20CE       _ajtktag
 0069:20E8       _ajtkid
 0069:20EB       _ajtksts
 0069:20FE       _ajtktcb
 0069:2122       _ajsmcre
 0069:2141       _ajsmwat
 0069:2141       _ajsmrsv
 0069:215A       _ajsmsig
 0069:2167 idle  _ajsmget
 0069:2174       _ajsmrls
 0069:2181 idle  _ajsmfre
 0069:218E       _ajsmdel
 0069:219B idle  _ajsmtag
 0069:21B7       _ajtkcre
 0069:21CD       _ajtkpry
 0069:21DA       AMMAL
 0069:2244       AAENTR
 0069:2527 idle  AMTKPRY
 0069:2536       AATKPRY
 0069:2595       AMTKSLC
 0069:260D       AAIVTX
 0069:264C       AAIVTR
 0069:267D       AAIVTW
 0069:26A7       AAISPM
 0069:26D4       AMINRM
 0069:2708 idle  AMIRRM
 0069:272E       AATKCRE
 0069:28A9 idle  AAISPW
 0069:28A9 idle  AAIDTW
 0069:28A9 idle  AAIDTS
 0069:28A9 idle  AAIDTR
 0069:28A9 idle  AAIDTX
 0069:28A9 idle  AAIDTM
 0069:28B0 idle  AMIRPM
 0069:28B0       AMINPM
 02F4:000E       _ConfigDataInitialize
 02F4:0047       _ConfigDataGetPointer
 0301:0003       _DataMgrInitialize
 0301:026C       _DataMgrLockNodeForRead
 0301:0294       _DataMgrLockNodeForWrite
 0301:02BC       _DataMgrUnlockNodeDirty
 0301:02CE       _DataMgrUnlockNode
 0301:02F0       _DataMgrSetCallback
 0301:0306       _DataMgrUpdateImmediate
 0301:0351       _DataMgrNodeUpdated
 0301:03AF       _DataMgrValidateNodeSize
 0301:03CE       _DataMgrForceUpdate
 0301:0475       _DataMgrForceRead
 0301:0543       _DataMgrReset
 0301:05F9 idle  _DataMgrUpdateMode
 0301:0610       _DataMgrResetNode
 0301:062C       _DataMgrGetNodeDefaults
 0301:064D idle  _DataMgrIsNodeConst
 0301:0664 idle  _DataMgrIsNodeCal
 0301:067B       _DataMgrRestartUpdate
 0460:0009       _IntCtrlInitialize
 0460:011D       _IntCtrlSetHandlerProc
 0460:0139       _IntCtrlGetHandlerProc
 0460:017D idle  _i_IntCtrlEnableInterruptNesting
 049D:0004       _main
 04A1:0002       _FillMemory
 04A1:0024       _CopyMemory
 04A1:004D       _MemoryAssign
 04A1:0090       _uumemget
 04A1:0130 idle  _GetAllocatedMemorySize
 04A1:0138       _AllocMemory
 04A1:021A       _FreeMemory
 04A1:029B       _CompareStrings
 04A1:02CF       _segtolin
 04A1:02E9       _lintoseg
 04A1:0309       _AllocMemoryWithError
 04D5:0008       _sysSystemInitialize
 050C:000E       _uiSendUserMessage
 050C:0034       _uiSendUserMessageWait
 050C:005A       _uiSendUserMessageWithData
 050C:008C       _uiSendUserMessageWithDataWait
 050C:00C3       _uiSendStateChangeMessage
 050C:00E9       _uiSendOperationUpdate
 050C:010F       _uiSendVariableUpdate
 050C:0122       _uiSendUpdateAll
 050C:0147       _UIManagerInit
 050C:01CF       _UIStateManager
 050C:03DB       _uiSetNextState
 050C:03F3       _uiSetUserVariable
 050C:042B       _uiGetStatePtr
 050C:0446       _uiGetCurrentState
 050C:044A       _uiRedrawCurrentState
 050C:04E0       _uiGetNumLanguages
 050C:0502       _uiUpdateStateChange
 050C:050D       _uiGetUpdatedState
 050C:0511       _UITimerProc
 050C:0541       _uiTimerProcess
 05C3:0004       _pwSrcSetOp
 05C3:06F2       _pwSrcExecuteAction
 05C3:0708       _pwSrcGetOp
 05C3:0BAF       _pwSrcIsOpAvail
 05C3:0D5C       _pwSrcGetOpDescriptor
 05C3:10AC       _pwSrcInitialize
 05C3:1305       _pwSrcStart
 05C3:1310       _pwSrcForceMode
 05C3:1338 idle  _pwSrcForceModeCancel
 05C3:135A idle  _pwSrcSelectMode
 05C3:1402 idle  _pwSrcGetModeWindow
 05C3:1462       _pwSrcGetModeSource
 05C3:14CE idle  _pwSrcGetModeInfo
 05C3:153C       _pwSrcGetSourceStatus
 05C3:15F2       _pwSrcChangeState
 05C3:15FD idle  _pwSrcGetSourceStatusSpecific
 05C3:1679       _pwSrcSuspend
 05C3:16B4       _pwSrcSuspended
 05C3:16CA idle  _pwSrcEnableSource
 05C3:1762 idle  _pwSrcEnableAll
 05C3:178D       _i_pwSrcForceResync
 05C3:17F1       _i_pwSrcChannelSearch
 05C3:181B       _i_pwSrcGetSrc
 05C3:1864       _i_pwSrcGetWindow
 05C3:4426       _i_pwSrcTask
 0A19:0000       _pwPeriodicInitialize
 0A19:00B2       _pwPeriodicStartTask
 0A19:00DB       _pwPeriodicCreate
 0A19:0197 idle  _pwPeriodicDelete
 0A19:01CC idle  _pwPeriodicStart
 0A19:02BE       _pwPeriodicRestart
 0A19:03D6 idle  _pwPeriodicStop
 0A19:042B       _BackgroundMgr
 0A6A:000B       _pwRosInitialize
 0A6A:000C       _pwRosInSysInit
 0A6A:0017 idle  _pwRosIsInSysInit
 0A6A:001D       _pwRosSendMessage
 0A6A:0041       _pwRosSendMessageWait
 0A6A:0061       _pwRosCreateTimer
 0A6A:009C idle  _pwRosDeleteTimer
 0A6A:00AA       _pwRosStartTimer
 0A6A:00C0       _pwRosStopTimer
 0A6A:00D4       _pwRosReadTimer
 0A6A:00E2       _pwRosCreateSemaphore
 0A6A:0105 idle  _pwRosDeleteSemaphore
 0A6A:011A       _pwRosReserveSemaphore
 0A6A:0160       _pwRosReleaseSemaphore
 0A6A:0175       _pwRosWaitSemaphore
 0A6A:01A7       _pwRosSignalSemaphore
 0A6A:01BC       _pwRosConvertMsToSystemTicks
 0A6A:01E7       _pwRosSetInterruptVector
 0A6A:01FD       _pwRosSystemTick
 0A6A:0203       _pwRosGetSystemClock
 0A6A:0227       _pwRosTaskDelay
 0A6A:025E       _pwRosGetCurrentTaskId
 0A6A:026E       _pwRosGetTaskId
 0A6A:0287       _pwRosGetCurrentTaskPriority
 0A6A:02A3       _pwRosGetTaskPriority
 0A6A:02BC       _pwRosSetTaskPriority
 0A6A:02CF       _pwRosIsTaskSuspended
 0A6A:02EB       _pwRosEventFlagCreate
 0A6A:0306       _pwRosEventFlagWait
 0A6A:0336 idle  _pwRosGetTaskStack
 0A6A:0339       _pwRosAreInterruptsEnabled
 0A6A:034C       _pwRosEventFlagSignal
 0A6A:0362       _pwRosTaskSuspend
 0A6A:0370       _pwRosTaskResume
 0A6A:037E       _pwRosTaskWake
 0A6A:038C       _pwRosTaskSignal
 0A6A:03AC       _pwRosTaskSignalWait
 0A6A:03DC idle  _pwRosTaskCreate
 0A6A:0419       _pwRosTaskCreateComplete
 0A6A:04CF       _pwRosTaskTrigger
 0A6A:04DD       _pwRosReadSystemTicks
 0A6A:04E3       _pwRosCalledFromInterrupt
 0A6A:04FC       _FatalExit
 0ADA:000E       _i_OutputScalerGetDataMgrNode
 0BF9:017E idle  _CalcData
 0DB8:3AC0 idle  _GPGetGPortPhase
 0DB8:467B       _Set_Capture_Enable
 14CD:0F88 idle  _CheckFormat
 14CD:10CE idle  _VideoFormatChanged
 14CD:26F7       _SetTunerVideoFormat
 14CD:270A idle  _ColseCaptureSetup
 1781:11D4 idle  _Read1230Reg
 1781:1213 idle  _Write1230Reg
 1781:16BA       _PW1230_50_60_Init
 1781:16C2       _ChangePipSize
 1781:190C       _ChangePipLeftPos
 1781:1959       _ChangePipTopPos
 1781:19A6       _ChangePipAlpha
 1A02:063A idle  _SrvSetupDisplayMode
 1B07:04DA idle  _PoweronHardware
 1B07:0AB8       _WriteTunerDiv
 1B07:0B0A       _SetChannel
 1B07:0C09       _GetTunerStatus
 1B07:0C23       _SetTunerVideoStandard
 1B07:0CBE       _ChangeTunerStandard
 1B07:0D00       _GetTunerVideoStandard
 1B07:0D4F       _SetTunerAudioStandard
 1B07:0DCA       _GetTunerAudioStandard
 1B07:0E21 idle  _SetTunerAFCStandard
 1B07:0E80 idle  _GetTunerAFCStandard
 1B07:0E8A idle  _SetTunerHz50_60
 1B07:0EDE idle  _GetTunerHz50_60
 1B07:0EE8       _SetStandardAndChannel
 1B07:1021       _GetVideoAudioStandard
 1C0C:0398       _GetAFCStatus
 1C48:0C01 idle  _ChangeChannelMute
 1C48:0CAA idle  _SetVolume
 1C48:0CFA idle  _GetMuteState
 1C48:0CFE idle  _SetMuteState
 1D1C:0007       _dvDriverServiceInitialize
 1D1C:0047       _dvDriverServiceInitializeDrivers
 1D1C:0063       _dvDriverService
 1D1C:00B7       _dvDriverGetParameter
 1D1C:010C       _dvDriverSetParameter
 1D1C:0161       _dvDriverGetParameterDescriptor
 1D1C:01B6       _dvDriverIsRequestAvailable
 1D1C:020B       _dvDriverValidateData
 1D1C:02A3       _dvDriverCreateRequestData
 1D1C:02E3       _dvDriverClassService
 1D1C:03B5       _dvDriverClassServiceDevices
 1D1C:03E9       _dvDriverClassServiceDeviceIDs
 1D1C:043B       _dvDriverSetParameterDword
 1D1C:046F idle  _dvDriverSetParameterPointer
 1D1C:04A4       _dvDriverGetParameterDword
 1D1C:04EC       _dvDriverGetOpDescriptor
 1D1C:0520       _dvDriverServiceSend
 1D1C:0555 idle  _dvDriverServiceGetFirstClassDev
 1D1C:059B       _i_dvDriverUnusedFunctionCPC
 1D1C:059E       _i_dvDriverUnusedFunctionCP
 1D7D:0004       _i_pwCalculateCRC16
 1D7D:001C       _i_pwCalculateCRC16Continuation
 1D84:0008       _pwOemInitialize
 1D84:0159       _pwOemReceiveHostMessage
 1D84:0171       _pwOemDPMSStateChange
 1D84:0172       _pwOEMIsOpAvail
 1D84:03B2       _pwOEMGetOp
 1D84:0932       _pwOEMSetOp
 1D84:1130       _pwOEMExecuteAction
 1D84:14C8       _pwOEMOpDescriptor
 1D84:17A4 idle  _pwOEMGetGuiData
 1D84:1817 idle  _pwOEMSetGuiData
 1D84:1896       _pwOEMNewSourceFound
 1D84:1897       _pwOEMMatchEvent
 1D84:189D       _pwOemGetCustomString
 1D84:18C5       _pwOemOsdWindowEnable
 1D84:18C6       _pwOemDataMgrInitialize
 1D84:18CA       _pwOemSpecialProcessing
 1D84:18CB       _pwOemDisplaySetPower
 1D84:18CF idle  _pwOemIsNV320
 1D84:18DD       _GetCurrentSourceID
 1D84:18E1       _SetPictureUserMode
 1D84:1999       _SavePictureUserMode
 1D84:1ABB idle  _TimerOneSec
 1D84:1AFE       _TimerOneMin
 1D84:1C39 idle  _GetFP13State1111
 1D84:1C76       _VPC3230FPAccess
 1D84:1D13 idle  _GetFP13State
 1D84:1ED7 idle  _Get3230SignalLoss
 1D84:1F45 idle  _Get3230VideoStandard
 1D84:1F62 idle  _BlueScreen
 1D84:1FC4 idle  _SetBlueScreen1230
 1D84:2036 idle  _GetBlueScreen1230
 1D84:205D       _Check_Video_Caption_Pos
 1D84:207B idle  _SetPW1230ToCinameScalerMode
 1D84:20D3 idle  _SetPW1230ToSubtitleScalerMode
 1D84:212B idle  _SetPW1230ToNormalScalerMode
 1D84:2189       _INSearchMenu
 1D84:218D idle  _ProcessPerfectPicture
 1FB0:0002       _hlIntInitialize
 1FB0:0010       _hlIntSetVectorBase
 1FB0:0038       _hlIntMasterEnable
 1FB0:007F idle  _hlIntDisableAll
 1FB0:00F7       _hlIntEnable
 1FB0:0115       _hlIntClearPendingFlag
 1FB0:012F       _hlIntClearPendingFlagFromTheInterrupt
 1FB0:0149       _hlIntClearActiveFlag
 1FB0:0163 idle  _hlIntSetExternalIntMode
 1FB0:0181       _hlIntSetPolarity
 1FB0:019F       _hlIntSetPriority
 1FCE:000F       _pwIspCoreDivideError
 1FCE:0011       _pwIspCoreSingleStep
 1FCE:0013       _pwIspCoreNMI
 1FCE:0015       _pwIspCoreBreakpoint
 1FCE:0017       _pwIspCoreIntoOverflow
 1FCE:0019       _pwIspCoreArrayBounds
 1FCE:001B       _pwIspCoreUnusedOpcode
 1FCE:001D       _pwIspCoreEscOpcode
 1FCF:000F idle  _pwVersion
 1FCF:0018       _pwMiscInitialize
 1FCF:0045       _pwMiscSaveAndRestoreInit
 1FCF:00F9 idle  _pwMiscGetRange
 1FCF:0292       _pwMiscIsOpAvail
 1FCF:038A idle  _pwMiscGetParm
 1FCF:03DB idle  _pwMiscSetParm
 1FCF:0448       _pwMiscWaitForDisplayVSync
 1FCF:046B       _pwMiscAwakeDisplayVSync
 1FCF:048C       _pwMiscGetOpDescriptor
 1FCF:04A8       _pwMiscGetOp
 1FCF:066B       _pwMiscSetOp
 1FCF:083B       _pwMiscExecuteAction
 209C:0166       _hlRegisterWaitForField
 209C:01BD       _hlRegisterShadowFill
 209C:01BE       _hlgcRegisterGet
 209C:01D5       _hlgcRegisterSet
 209C:01E9       _hlgpRegisterGet
 209C:0200       _hlgpRegisterSet
 209C:0214       _hlvpRegisterGet
 209C:022B       _hlvpRegisterSet
 209C:023F       _hlosdRegisterGet
 209C:0257       _hlosdRegisterSet
 209C:026C       _hlvsRegisterGet
 209C:0284       _hlvsRegisterSet
 209C:0299 idle  _hlhsRegisterGet
 209C:02B1       _hlhsRegisterSet
 209C:02C6       _hlegpRegisterGet
 209C:02DE       _hlegpRegisterSet
 209C:02F3 idle  _hledpRegisterGet
 209C:030B       _hledpRegisterSet
 209C:0320       _hldpRegisterGet
 209C:0338       _hldpRegisterSet
 209C:034D       _hlwdRegisterGet
 209C:0365       _hlwdRegisterSet
 209C:037A       _hlGammaRegisterSet
 209C:03D7       _hlosdPaletteRegisterSet
 209C:03F9       _hlosdPaletteRegisterGet
 209C:041B       _hlioRegisterGet
 209C:0433       _hlioRegisterSet
 209C:0448       _hltmRegisterGet
 209C:0460       _hltmRegisterSet
 209C:0475       _hlintRegisterGet
 209C:048D       _hlintRegisterSet
 209C:04EF       _hlrsRegisterGet
 209C:0507       _hlrsRegisterSet
 209C:051C       _hlirRegisterGet
 209C:0534       _hlirRegisterSet
 209C:0549 idle  _hltwRegisterGet
 209C:0561 idle  _hltwRegisterSet
 209C:0576       _hlrsDelayedWriteBegin
 209C:0592       _hlrsDelayedRegisterWrite
 209C:05E3       _hlrsDelayedWriteEnd
 209C:05F3       _hlrsDelayedWriteUpdateDuringBlankingPeriod
 2106:0006       _hlHlayerInit
 2106:001F       _hlInitializeAfterDataMgr
 2106:00A6       _hlIsWrapModeOn
 2106:00AF       _hlSetSignalValidFlag
 2106:0102       _hlGetSignalValidFlag
 2106:0109       _hlIsSourceGport
 2106:0132 idle  _hlChangeMemConstraint
 2106:0160       _hlGetClockRates
 2106:0180       _hlGetClockRatesPtr
 2106:018B       _hlSetClockRates
 2106:01AB       _hlAdjustClockRates
 2106:01D6       _hlMemChangeNeeded
 2106:0225       _hlIsModeSupported
 2106:0245 idle  _hlChangeMemoryConfiguration
 2106:029F       _hlSetMemoryConfiguration
 2106:0313 idle  _hlGetMemoryConfiguration
 2106:0339       _hlGetInputResolutionSize
 2106:034E       _hlGetInputResolutionRect
 2106:036F       _hlPositionUpdateDuringBlankingPeriod
 2106:0538       _i_hlGetOutputResolutionSize
 2106:0564       _i_hlGetOutputResolutionRect
 2106:059F       _i_hlHlayerDataGet
 2106:05A5       _i_hlHlayerTempDataGet
 2106:05AB       _i_hlSetupOutputDisplay
 2106:062D idle  _i_hlGetVLDelay
 2106:0631       _i_hlGetIOResolutionRects
 2106:0650 idle  _i_hlCalculateFramelockValues
 2106:073C idle  _i_hlCalculateDpldly
 2106:12A5       _i_hlRecalculateFramelockValues
 2106:1309 idle  _i_hlIsHperInvalid
 2106:1317       _i_hlGetDvpcnt
 2106:1385       _i_hlIsModeSupported
 2106:13AB       _i_hlSetModeData
 2106:13D0       _i_hlCheckFailsafeMode
 2106:13E4 idle  _i_hlSetDefaultDCLK
 2106:1432       _i_hlSetLastDCLK
 2106:1444       _i_hlGetActualRequestedDCLK
 2347:0006 idle  _pwHostTask
 2347:04D8       _pwHostStart
 2347:05E0       _pwHostLogTrace
 2347:0695       _pwHostLogError
 2347:0750 idle  _pwHostSendOemMessage
 2347:07D4 idle  _ProcessSystemMessage
 2347:08E0 idle  _ProcessEventMessage
 2347:08FE idle  _ProcessOperationMessage
 2347:0AB1 idle  _ProcessVariableMessage
 2347:0BC9 idle  _ProcessUIStateMessage
 2347:0C26 idle  _ProcessForceModeMessage
 2347:0D99 idle  _ProcessDiagReadMessage
 2347:14F4 idle  _ProcessDiagWriteMessage
 2347:1A48 idle  _ProcessDMReadMessage
 2347:1A9C idle  _ProcessDMWriteMessage
 2347:1ACC idle  _i_pwHostSuspend
 2347:1B5D idle  _i_pwHostIsSuspended
 2347:1B92 idle  _FindHostTask
 2347:1BD3 idle  _ProcessOemMessage
 2347:1C02 idle  _ProcessPWCmdMessage
 2347:1D51 idle  _pwCmdExecute
 2347:1E5C idle  _ValidHeader
 2347:1EDB idle  _ResetBuffer
 2347:1EE1 idle  _SendBuffer
 2347:1F09 idle  _BufferBytes
 2347:1FB7 idle  _SendMessage
 2347:20B3 idle  _SendResponse
 2347:2114 idle  _GetBytes
 2347:21A9 idle  _SendBytes
 2566:0001       _uiBhvSetUserVariable
 2566:003F       _uiBhvGetUserVariable
 2566:005B       _uiBhvClearUserVariable
 2566:0073       _uiBhvToggleUserVariable
 2566:008B       _uiBhvSetSystemVariable
 2566:00CE       _uiBhvGetSystemVariable
 2566:00E6       _uiBhvClearSystemVariable
 2566:00FA       _uiBhvToggleSystemVariable
 2566:010E       _uiBhvGetBehaveInfo
 2566:0267       _uiBhvEvaluateCondition
 2566:0279       _uiBhvGetSubMenu
 2566:02A1       _uiBhvGetSubMenuParent
 2566:036A       _uiBhvGetGrayCondition
 2566:039D       _uiBhvGetHideCondition
 2566:03D0       _uiBhvGetSelectCondition
 2566:0403       _uiBhvGetManualChildMenu
 2566:0436       _uiBhvGetAlternateRendering
 2566:0527       _uiBhvEnableConditionCache
 25F7:000D       _hlScalerInit
 25F7:00D5 idle  _i_hlScalerGetNLFlags
 25F7:00D9 idle  _i_hlScalerGetNLVStretch
 25F7:00DD idle  _hlScalerVSSetWindow
 25F7:0110       _hlScalerSetupWindows
 25F7:013D idle  _hlScalerSetInputClipRect
 25F7:01A5 idle  _hlScalerSetOutputDispRect
 25F7:021E idle  _hlScalerInputRes
 25F7:0233       _hlScalerSetMode
 25F7:023E       _hlScalerGetMode
 25F7:024C idle  _i_hlScalerGetScaleSource
 25F7:0250 idle  _hlScalerGetInputRes
 25F7:0265       _hlScalerOutputRes
 25F7:02AE idle  _hlScalerGetOutputRes
 25F7:02C3 idle  _hlScalerGetDesiredOutputRes
 25F7:02D8       _hlScalerGetInputRect
 25F7:02EF       _hlScalerGetOutputAspect
 25F7:02FD       _hlScalerGetOutputRect
 25F7:0314 idle  _hlScalerPosition
 25F7:033F       _hlScalerOffset
 25F7:0354       _hlScalerSharpness
 25F7:0377       _hlScalerNonlinearity
 25F7:038E idle  _hlScalerFlipping
 25F7:0399       _hlScalerRotate
 25F7:03A4       _hlScalerIsRotateEnabled
 25F7:03AB       _hlRotateRectIfNeeded
 25F7:03EB idle  _hlScalerHasRotation
 25F7:03EE       _hlScalerHasNonlinear
 25F7:03F2       _hlScalerHasZoom
 25F7:03F6 idle  _hlScalerHasKeystone
 25F7:03F9 idle  _hlScalerHasEnhancedVideo
 25F7:03FC       _hlScalerKeystoneMode
 25F7:0407 idle  _hlScalerKeystoneModeGet
 25F7:040B       _hlScalerUpdateEnable
 25F7:0420       _hlScalerSetLinearRegion
 25F7:0431       _hlScalerConfigure
 25F7:048B       _hlScalerSetFrameBufferMode
 25F7:04A2 idle  _hlScalerUpdateCoefficients
 25F7:04F4       _hlScalerUpdateDuringBlankingPeriod
 25F7:0515       _hlScalerSetKeystoneVertScaleMax
 25F7:0520       _hlScalerSetZoom
 25F7:052B       _hlScalerGetZoom
 25F7:0539       _i_hlScalerGetZoomMinInputSize
 25F7:0587       _i_hlScalerResetCallback
 25F7:0592       _i_hlScalerSetOverlap
 25F7:05F3 idle  _i_hlScalerGetDataHeight
 27FB:0007       _hlDisplayInitialize
 27FB:0049       _hlDisplayInitTCON
 27FB:0856 idle  _hlDisplayUpdateShadowedRegisterImages
 27FB:0865       _hlDisplaySetBlankColor
 27FB:08B5 idle  _hlDisplaySetBrightness
 27FB:08F9 idle  _hlDisplayGetBrightness
 27FB:094D       _hlDisplaySetContrast
 27FB:0AA9       _hlDisplaySetPower
 27FB:0C52       _hlDisplaySetWindowPos
 27FB:0CE9       _hlSetGammaEntry
 27FB:0D00       _hlHasColorMatrix
 27FB:0D04       _hlDisplaySetColorMatrix
 27FB:0D74       _hlHasColorWarping
 27FB:0D77       _hlDisplayHasBorder
 27FB:0D7A       _hlDisplaySetVLockMode
 27FB:0E3F       _hlDispCheckFramelock
 27FB:0E96       _hlDispSetPanel
 27FB:0EFE       _hlDispGetCurrentPanelParams
 27FB:0F2F       _i_hlDisplayVsyncProcessing
 27FB:0FC9       _i_hlInitOutputDisplay
 293C:0001       _hlInitTimers
 293C:0063       _hlTimerSetup
 293C:00A0 idle  _hlTimerSetupTicks
 293C:017F idle  _hlTimerGetTimeuSecs
 293C:0276 idle  _hlTimerGetTimeTicks
 293C:0295       _hlTimerSave
 293C:02E8       _hlTimerRestore
 293C:0361       _hlTimersSetPrescaler
 293C:03D3       _hlTimerStart
 293C:0407       _hlTimerStop
 293C:0445       _hlResetWatchDogTimer
 2981:0003       _hlInitialize
 2981:03A1       _hlGetSettings
 29BB:0007       _hlRomWaitStatesSet
 29BB:005E       _hlRamWaitStatesSet
 29BB:00B5       _hlMiscCSWaitStatesSet
 29BB:010C       _hlCfgWaitStates
 29DA:0006 idle  _TempDelay
 29DA:0032       _dvGPIOInitialize
 29DA:0205       _dvGPIOInitGPO
 29DA:0253       _dvGPIOsetField
 29DA:02A7       _dvGPIOgetField
 29DA:0412 idle  _dvGPIOgetBool
 29DA:0443       _dvGPIOgetMask
 29DA:04A2 idle  _dvGPIOgetFlags
 29DA:04E3 idle  _i_dvGPIOgetPortType
 29DA:052D       _i_dvGPIOlock
 29DA:053E       _i_dvGPIOunlock
 29DA:0549 idle  _i_dvGPIOgetShadowPointer
 29DA:0599       _i_dvGPIOgetAddress
 29DA:05E8       _i_dvGPIOgetMask
 2A5D:000C idle  _dvOemInterfaceGetIndex
 2A5D:0040       _dvOemInterfaceInitialize
 2A5D:0062 idle  _dvOemInterfaceRegistersAccess
 2A5D:018A       _dvOemInterfaceReadRegisters
 2A5D:01A4       _dvOemInterfaceWriteRegisters
 2A5D:01BE idle  _dvOemInterfaceBlockAccessDevice
 2A5D:0318 idle  _dvOemInterfaceBlockAccess
 2A5D:0347       _dvOemInterfaceBlockRead
 2A5D:0365       _dvOemInterfaceBlockReadAddress
 2A5D:0385       _dvOemInterfaceBlockWrite
 2A5D:03A3       _dvOemInterfaceBlockWriteAddress
 2A5D:03C7 idle  _dvOemInterfaceReserve
 2A5D:03FA       _dvOemInterfaceGetId
 2AA2:000A       _pwDPMSInitialize
 2AA2:024D       _pwDpmsStartTask
 2AA2:0258 idle  _i_pwDpmsTask
 2AA2:030B       _pwDPMSIsOpAvail
 2AA2:038C       _pwDPMSGetOpDescriptor
 2AA2:0463       _pwDPMSGetOp
 2AA2:0524       _pwDPMSSetOp
 2AA2:05C3       _pwDPMSExecuteAction
 2AA2:05E9 idle  _pwDPMSPause
 2AA2:05FF idle  _pwDPMSPauseGet
 2AA2:0612 idle  _pwDPMSEnable
 2AA2:06A0 idle  _pwDPMSEnableGet
 2AA2:06B1       _pwDPMSGetCurrentState
 2AA2:06BF idle  _pwDPMSForcePowerState
 2AA2:06E9 idle  _pwDPMSGetOnTimeRange
 2AA2:0791 idle  _pwDPMSGetOnTime
 2AA2:0846 idle  _pwDPMSSetOnTime
 2AA2:09B6 idle  _pwDPMSResetOnTime
 2AA2:0A3C idle  _pwDPMSGetLampParms
 2AA2:0A8A idle  _pwDPMSSetLampParms
 2AA2:0B0A idle  _pwDPMSGetLampRange
 2AA2:0B50       _pwDPMSUserInput
 2AA2:19F0 idle  _DPMSTimer
 2C63:0008       _pwOsdInitialize
 2C63:00C6 idle  _pwOsdTransparentModeEnable
 2C63:00DD idle  _pwOsdIsTransparentModeEnabled
 2C63:00E7       _pwOsdGetTransparentColor
 2C63:0169       _pwOsdSetMode
 2C63:01EB       _pwOsdSuspendDrawing
 2C63:020B       _pwOsdRestoreWindow
 2C63:0247       _pwOsdIsCaptureBlanked
 2C63:0256       _pwOsdSetBlankingColor
 2C63:028B       _pwOsdBlankCapture
 2C63:02EB       _pwOsdUnblankCapture
 2C63:0355       _pwOsdWindowEnable
 2C63:039F       _pwOsdIsWindowEnabled
 2C63:03A9       _pwOsdSetWindowPos
 2C63:04BE       _pwOsdGetWindowPos
 2C63:04EC       _pwOsdGetPosHorz
 2C63:0500       _pwOsdGetPosVert
 2C63:0514       _pwOsdGetPosDiscrete
 2C63:0528       _pwOsdSetPosHorz
 2C63:0547       _pwOsdSetPosVert
 2C63:0566       _pwOsdSetPosDiscrete
 2C63:062F       _pwOsdGetUserPosition
 2C63:0701       _pwOsdGetGridWindow
 2C63:0789 idle  _pwOsdBlockOperationLock
 2C63:079A idle  _pwOsdBlockOperationUnlock
 2C63:07A5       _pwOsdSetGraphicOffset
 2C63:07C5 idle  _pwOsdGetGraphicOffset
 2C63:07DC       _pwOsdDrawRectangle
 2C63:08F8       _pwOsdClearRectangle
 2C63:0936       _pwOsdDrawHollowRect
 2C63:0BC0       _pwOsdDrawBitmap
 2C63:0CD5       _pwOsdDrawBlitmap
 2C63:0D57       _pwOsdDrawBlitItem
 2C63:0DFB idle  _pwOsdSetCharFont
 2C63:0E23 idle  _pwOsdDrawChar
 2C63:0E66 idle  _pwOsdDrawString
 2C63:11EE       _pwOsdGetStringSize
 2C63:12E2       _pwOsdDrawText
 2C63:1342       _pwOsdDrawText2
 2C63:1608       _pwOsdDrawNumber
 2C63:1869       _pwOsdFillWindow
 2C63:18C4 idle  _pwOsdClearWindow
 2C63:18D0       _pwOsdIsPointValid
 2C63:18F9 idle  _pwOsdIsRectangleValid
 2C63:1969       _pwOsdSetOverlayColors
 2C63:198B       _pwOsdLowColorOverlayFunctionEnable
 2C63:19C6       _pwOsdEnableSolidBackground
 2C63:1A38       _pwOsdBackgroundIsSolid
 2C63:1A41 idle  _pwOsdRotateWindowPos
 2C63:1A93       _pwOsdGetOrientation
 2C63:1A9D       _pwOsdSetOrientation
 2C63:1AD1       _pwOsdSetColorOverride
 2C63:1AEE       _pwOsdClearColorOverride
 2C63:1AF5       _pwOsdHollowForceModeEnable
 2C63:1B0C idle  _i_pwOsdClearColor
 2C63:1B1E       _i_pwOsdResumeDrawing
 2C63:1B3B       _i_pwOsdRotatedOsdPosition
 2C63:1B78       _i_pwOsdRotateOsdRectangle
 2E6F:0009       _hlGenCtlInitialize
 2E6F:003C idle  _hlGenCtlLockRegistersFromUpdate
 2E6F:004A       _hlGenCtlLockRegistersEnable
 2E6F:005C idle  _hlGenCtlIsLockEnabled
 2E6F:005F idle  _hlGenCtlLockSyncStateClear
 2E6F:0067 idle  _hlGenCtlLockSyncStateRestore
 2E6F:006F idle  _hlGenCtlShadowRegistersEnable
 2E6F:0081 idle  _hlGenCtlShadowRegistersUpdate
 2E6F:0082       _hlGenCtlBlockOperationLock
 2E6F:00CB       _hlGenCtlBlockOperationUnlock
 2E6F:00E9       _hlGenCtlHasFailsafe
 2E7D:0012       _pwInputInitialize
 2E7D:00A6       _pwInputSendSignal
 2E7D:00BA       _pwInputRegisterCallback
 2E7D:00F5       _pwInputTaskStart
 2E97:0000       _pwOperationsInitialize
 2E97:0037 idle  _pwOpGetUIIncrement
 2E97:0066       _pwOpExecuteIsOpAvail
 2E97:00DE       _pwOpExecuteSetValue
 2E97:02A2       _pwOpExecuteGetValue
 2E97:03BF       _pwOpExecuteIncrementCrop
 2E97:0463       _pwOpExecuteIncrement
 2E97:069F       _pwOpExecuteGetCropRange
 2E97:081F       _pwOpExecuteGetRange
 2E97:0855 idle  _pwOpExecuteGetLongRange
 2E97:08DB       _pwOpExecuteAction
 2E97:095F idle  _pwOpCroppingMode
 2E97:0980       _pwOpGetDescriptor
 2F47:000A       _uiEventMatchFirst
 2F47:003A       _uiEventMatchNext
 2F47:0072       _uiEventMatchEnterExitFirst
 2F47:00B1       _uiEventMatchEnterExitNext
 2F72:000A       _uiBhvMenuSetupState
 2F72:01AF       _uiBhvIsMenuState
 2F72:01B8       _uiBhvGetActiveMenu
 2F72:01EB       _uiBhvSetActiveMenu
 2F72:0251       _uiBhvMenuGetParent
 2F72:029C       _uiBhvMenuGetChild
 2F72:02F0       _uiBhvGetFirstVisibleMenu
 2F72:0309       _uiBhvGetNextVisibleMenu
 2F72:0393       _uiBhvMenuGetInfoByID
 2F72:03FA       _uiBhvMenuSetActiveItem
 2F72:04BF       _uiBhvMenuSetVisibility
 2F72:04DC       _uiBhvMenuIsVisible
 2F72:04FB       _uiBhvMenuShowChild
 2F72:05C5       _uiBhvMenuGridRowItems
 2F72:0630       _uiBhvSetItemInvertFlag
 2F72:0647       _uiBhvGetItemInvertFlag
 2F72:065B       _uiBhvSetItemGrayFlag
 2F72:0672       _uiBhvGetItemGrayFlag
 2F72:0686       _uiBhvIsMenuItemGray
 2F72:06B8       _uiBhvIsMenuItemVisible
 2F72:06F4       _uiBhvMenuAreSubItemsPresent
 2F72:0728       _uiBhvMenuGetWrapEnable
 2F72:0746       _uiBhvMenuNextItem
 2F72:07B2       _uiBhvMenuPrevItem
 2F72:0827       _uiBhvMenuSetChanged
 2F72:082D       _uiBhvMenuGetChanged
 2F72:0837       _uiBhvMenuGetInfo
 2F72:08E0       _uiBhvMenuUpdateChildPositions
 3140:0004       _uiExecuteAllControls
 3140:00A5       _uiUpdateControls
 3140:014A       _uiSetNewStateForClipping
 3140:015C       _uiClipControlRectangle
 3140:01F4       _uiCheckClipping
 3140:0234       _uiCtlUpdateDisplay
 3140:0344 idle  _uiCtlApplyCropping
 318B:0008       _uiCtlMenu
 318B:01BF       _uiExecuteMenuActiveItem
 318B:052C       _uiExecuteMenuNavigate
 318B:08CA       _uiExecuteMenuSelectList
 318B:09CB       _uiCtlMenuRenderContent
 318B:0A5D idle  _uiCtlMenuSelectItem
 318B:0AE9       _i_uiCtlMenuSuspendDrawing
 3316:000D       _uiDrawDrawList
 3316:0259       _uiSetDefaultOsdPalette
 3316:026E       _uiSetDefaultOverlayFunctions
 3316:02AE       _uiGetBackgroundColor
 3316:02B6       _uiSetBackgroundColor
 3316:02C8       _uiDrawItem
 3316:03C4       _uiUndrawItem
 3375:0005       _uiOsdZeroPosition
 3375:003C       _uiOsdGetHorzStepSize
 3375:0068       _uiOsdGetVertStepSize
 3375:0094       _uiOsdChangePosAndSize
 3375:01D8       _uiOsdUpdatePosition
 3375:027C       _uiClearOSD
 33CB:0009       _uiClearModifiedOpsList
 33CB:0010       _uiAddToModifiedOpsList
 33CB:005B       _uiModifiedOpListIsEmpty
 33CB:006A       _uiOpIsInModifedOpsList
 33CB:0095       _uiExecuteEnterExitOperations
 33CB:011D       _uiStartStopTimer
 33FA:0002       _uiBhvConditionMgrSetupState
 33FA:00B5       _uiBhvConditionMgrUpdateConditions
 33FA:0114       _uiBhvConditionMgrUpdateState
 33FA:01D4       _uiBhvConditionMgrGetCondition
 33FA:0213       _uiBhvSetupOffsetPaint
 33FA:043D       _uiBhvResetOffsetPaint
 348F:000F       _uiBhvDynamicMgrSetupState
 348F:009D       _uiBhvDynamicMgrUpdateState
 348F:0462       _uiBhvDynamicMgrGetBehaviorEntry
 34F1:000C       _i_pwSrcInputInitialize
 34F1:0096       _i_pwSrcInputGetSourceCount
 34F1:009C       _i_pwSrcInputGetNextSrc
 34F1:00B4       _i_pwSrcInputGetPreviousSrc
 34F1:00D1       _i_pwSrcInputRouteSrc
 34F1:01C3       _i_pwSrcInputRouteSrcMonitor
 34F1:036C       _i_pwSrcInputUnRouteSrc
 34F1:03AB       _i_pwSrcInputGetSourceRoute
 34F1:03E2 idle  _i_pwSrcInputGetPortRoute
 34F1:0401       _i_pwSrcInputGetSource
 34F1:0423 idle  _i_pwSrcInputCancelRoute
 34F1:043E idle  _i_pwSrcInputGetLastDeviceIndex
 34F1:045B idle  _i_pwSrcInputGetDevice
 34F1:0480 idle  _i_pwSrcInputIsDeviceInActiveRoute
 34F1:054D       _i_pwSrcInputIsDriverServiceAvail
 34F1:065D       _i_pwSrcInputDriverServiceAllDevices
 34F1:069D       _i_pwSrcInputDriverService
 34F1:08B7       _i_pwSrcInputPortIndex
 34F1:08CF       _i_pwSrcInputSearchDeviceList
 35E6:000F       _i_pwSrcAutoInitialize
 35E6:001B       _i_pwSrcAutoCancelAuto
 35E6:0031       _i_pwSrcAutoComputeAutoFlags
 35E6:0099       _i_pwSrcSettingAutoSetup
 3666:0000       _i_pwSrcAutoADCCalibrate
 376D:0002       _i_pwSrcSettingInitialize
 376D:0098       _i_pwSrcSettingSetOp
 376D:0561       _i_pwSrcSettingGetOp
 376D:09E3       _i_pwSrcSettingIsOpAvail
 376D:0B02       _i_pwSrcSettingSetup
 376D:0EE7       _i_pwSrcSettingClearSetting
 376D:0F2B       _i_pwSrcSettingBroadcastSettings
 376D:0F45       _i_pwSrcSettingOpDescriptor
 376D:10F3       _i_pwSrcSettingUpdateFactoryDefaults
 376D:1152       _i_pwSrcSettingRestoreOriginalSettings
 376D:11D7       _i_pwSrcSettingUpdateOriginalSettings
 376D:1233       _i_pwSrcSettingGetDefaultBrightness
 376D:127C       _i_pwSrcSettingGetDefaultContrast
 3A6E:0006       _i_pwSrcDetInitialize
 3A6E:0015       _i_pwSrcDetPort
 3A6E:08A7       _i_pwSrcDetCheckOutOfRange
 3A6E:0954       _i_pwSrcDetSpecificMode
 3A6E:0978       _i_pwSrcDetMonitor
 3A6E:09EF idle  _i_pwSrcDetCancelDetection
 3A6E:09FA       _i_pwSrcDetectionGetAlternate
 3A6E:0AF5       _i_pwSrcDetGetModeData
 3A6E:0BBE       _i_pwSrcDetSetPixelMode
 3A6E:0D82       _pwSrcDetectionCheckAlternateResolution
 3BB5:0000       _i_pwSrcDisplayInitialize
 3BB5:00C8       _i_pwSrcDisplaySetOp
 3BB5:01DF       _i_pwSrcDisplaySetOpWindow
 3BB5:0540       _i_pwSrcDisplayGetOp
 3BB5:05F1       _i_pwSrcDisplayGetOpWindow
 3BB5:0815       _i_pwSrcDisplayIsOpAvailWindow
 3BB5:08AC       _i_pwSrcDisplayOpDescriptorWindow
 3BB5:0A4B       _i_pwSrcDisplayOpDescriptor
 3BB5:0AC9       _i_pwSrcDisplayScaleWindow
 3BB5:0DF9       _i_pwSrcDisplayShowBitmap
 3BB5:0F5A       _i_pwSrcDisplayClearBitmap
 3BB5:0F83       _i_pwSrcDisplayShowSource
 3BB5:1141       _i_pwSrcDisplayClearSource
 3BB5:1224       _i_pwSrcDisplaySetupForAutoX
 3BB5:1305       _i_pwSrcDisplayWindowDisplayable
 3BB5:1349       _i_pwSrcDisplayInhibit
 3BB5:1370       _i_pwSrcDisplayChange
 3BB5:13F5       _i_pwSrcDisplayWindowMgrRefresh
 3D81:0005       _i_pwSrcTestDisplayPattern
 3D81:001E       _i_pwSrcTestDisplayBitmap
 3D81:0047       _i_pwSrcTestGetParameters
 3D81:00E2       _i_pwSrcTestDraw
 3D81:01C7       _pwSrcTestGetNumberOfTestPatterns
 3DCA:000D idle  _hlOsdSetPaletteGain
 3DCA:0024       _hlOsdSetPalette
 3DCA:0043       _hlOsdSetPaletteColor
 3DCA:00E7       _hlOsdGetGrayTable
 3DCA:00ED       _hlOsdGetGrayMode
 3DCA:00F1       _hlOsdSetGrayMode
 3DCA:0106       _hlOsdLoColorDrawRectangle
 3DCA:01E0       _hlOsdLoColorDrawBitmap
 3DCA:02CC       _hlOsdLoColorDrawBitmapRect
 3DCA:03A4       _hlOsdLoColorGetPixel
 3E42:000E       _i_pwSrcUtilIntialize
 3E42:002E       _i_pwSrcUtilSendSourceBasedEvent
 3E42:0120       _i_pwSrcUtilSendWindowBasedEvent
 3E42:020B       _i_pwSrcUtilSrcCtlReadLock
 3E42:0226       _i_pwSrcUtilSrcCtlReadUnlock
 3E42:0233       _i_pwSrcUtilSrcCtlWriteLock
 3E42:024E       _i_pwSrcUtilSrcCtlWriteUnlock
 3E42:0257       _i_pwSrcUtilEnableCapture
 3E42:0291       _i_pwSrcUtilDisplayBlank
 3E42:02A8       _i_pwSrcUtilOsdBlank
 3E42:02BF       _i_pwSrcUtilGetNextSrc
 3E42:0323       _i_pwSrcUtilGetPrevSrc
 3E42:0387       _i_pwSrcUtilGetStatus
 3E42:03B8       _i_pwSrcUtilAutoDisable
 3E42:040F       _i_pwSrcUtilGetAutoDisable
 3E42:042B       _i_pwSrcUtilGetAutoDisables
 3E84:000F       _i_pwSrcTVInitialize
 3E84:00AB       _i_pwSrcTVSetOp
 3E84:03F3       _i_pwSrcTVSetOpWindow
 3E84:083F       _i_pwSrcTVGetOp
 3E84:0993       _i_pwSrcTVGetOpWindow
 3E84:0B95       _i_pwSrcTVIsOpAvail
 3E84:0C35       _i_pwSrcTVOpDescriptor
 3E84:0CE4       _i_pwSrcTVOpDescriptorWindow
 3E84:0E2D       _i_pwSrcTVChannelSearchAdvance
 3E84:177E idle  _MySetupDefaultDisplayMode
 3E84:17AB       _SetCurrentChannel
 3E84:17BD       _SetCurrentDivisor
 3E84:1836 idle  _SetTunerDivisorMaxMin
 3E84:1D79 idle  _i_pwSrcTvUpdateRating
 3E84:1D9A idle  _Bri_Con_Col_Zero
 3E84:1DE0 idle  _Bri_Con_Col_Back
 3E84:1E84 idle  _Picture_UnBlack
 3E84:1F3F       _GetnotsaveFlag
 3E84:1F53 idle  _SetFirstTimeChangeBand
 4079:000A       _hlRectCopy
 4079:0045       _hlRectOffset
 4079:008B       _hlRectCenterRect
 4079:00EE       _hlRectCenterOnPoint
 4079:0153       _hlRectInflate
 4079:0199       _hlRectFromSize
 4079:01C8       _hlSizeFromRect
 4079:01F6       _hlRectWidth
 4079:0205       _hlRectHeight
 4079:0215       _hlRectExpandToFit
 4079:0300       _hlRectLocate
 4079:034A       _hlRectLimitToRect
 4079:0462       _hlRect1EnclosesRect2
 40C3:000C       _hlSerialInitialize
 40C3:00AF       _hlSerialGetBaudRate
 40C3:00C7       _hlSerialSetBaudRate
 40C3:0290 idle  _hlSerialGetByte
 40C3:02B1       _hlSerialGetData
 40C3:03D5       _hlSerialTransmitData
 40C3:04F8 idle  _hlSerialTransmitByte
 40C3:0517 idle  _hlSerialClearTransmitBuffer
 40C3:052D idle  _hlSerialClearReceiveBuffer
 40C3:053D       _hlSerialEnable
 40C3:0565 idle  _hlSerialGetEnable
 40C3:0569       _hlSerialRestart
 40C3:059D idle  _i_hlSerialGetOutBuffCharCount
 411D:000F       _i_dvScalerModeGet
 411D:007A       _i_dvScalerModeSet
 411D:0178       _i_dvScalerUpdate
 41BB:000A       _i_dvScalerZoomInitialize
 41BB:002B       _i_dvScalerZoomReset
 41BB:004C       _i_dvScalerZoomGetMagnification
 41BB:005F       _i_dvScalerZoomGetRange
 41BB:0170       _i_dvScalerZoomGetCenter
 41BB:0185       _i_dvScalerZoomSetCenter
 41BB:019A       _i_dvScalerZoomSetMagnification
 41BB:02FA       _i_dvScalerZoomGetPan
 41BB:0336       _i_dvScalerZoomSetPan
 41BB:040D       _i_dvScalerZoomGetMaximum
 41BB:046D       _i_dvScalerZoomGetMinimum
 41BB:04B4 idle  _i_dvZoomSetRect
 4207:000B       _i_dvScalerGetFilter
 4207:0022       _i_dvScalerSetFilter
 4207:008A       _i_dvScalerSetupFilter
 4207:009D idle  _i_dvScalerResetFilter
 4228:000D       _i_dvScalerGetStretch
 4228:0024       _i_dvScalerSetStretch
 4228:00CF       _i_dvScalerStretchGetRange
 4228:00FA       _i_dvScalerGetClipping
 4228:01EE       _i_dvScalerSetClipping
 4228:038F       _i_dvScalerGetClippingOffset
 4228:03F0       _i_dvScalerSetClippingOffset
 4228:0539       _i_dvScalerGetLinearRegion
 4228:0550       _i_dvScalerSetLinearRegion
 4228:0572       _i_dvScalerLinearRegionGetRange
 4281:000D       _hlVideoInitialize
 4281:006B       _hlVideoCaptureEnable
 4281:0079 idle  _hlVideoGetCaptureWindowExpansion
 4281:008F       _hlVideoSetCaptureWindowExpansion
 4281:0113 idle  _hlVideoGetCaptureWindowOffsets
 4281:012A       _hlVideoSetCaptureWindowPos
 4281:027F       _hlVideoGetCaptureWindowPos
 4281:036F       _hlVideoSetRotateMode
 4281:038A       _hlVideoSetInputMode
 4281:0457       _hlVideoSetFrameBufferMode
 4281:04A1       _hlVPortInputResolutionChange
 4281:04C3       _i_hlVPortChangeVPosition
 4281:04E7       _i_hlVportUpdateOnDportVSync
 4281:055C       _i_hlVideoMemoryWasReconfigured
 4281:0570       _i_hlVideoChangedScaleMode
 4281:0587       _i_hlVPortGetVDataStart
 4281:058F       _i_hlVPortSetDataEnableOffset
 4281:05A0 idle  _i_hlVPortGetFieldSize
 42DC:0006 idle  _LimitXTo
 42DC:0029       _ResolutionsAreValid
 42DC:00D8       _SetScaleParamsPct
 42DC:03FE       _SetScaleParamsRect
 432A:000B       _hlImageMemFillRect
 432A:0051       _hlImageMemFill
 432A:00C7 idle  _hlImageMemReadRect
 432A:01D2       _hlImageMemCalcPoint
 432A:027D idle  _hlImageMemPixelCount
 432A:02D6       _hlImageWordGranularity
 432A:030F       _hlImagePixelGranularity
 432A:034D       _hlImageRead24BitPixel
 4389:000F idle  _hlGraphicGetCaptureWindowExpansion
 4389:0025       _hlGraphicSetCaptureWindowExpansion
 4389:00A9 idle  _hlGraphicGetCaptureWindowOffsets
 4389:00C0       _hlGraphicSetCaptureWindowPos
 4389:0202       _hlGraphicGetCaptureWindowPos
 4389:02FD       _hlGPortInputResolutionChange
 4389:032B       _hlGPortGetInputSourceHLines
 4389:0339 idle  _hlGPortGetActualHLines
 4389:0347       _hlGPortSetActualHLines
 4389:0357       _i_hlGraphicInitialize
 4389:0425       _i_hlGraphicMemoryWasReconfigured
 4389:0439       _i_hlGraphicSetBlackDetectLevel
 4389:0466       _i_hlGraphicGetHalfSampleMode
 4389:0473       _i_hlGraphicSetFrameBufferMode
 4389:04A0       _i_hlGraphicCaptureEnable
 4389:04F9 idle  _i_hlGraphicDualRevSetting
 4389:0536       _i_hlGraphicUpdateLineAB
 4389:0596       _i_hlGraphicSetChannelMode
 4389:061F       _i_hlGPortChangeVPosition
 4389:0643       _i_hlGraphicChangedScaleMode
 4389:065A       _i_hlGportUpdateOnDportVSync
 4389:06CB       _i_hlGPortGetVDataStart
 4389:06D3       _i_hlGPortSetDataEnableOffset
 4389:06E4 idle  _i_hlGPortGetFieldSize
 441A:0005       _hlDPortISPInitialize
 441A:0051 idle  _hlDPortISPGetVBlankCount
 441A:0055       _i_hlDPortISPGetOsdColor
 441A:0082       _i_hlDPortISPSetOsdColor
 441A:0092       _i_hlDPortISPGetDvpcnt
 441A:00E7       _i_hlDPortEnableDvpcntUpdates
 4436:000B       _hlAutoInitialize
 4436:001E       _hlAutoPhaseModeEnable
 4436:01EE idle  _hlAutoIsInterlaced
 4436:0247 idle  _hlAutoIsInterlacedDetected
 4436:0279       _hlAutoForceInterlacedMode
 4436:0284       _hlAutoInitVideoPort
 4436:03B3       _hlAutoEndVideoInit
 4476:000F       _hlGPortISPInitialize
 4476:005F       _hlGPortISPEnable
 4476:007B idle  _hlGPortISPIsSafetyModeEnabled
 4476:007F       _hlGPortISPGetVBlankCount
 4488:000B       _hlVPortISPInitialize
 4488:005C       _hlVPortISPEnable
 4488:0078 idle  _hlVPortISPIsSafetyModeEnabled
 4488:007C       _hlVPortISPGetVBlankCount
 449A:0040       _BroadcastOperationID
 449A:0095       _SendMessageToDevice
 449A:013C       _SoftReset
 449A:0308       _MyDelay
 44CD:0004       _i_pwSrcSyncMonitorInitialize
 44CD:001A       _i_pwSrcSyncMonitorEnable
 44CD:0116       _i_pwSrcSyncMonitorDisable
 44CD:01C5 idle  _i_pwSrcSyncMonitorDisableAll
 44FA:000A       _dvKeypadService
 44FA:00F8       _dvKeypadInitialize
 44FA:0204       _dvKeypadProcessCommand
 44FA:0425 idle  _dvKeypadAnyKey
 455C:000B idle  _dvPwmEnable
 455C:009B idle  _dvPwmInitialize
 455C:016C       _dvPwmSetLevel
 455C:021A       _dvPwmGetLevel
 455C:022E       _dvPwmGetRange
 4581:0002       _hlOsdInitialize
 4581:0067       _hlOsdSetMode
 4581:0068 idle  _hlOsdGetMode
 4581:0075       _hlOsdWindowEnable
 4581:010F idle  _hlOsdIsWindowEnabled
 4581:0116       _hlOsdSetWindowPos
 4581:0397       _hlOsdGetWindowPos
 4581:0411       _hlOsdBlankModeEnable
 4581:0455 idle  _hlOsdIsBlankModeEnabled
 4581:046D       _hlOsdOverlayFunctionEnable
 4581:048C       _hlOsdSetOverlayColors
 4581:061D idle  _hlOsdSetOverlayColorGain
 4581:0633       _hlOsdPixelDoublingEnable
 4581:0687       _hlOsdIsPixelDoublingEnabled
 4581:06D3       _hlOsdComputeOsdSize
 4581:0708       _hlOsdCaptureOverlap
 4581:073D       _hlOsdUpdateDuringBlankingPeriod
 4581:07CB       _i_hlOsdGetOsdConfig
 461D:0007       _hlInfraredInitialize
 461D:001C       _hlInfraredSetTimeBase
 461D:0083       _hlInfraredGetData
 461D:0115 idle  _hlInfraredInitializeEdgeDetectMode
 461D:012A idle  _hlInfraredGetPulseWidth
 461D:016B idle  _hlInfraredSetIRPOL
 464A:000B idle  _hlSetMiscChipSelectBaseAddress
 464A:0043 idle  _hlMiscChipSelectEnable
 464A:0070       _hlGetInternalCpuRamSize
 4655:0003       _dv2wireInitialize
 4655:0009       _dv2wireReserve
 4655:007D       _dv2wireBlockWriteAddress
 4655:0115       _dv2wireBlockWrite
 4655:0195       _dv2wireBlockReadAddress
 4655:0281       _dv2wireBlockRead
 46E0:0008 idle  _TestLEDops
 46E0:0038       _dvLEDInitialize
 46E0:013B idle  _dvLEDSet
 46E0:017B idle  _dvLEDGet
 46E0:0189       _dvLEDSetStateSingle
 46E0:01C4 idle  _dvLEDSetStateMultiple
 46E0:0513       _dvLEDUpdateLEDs
 46E0:0514       _dvLEDBlinkPause
 46E0:0526       _dvLEDBlinkResume
 4760:0007       _dvOemLampBacklightInit
 4760:000A       _dvOemLampSetLevel
 4760:000B       _dvOEMLampGetLampRange
 4760:0028       _dvOemLampEnable
 4760:003A       _dvOemLampGetEnable
 4765:0008       _dvOemUnitPowerSet
 4765:0013       _dvOemUnitPowerIsOn
 4767:0001       _RenderBlitMap
 4767:0087       _RenderBlitMapMenuItems
 4767:0127       _BlitMapSetTranslucent
 4767:013F idle  __BlastBits
 483F:0000       _pwOpPrintfIsStringFormatted
 483F:002A       _pwOpPrintf
 4934:0008       _dvIRremoteInitialize
 4934:005A       _dvIRProcessJoystickCommand
 4934:0081       _dvIRProcessKeycodeCommand
 4934:00A5 idle  _dvIRAnyKey
 4948:0001       _pwOSDGetOpDescriptor
 4948:00D7       _pwOSDIsOpAvail
 4948:0136       _pwOSDGetOp
 4948:0197       _pwOSDSetOp
 4948:0289       _pwOSDExecuteAction
 4975:000A       _uiBhvMenuID
 4975:0016       _uiBhvMenuItem
 4975:0022 idle  _uiBhvControlType
 4975:002D       _uiBhvBoundOp
 4975:0039       _uiBhvBoundTarget
 4975:0045       _uiBhvBoundOpType
 4975:00A9       _uiBhvBoundValue
 4975:0106       _uiBhvGetRectangle
 4975:01F7       _uiBhvControlItemID
 4975:0203       _uiBhvIsContainerMenu
 4998:0004 idle  _uiGetFirstControl
 4998:001D idle  _uiGetNextControl
 4998:0030       _uiGetFirstMenu
 4998:0051       _uiGetNextMenu
 4998:00CF       _uiGetFirstMenuItem
 4998:0292       _uiGetNextMenuItem
 4998:031B       _uiGetFirstMenuItemBound
 4998:0372       _uiGetNextMenuItemBound
 4998:03E3       _uiGetFirstBoundControl
 4998:0404       _uiGetNextBoundControl
 4998:047B       _uiGetFirstTopLevelControl
 4998:049C       _uiGetNextTopLevelControl
 4998:0509       _uiGetControlByID
 4A00:0009       _uiCtlGauge
 4A4F:0005       _uiCtlNumber
 4A71:000A       _uiCtlButton
 4A86:000F       _uiCtlText
 4A9E:0003       _uiCtlDynamic
 4B37:000F       _uiCtlBorder
 4B4E:000F       _uiShowPaneByIndex
 4B4E:0010       _uiHidePaneByIndex
 4B4F:0001       _i_pwSrcAutoPositionCancelAuto
 4B4F:0008       _i_pwSrcAutoPositionClearData
 4B4F:000F       _i_pwSrcAutoOptimizePosition
 4B8D:000D       _i_pwSrcAutoFreqPhaseCancelAuto
 4B8D:0014       _i_pwSrcAutoFreqPhaseInitialize
 4B8D:0278       _i_pwSrcAutoFreqPhaseClearData
 4B8D:02D5       _i_pwSrcAutoOptimizePhaseGPort
 4B8D:02FF       _i_pwSrcAutoOptimizeFrequency
 4C81:0009       _i_pwSrcAutoBrightContClearData
 4C81:0010       _i_pwSrcAutoBrightContCancelAuto
 4C81:0017       _i_pwSrcAutoOptimizeBrightnessAndContrast
 4CD7:0002       _hlHiColorDrawBitmap
 4CD7:0116       _hlHiColorRgbToPacked
 4CD7:013E       _hlHiColorRefToPacked
 4CD7:015D       _hlHiColorPackedToRef
 4CD7:019C       _hlHiColorDrawTiledBitmap
 4D39:0001       _SetDataTransferInfo
 4D39:0089 idle  _OutputByteBlock
 4D39:00BF       _OutputByteBlocksSkip
 4D39:01CD       _OutputWordBlock
 4D39:020B       _OutputRleByteBlockRLE
 4D39:0427       _OutputRleWordBlockRLE
 4D85:0000       _dvIRDriverInitialize
 4D85:01AB       _dvInfraredGetRepeatCount
 4D85:01B9 idle  _dvInfraredSetRepeatCount
 4D85:01C4       _dvIRSetKeycode
 4D85:01CF       _dvIRGetKeycode
 4D85:020E       _dvIRGetJoystickData
 4D85:024F idle  _RepeatValid
 4DD0:0003       _dvKeypadDriverInit
 4DD0:0027       _dvKeypadPoll
 4DDC:0000 idle  __romdata_end
 4DDC:0000 idle  __romdata_start
 4DDD:0000       __romfardata_end
 4DDD:0000       __romfardata_start
 4DDE:0000 idle  __romfunction_start
 4DDE:0000 idle  __romfunction_end
 4DDF:0000 idle  __ramfunction_start
 4DDF:0000 idle  __ramfunction_end
 4DE0:0000 idle  _DATASEG@
 4DE0:0000 idle  __data_start
 4DE0:0020 idle  __Exception_list
 4DE0:0022 idle  __8086
 4DE0:0080 idle  __exitbuf
 4DE0:0084 idle  __exitfopen
 4DE0:0088 idle  __exitopen
 4DE0:00C8 idle  _GPMonitorVSyncData
 4DE0:01C7 idle  _Timer_No_Signal
 4DE0:01DF       _m_wPipLeftPos
 4DE0:0316 idle  ___brklvl
 4DE0:0318 idle  ___heapbase
 4DE0:03F0 idle  _m_dwCurrentChannel
 4DE0:0416 idle  _m_bSignalCallingTask
 4DE0:0424       _m_InputClipWindow
 4DE0:042C       _m_OutputDispWindow
 4DE0:0434       _m_OriginalScaleModeInputWindow
 4DE0:043C       _m_nHorzStretch
 4DE0:043E       _m_nVertStretch
 4DE0:0440       _m_wNLFlags
 4DE0:0442       _m_nHorzLinearRegion
 4DE0:0444       _m_nVertLinearRegion
 4DE0:0508       __ctype
 4DE0:060A idle  __ScanTodVector
 4DE0:060A idle  __RealCvtVector
 4DE0:0614       _uistid
 4DE0:0616       _sctlid
 4DE0:0618       _bgndid
 4DE0:061A       _uitmid
 4DE0:061C       _o2semid
 4DE0:061E       _bksemid
 4DE0:0620       _txsemid
 4DE0:0622       _rxsemid
 4DE0:0624       _scsemid
 4DE0:0626       _hssemid
 4DE0:0628       _hlsemid
 4DE0:062A       _iosemid
 4DE0:062C       _gpsemid
 4DE0:062E       _vpsemid
 4DE0:0630       _dmsemid
 4DE0:0632       _dpsemid
 4DE0:0634 idle  _ursemid
 4DE0:0636 idle  _ussemid
 4DE0:0638       _gisemid
 4DE0:063A       _o3semid
 4DE0:0640 idle  __bss_start
 4DE0:0640       __stklen
 4DE0:0F32       _g_pGlobals
 4DE0:10F6       _m_HSINPOL_ACTIVE
 4DE0:113C       _m_b60Hz
 4DE0:126C idle  _afcCOUNT
 4DE0:1274 idle  _m_TunerVideoAudioStandard
 4DE0:1290       _m_bSystemPowerOff
 4DE0:1292 idle  _Start_Always_Power_Off_Timer_Flag
 4DE0:12F8       _m_cPannelType
 4DE0:12F9 idle  _m_cUserScaleMode
 4DE0:12FA       _m_bTimerOnFlag
 4DE0:15E8       __atexitcnt
 4DE0:15EA       __atexittbl
 4DE0:160A idle  _errno
 4DE0:1A24 idle  _m_wOutThreshold
 4DE0:1A26 idle  _m_wBytesToWrite
 4DE0:1A5E idle  _m_nXOffset
 4DE0:1A60 idle  _m_nYOffset
 4DE0:1C60 idle  __nvram_start
 4DE0:1C60       __staticdata_end
 4FA7:0000 idle  __stack_bottom
 4FA7:0000 idle  _STACKSEG@
 4FA7:0000 idle  __stack_segment
 4FA7:0100 idle  __stack_top
 4FB8:0000       __fardata_start
 4FB8:0000       __fardata_end
 4FB9:0000 idle  __farconst_start
 4FD6:0000       _g_drvRS232DriverVTable
 4FD8:0000       _g_drvOutputScalerDriverVTable
 4FDA:0000       _g_drvImageMemoryDriverVTable
 4FDC:0000       _g_drv24CxxDriverVTable
 4FDE:0000       _g_drvDPortDriverVTable
 4FE0:0000       _g_drvInputPortDriverVTable
 4FE2:006C       _g_drvckPG18E1DriverVTable
 4FED:0004       _g_drvadAD9883DriverVTable
 500E:0007       _g_drvvdVPC3230DriverVTable
 5010:0000       _g_drvTMDSGenericDriverVTable
 5030:000D       _g_drvdePW1230DriverVTable
 5033:0000       _g_drvZ86129DriverVTable
 5035:0000       _g_drvTDA9851DriverVTable
 5037:0000       _g_drvSwitcherSHASTA2DriverVTable
 503F:003C       _g_drvColorSpaceDriverVTable
 5044:0000 idle  _m_cVideoFormatSTD
 5044:0006 idle  _m_wCableChDivideRF
 5044:0012       _g_drvFI1256DriverVTable
 5047:0000       _g_drvdeTDA9885DriverVTable
 5066:0000 idle  _m_VolumeControlTable2
 5066:0065 idle  _SCART_INPUT_PRESCALE_DEFAULT
 5066:0066 idle  _SCART_INPUT_PRESCALE_TV
 5066:0067 idle  _SCART_INPUT_PRESCALE_AV
 5066:0068 idle  _SCART_INPUT_PRESCALE_YPbPr
 5066:0069 idle  _SCART_INPUT_PRESCALE_PC
 5066:006A       _g_drvNJW1144DriverVTable
 5116:0000 idle  __farconst_end
 5117:0000       __farbss_start
 5117:0000       __farbss_end
 5118:0000       __farheap_start
 5118:0000 idle  __farheap_end


Program entry point at 0000:0000

